:109C6A00414952434F544543004256332E33342020
:109C7A00524F4D004241542000532F4E2146414934
:109C8A004C555245005245454E54455221532F4E8C
:109C9A0000434F4E5441435420414952434F544587
:109CAA004300475053004032444000403344400090
:109CBA004F5052214E4F55404D454E55000A160001
:109CCA000180000300007E0000FE00001E00003636
:109CDA000003E60001C4000000000FFFE043415505
:109CEA005440534154454C200043414C4942404161
:109CFA004C542300504943545552450052414E4B4F
:109D0A00494E47004D415020202020200043454E17
:109D1A00544552202000564152494F2020200042EB
:109D2A0041524F4752414D00525554452020202060
:109D3A00004C414E474120202000504354215452A8
:109D4A005345004D4152434152452000494553492C
:109D5A005245200020202021444953212020202040
:109D6A004D45440020545241434B214F4E20200080
:109D7A0020545241434B214F464620004D41524BFD
:109D8A000020545241434B2D5550212000204E4F64
:109D9A005254482D555021200021494553495245D6
:109DAA0001525554414053454C43015345542041B7
:109DBA004C5449444E015A424F52555249206869FF
:109DCA00015A424F5255524921544F54015043545B
:109DDA002154525345556869015255544520202053
:109DEA00206869014149525350414345686901530A
:109DFA004554415249202068690053455421414C39
:109E0A005449444E4500414C54444E452142415226
:109E1A004F00414C5449444E452147505300514E3E
:109E2A004820202020402148504100464C0041470C
:109E3A00454E44412020474F414C41003E4945533D
:109E4A004952450049455349524501524153504EE2
:109E5A0053015452494D4954015354455247200025
:109E6A002149455349524501434F4D3A202020206C
:109E7A00202001544E432031232035374B01544EC4
:109E8A004320312320392E360101505743403130C7
:109E9A00234035374B015057434031302340313945
:109EAA004B01014D5850403130234035374B014D5D
:109EBA0058502034232035374B014D585020312338
:109ECA002035374B014D5850403130234031394B02
:109EDA00014D58502031232031394B002149455337
:109EEA004952450150554E4354204E4F5501454461
:109EFA0049542050554E435401535445524721501A
:109F0A00554E43540101434F4D3A015052494D4970
:109F1A00524521504354015452494D49542050430B
:109F2A0054015452494D40544F5440504301014446
:109F3A004953542050432D504301535445524740EE
:109F4A00544F5440505400444953542021425247DC
:109F5A000053414C562000504F5A2041435455411A
:109F6A004C412E0053544F43202020202020002013
:109F7A0053544F52452157505420002046554C4CBB
:109F8A002000214053544552474500534552200072
:109F9A004952444100555342200055534220004C37
:109FAA00495354005452494D002045524F4152459D
:109FBA00205452414E534D49540021494553495268
:109FCA004501525554414053454C43015043542195
:0D9FDA0052555441214E4F01454449542039
:109FE700525554412001525420494E56455253412F
:109FF700015354455247215043542152015354456C
:10A00700524720525554410143594C20524144492B
:10A01700555301434F4D3A015052494D495245203E
:10A027005254015452494D49542152555441014308
:10A037004845434B20525500525554412153454CF6
:10A047004354004E404F405500204E4F5540504F0F
:10A05700534021002140494E564552532040004964
:10A067004E564552530053544552472150435400CE
:10A077005354455247205254004E4F204520474FD6
:10A087004C2020005452494D49544052540020203E
:10A097005241444955530021494553495245014CC2
:10A0A7004F4144404354522150430156494557407C
:10A0B7004354520144454C40414C4C2143545201B6
:10A0C70001434F4D3A015245435620204354520114
:10A0D70053454E4420204354520056494557204388
:10A0E70054520020204D4F56450020204D4F5645D5
:10A0F70020544F005343414C452020582F592020CE
:10A107004558495400434C52204449535400415543
:10A11700544F43454E54004155544F204F46460037
:10A127002020205343414C450044495354204B4D74
:10A137000044495354204E4D002149455349524547
:10A1470001564152494F2020206869015345544127
:10A15700524520586869015254452D53455420688B
:10A16700690147454E4552414C20686901504943B2
:10A1770054555245536869010101454153592D53BF
:10A187004554015345542146414252494341015ADE
:10A19700424F522054455354200144454C21414CD1
:10A1A7004C21464C490021494553495245015349E1
:10A1B7004E4B544F4E4501434F42212D20014D4FE9
:10A1C7004440434F422001434F4240494E562001ED
:10A1D700564152205443402020402301564F4C55AE
:10A1E7004D4501564152494F204E554C4C0150495F
:10A1F70054434801504552494F440156415220416A
:10A207005640203040230154454320202040303021
:10A21700402501534F554E44434845434B0053494E
:10A227004E4B21544F4E450053494E4B54214F46F8
:10A2370046004E4F542150524553454E5400544505
:10A24700535420564152494F004C494E49535445A7
:10A25700403130404D494E20202000494E41494E63
:10A2670054452044452054455354002149455349FA
:10A27700524501494E524547495354014155544FA0
:10A2870043454E5401014D45442F4449535401461B
:10A29700494E4554452020014C2F44010157494E52
:10A2A7004421542D55500143454E5421542D5550AA
:10A2B70001574159505421425247002149455349BA
:10A2C70052450153544152544054494D4501464962
:10A2D7005253540144454C544120203A014D554CAA
:10A2E7005449504C45014C4153540143594C53492F
:10A2F7004740202040230153454C40524F55544579
:10A307000101010143594C520143594C20542D5529
:10A317005000214945534952450101554E495401C1
:10A32700434C49434B40302C40202301434F4E546C
:10A3370052415354014E4D45412131383301494D66
:10A34700502F414750530101432D564152494F0168
:0DA357004D454D4F525944554D50004D4558
:10A364004D4F525944554D5000455849535441217D
:10A3740050435421545241534555005043542154A1
:10A384005253455500204945534952452021005018
:10A3940052494D495245004C49424552003C2D20FA
:10A3A4004C495354202D3E202045584954005345D0
:10A3B4004C004E455854004E4558542054505400B7
:10A3C400505245562054505400434C5220404C4562
:10A3D4004700434C52204053554D00494E43484991
:10A3E4005320202020200020494E4300455345435C
:10A3F4002047505320002053544F43202020005224
:10A4040055544120004C414E47412020004C4953B3
:10A4140054410054534500414C544030005255546B
:10A424004120474F414C410020544F4F404D55432C
:10A4340048200021404C4953544053454C0020507F
:10A4440043544053454C40210021405052494D490A
:10A45400524540002020404F204B40202021004FF7
:10A464004B00564152004649580047415445215833
:10A47400004C4E45205354415254200053544359E8
:10A484004C2000404F46460054502000406A40494A
:10A494004E20004067404F555400204553554152CB
:10A4A4004520210020494553490045444954004072
:10A4B4004440414000454449542020204E4F5520FB
:10A4C4002053544F43004E4558542053454C454364
:10A4D400542045584954005843542D464C49474844
:10A4E4005420005553454400454E54455220004DD8
:10A4F4004D2E4D4D4D20004D4D2753532E53005797
:10A504004753213834002040554054404D402000EA
:10A51400554054404D002055544320004C4F434176
:10A524004C005357495353474400414C540053552E
:10A5340049405800415647402030402300353030D0
:10A54400003136343000205D203130404B632F70B1
:10A55400005D2020203140632F2300205D20203522
:10A56400404B5453005D203230304046504D004043
:10A574006340204B63004654204B630040634020FB
:10A584004E4D004654204E4D004D2F530032303076
:10A594005E003530305E003122003222003322006A
:10A5A400352200382200464C3700464C31360046EE
:10A5B4004C333300464C363500463130300046319A
:10A5C40036300046323630005E252640534F470071
:10A5D4005E25264054415300414C540056415200DC
:10A5E400225E2F24004B545300532F4E002224008C
:10A5F4004B5400225E004E4D00302C3500312C307F
:10A6040000322C3000302C3600312C3200322C3504
:10A6140000332C3800372C350040313500403330BE
:10A6240000403630005441534B00464C2D444154B5
:10A634004500545000544F46005354410046494E7F
:10A64400004C414E00534554204F46465345540058
:10A6540049534120484549474854004155544F2DDA
:10A66400474F200053544152540020434845434B24
:10A6740040414C4C005241442044495354004053FF
:10A68400454C404845494748543A00475053404296
:10A6940041524F40414C4C0053494E4B40312D32B6
:05A6A40021632F2300DB
:1064F400304D2475A7049005C2E0F51CE0F51DE0BD
:10650400F51EE0F51FE0F56DE0F56EE0F56FE0F5E2
:10651400541270B6126AF42275C70375C6E475B9CD
:1065240001E5BCB481431270B61256DC8E628F63EF
:106534007568F97569001265CA203C2D203B2B1241
:1065440066FF1266D3856D1C856E1D856F1E85548E
:106554001F126636203C12203243201D231266FF90
:10656400126AF4E532242850DC22126636203CF903
:10657400203DF6203205201DBD80EF301DB880EA95
:106584001266FF126AF4856D1C856E1D856F1E856B
:10659400541F1266E9126AF4203DCE8099126922D2
:1065A400201D0D7553107400126885203DBB808634
:1065B400E553540FC553C4540F20350512679A8010
:1065C40003126885808BC23CD23B126686FD12663C
:1065D40086FC126686C39573F565EC9574F564EDD7
:1065E4009575600504600A800EE56424E05011800E
:1065F40006E56424204009126686126686026686D1
:10660400126686FD126686FC126686C39576F56769
:10661400EC9577F566ED9578600904600122E566EE
:10662400F48002E5668562F0A474E025F04002C2BD
:0D6634003B22C23C126686A2E7923DA2E620
:10664100921DA2E592324026A2E492E592E692E7FB
:10665100FC1266862565F565EC3564F5641266867F
:10666100FC1266862567F567EC3566F56622A2E4BD
:106671009235540F79C6F712668609F7301D051257
:106681006686F55322E5697023E56860302404408D
:106691002CE56875F004A485F0C7F5C675B901E568
:1066A100BCB4811985BD68756902801E54037010E0
:1066B10005C675B901E5BC056953690F22D23C22B3
:1066C100147004E5BD80F0147004E5BE80E9E5BFF7
:1066D10080E575A7009006F6E56DF0A3E56EF0A3E1
:1066E100E56FF0A3E554F02275A7009006F6E0F5FA
:1066F1006DA3E0F56EA3E0F56FA3E0F55422E56428
:10670100B2E7F56D85656EAB67E566FC30E707C3FB
:10671100E49BFBE49CFCAA62A9631253DCE56630AE
:10672100E707C3E49DFDE49EFEEEB2E7F56F8D54ED
:106731002275380C12698B1269D6D553012275382E
:106741000C12695C1269CCD55301227538001269AB
:0E6751007412699BD553012275380012695CE1
:10675F0012699BD553012275380312698B126A0790
:10676F00D553012275380312695C1269FDD55301A7
:10677F002275380F126974126A2CD553012275389D
:10678F000F12695C126A2CD553262290679F2373D0
:10679F008091807780688059804A803B802C801D53
:1067AF00800E80DA80CB80BC80AD809E808F808011
:1067BF0075381512698B126A4ED55301227538152B
:1067CF0012695C126A43D553012275380912697434
:1067DF00126A14D553012275380912695C126A14B2
:1067EF00D553012275380612698B1269BED5530134
:1067FF002275380612695C1269B3D55301227538B8
:10680F00121269741269E4D5530122753812126994
:10681F005C1269E4D553012202673275381512698B
:10682F008B126A4ED553012275380F12695C126AAA
:10683F002CD553012275380F126974126A2CD55357
:10684F00012275380312695C1269FDD55301227557
:10685F00380312698B126A07D5530122753800125B
:10686F00695C12699BD55301227538001269741245
:10687F00699BD553262290688A2373809E80A980B6
:10688F00B480BF80CA80D580E08010801B802680B6
:10689F0031803C80478052805D806875380C12696A
:1068AF005C1269CCD553012275380C12698B1269B1
:0E68BF00D6D553012275381212695C1269E4B5
:1068CD00D55301227538121269741269E4D553013A
:1068DD002275380612695C1269B3D55301227538D9
:1068ED000612698B1269BED55301227538091269DA
:1068FD005C126A14D5530122753809126974126A33
:10690D0014D553012275381512695C126A43D5539B
:10691D00012202682A78C686040886037AED12538E
:10692D009A78CAA60408A60378C686040886037A50
:10693D006212539A78CCA60408A60378C68604087A
:10694D0086037AB512539A78C8A60408A603227551
:10695D001A6A751B0A78CA8618088619126B9F78F1
:10696D00CC86060886072278C88618088619E4F5AD
:10697D001AF51B126B9F78C886060886072278C603
:10698D008618088619751A00751B01026B9FE51D87
:10699D002519F51DE51C3518F51CC3E51F9FF51FC1
:1069AD00E51E9EF51E22C3E51F9FF51FE51E9EF5F4
:1069BD001EC3E51D9519F51DE51C9518F51C22E561
:1069CD001D2FF51DE51C3EF51CC3E51F9519F51F83
:1069DD00E51E9518F51E22C3E51D9FF51DE51C9EB0
:0969ED00F51CC3E51F9519F51F07
:1069F600E51E9518F51E22E51F2FF51FE51E3EF52F
:106A06001EE51D2519F51DE51C3518F51C22C3E5E7
:106A16001D9519F51DE51C9518F51CE51F2FF51F8D
:106A2600E51E3EF51E22E51D2FF51DE51C3EF51C57
:106A3600E51F2519F51FE51E3518F51E22C3E51DB0
:106A46009FF51DE51C9EF51CE51F2519F51FE51E86
:106A56003518F51E22E51A7009E51B70058C068DA2
:106A66000722ED851BF0A4A2F792D5ED851AF0A4B6
:106A7600AEF0FFEC851BF0A4A2D53FEE35F0FF92F9
:106A8600D5EC851AF0A42FFFE435F030D50104FECD
:106A960022E4F51AF51BEF4E7003051B22EF65196C
:106AA6007006EE65187001227808C3EF33FFEE33E7
:106AB600FEEF9519F5F0EE95184003FEAFF0E51AD6
:106AC60033F51AD8E5F4F51A751BFF7805C3EF33CD
:106AD600FFEE33FEEF9519F5F0EE95184003FEAF85
:036AE600F0E51BBD
:106AE90033F51BD8E5F4C403F51B22E51D9511E523
:106AF9001C9510500BE56E9511E56D95105001220E
:106B0900E51F9511E51E9510500BE5549511E56F9C
:106B19009510500122E51D9513E51C9512400BE5D2
:106B29006E9513E56D9512400122E51F9513E51E3B
:106B39009512400BE5549513E56F951240012253C8
:106B49002CF8C3E51F9554FFE51E956FFE92605022
:106B590007C3E49FFFE49EFEC3E56E951DF519E5A5
:106B69006D951CF5189261500BC3E49519F519E45C
:106B79009518F518C3E5199FE5189E9262500AE524
:106B890018CEF518E519CFF519126A97E52C5407AF
:106B990075F003A4F538E538906BA573026BBD0257
:106BA9006BD1026BDF026BF7026C0A026C1D026C7F
:106BB9002B026C43851C16851D17C3E4951FF5151B
:106BC900E4951EF514026C56851C16851D17851E45
:106BD90014851F158077C3E4951DF517E4951CF5F9
:106BE90016C3E4951FF515E4951EF514805FC3E4FB
:056BF900951DF517E4F5
:106BFE00951CF516851E14851F15804CC3E4951F34
:106C0E00F517E4951EF516851C14851D158039851E
:106C1E001E16851F17851C14851D15802BC3E49524
:106C2E001FF517E4951EF516C3E4951DF515E495AD
:106C3E001CF5148013851E16851F17C3E4951DF5CC
:106C4E0015E4951CF5148000C3E5179513E516950C
:106C5E001210D70122E5159513E514951210D701E0
:106C6E0022E519F92517FFE518F83516FED3EF952D
:106C7E0011EE9510500122E5119517FDE5109516B0
:106C8E00FC402A4D6027126A5BE5152FF515E514B9
:106C9E003EF514E5159513E514951210D70122E56E
:106CAE00199DF9E5189CF8851016851117E5172919
:106CBE00FFE51638FEE5139FE5129E500BC3E51354
:106CCE009517F9E5129516F8E51A700AE51B700688
:106CDE00AA00AB018013E9851AF0A4E5F0FBE88564
:106CEE001AF0A42BFBE435F0FAE5152BFBE5143A6C
:066CFE00FAE5119BE51010
:106D04009A10D70122EB9515FDEA9514FCC3E515FD
:106D14009511E514951010D717E5139BE5129A50B9
:106D240036E5139515FFE5129514FE126FD38027EF
:106D3400EB9511FFEA9510FEAA00C001126FD3D0A3
:106D440003E5172BFBE5163AFAEB99F517EA98F5E4
:106D540016851115851014C2D5E5466002D2D5AA50
:106D640056E98AF0A4ABF0E88AF0A42B30D5047578
:106D7400F00384F8700122E5172513FDE51635129A
:106D8400FCED8AF0A4ABF0EC8AF0A42B30D50475AA
:106D9400F00384FEE5152513FDE5143512FCED8A98
:106DA400F0A4ABF0EC8AF0A42B30D50475F0038486
:106DB400F9E538906DBB73026DD3026DDF026DE8A7
:106DC400026DF1026DF7026E03026E0A026E0FC3CA
:106DD400743E9EFFC3743E99FE8032C3743E9EFF90
:106DE400AE018029AF06C3743E99FE8020AF06AE83
:0D6DF40001801AC3743E9EFEC3743E99FFD9
:106E0100800EC3743E99FF8007C3743E9EFEAF019E
:106E110008EF2437FFE51B7007E51A700CE8800EB8
:106E2100A2E7E51A50030460F488F0A4E5F06001DC
:106E310004F923FA98FBC3E998C333F9906E43E54B
:106E41003873026E5B026E88026EBD026EEA026FDB
:106E510017026F44026F71026F9E05A7800BEB3022
:106E6100E7032A8002291E1FFBEEC45403F583EEBB
:106E71005408C42FF582EE5407243883F5F0E04519
:106E8100F0F0D8DA05A72205A7800BEB30E7032A3B
:106E91008002290E1FFBEEC45403F583EE5408C48F
:106EA1002FF582EE5407240B83F5F0E045F0F0D87E
:106EB100DA05A722804020100804020105A7800BF3
:106EC100EB30E7032A8002291E0FFBEEC45403F5C1
:106ED10083EE5408C42FF582EE540724EC83F5F0B9
:106EE100E045F0F0D8DA05A72205A7800BEB30E7E3
:056EF100032A800229C4
:106EF6000E0FFBEEC45403F583EE5408C42FF5823F
:106F0600EE540724BF83F5F0E045F0F0D8DA05A784
:106F16002205A7800BEB30E7032A8002291F1EFB00
:106F2600EEC45403F583EE5408C42FF582EE5407DD
:106F3600249283F5F0E045F0F0D8DA05A72205A7FC
:106F4600800BEB30E7032A8002291F0EFBEEC454A8
:106F560003F583EE5408C42FF582EE5407246583A7
:106F6600F5F0E045F0F0D8DA05A72205A7800BEB8F
:106F760030E7032A8002290F1EFBEEC45403F58373
:106F8600EE5408C42FF582EE5407243883F5F0E05A
:106F960045F0F0D8DA05A72205A7800BEB30E7030A
:106FA6002A8002290F0EFBEEC45403F583EE540823
:106FB600C42FF582EE5407240B83F5F0E045F0F07C
:106FC600D8DA05A7228040201008040201EC701FC1
:086FD600ED20E740D2E023CFDB
:106FDE0023CF30E7F980357B08801A7B1080167B33
:106FEE002080127B40800E20E4ED20E3EE20E2EFC5
:106FFE0020E1F07B80EE8BF0A4CF8BF0A4E5F02F98
:10700E00FFEC8BF0A4CD8BF0A4E5F02D2499838FAB
:10701E00F0A433E5F033FBE98BF0A4E5F0C88BF078
:10702E00A428F9E435F0F822FFFEFCFAF8F6F4F2A3
:10703E00F0EFEDEBEAE8E6E5E3E1E0DEDDDBDAD901
:10704E00D7D6D4D3D2D0CFCECCCBCAC9C7C6C5C45F
:10705E00C3C1C0BFBEBDBCBBBAB9B8B7B6B5B4B379
:10706E00B2B1B0AFAEADACABAAA9A8A8A7A6A5A465
:10707E00A3A3A2A1A09F9F9E9D9C9C9B9A99999829
:10708E009797969594949392929190908F8F8E8DD0
:10709E008D8C8C8B8A8A898988878786868585845C
:1070AE00848383828281818075A7009070DCE5469F
:1070BE00FA24FA50027A05EA2323F978107F049312
:1070CE00F60809E9DFF99070F4EA93F556227FC2CB
:1070DE00803E7F4680BA7E8C81747D1882E87A303D
:1070EE0085D074608BA08080402010081271000241
:1070FE007356D215D274D273C219C23A1256DC8E9E
:10710E0047757D0075460575520212914612022191
:10711E00E53524EB500E1291467F1990A10C127694
:10712E00F012DD3FE55275F016A4F57012730C7572
:10713E007E151271D77F237E0990A0EA1277021274
:10714E00DD3F10000810010D10021280E212727F56
:10715E0075330180DA1272C475330180D2757E00E8
:10716E001271D77E0090A0FB1277357F237E05909B
:10717E00A0F112770212722812DD3FE55210000FB5
:10718E0010010510028780D5045403F55280CE12EB
:10719E0071D77F237E0B90A129127702E5466007F7
:1071AE001460041412411A12DD3FE5461000081057
:1071BE00010B10021180D860D6154680D2B405029C
:1071CE0080CD054680C902711B75320012DF157F16
:1071DE00017E1190A0E11277357E0012D5D6E57EA4
:1071EE00D26612D62D75170812DA601241597571D2
:1071FE0000C20612D77D741BFFF5177E0F90A130CB
:10720E00305D0390A138127735129189125D0D12FF
:10721E0046BFC20612651C021E03E55260141460BE
:10722E001E1460297F647E2D791C1272721E1FD966
:10723E00F9227F6A7E1F79281272721FD9FA227F75
:10724E00487E2D791C1272720F1ED9F9227F567E3E
:10725E003379281F12DE5A0F0F12DE5A1F12DE5A12
:10726E001ED9F0221E12DE5A0E0E12DE5A1E02DE3B
:10727E005AE552605514606814606D800075709EFA
:10728E001272F98003757000E5732540F573E435CD
:10729E0074F574E43575F575227570161272968054
:1072AE000375702DE5762542F576E5773541F57750
:1072BE00E43578F57822E55260CB1460DC1460E199
:1072CE0080007570441272B2800375705AE5739522
:0972DE0040F573E5749400F574A9
:1072E700E5759400F575227570711272DB80037570
:1072F7007088E5769542F576E5779541F577E578F7
:107307009400F57822E54690732293F540FEAD4749
:10731700E4FFFC12546F8E418F4222020C1830603A
:10732700C07F40120E9E121E1912DD3F1275D1EB5F
:107337007005909E3F800B1273DF90A45850039006
:10734700A49E7F3F7E0412770212DD3F12DE2012D9
:10735700DE5075370990A09E121CFF90736673026A
:1073670002930275260270FA0276020273560273BE
:107377007E0273970273287F2E12168680D17F367E
:107387007E0490A42C12770212DD3F12DE2080BF0C
:107397007F37120E9E121E1912DD3F1275B5124865
:1073A7004FD2AC1000A9306DFA12748F203BCF403A
:1073B700ED7568F97516001274DC40FB1276787F5C
:1073C700367E29E51612D3B612DD3F05161277A8C9
:1073D70078C6B6F7E20275AF7C0512484F12DC5942
:1073E700744112DC6A745312DC27EB12DC48127703
:1073F700BA5003DCE5227515F975160010000EE585
:1074070015602512743140051274585002D3227F3B
:107417003F7E29E51612D3B612DD3F7F1412DE3701
:107427000516E51664F870D4C322127D7075B9018C
:10743700E5BCB4811AE5BDF51570037516F778C676
:0B744700A616127EB9127EB1127EB1B3
:10745200C3027EB1D3227F0575F019D5E0FDD5F0C8
:10746200FA12484F12DC59744112DC6A744212DC7F
:10747200277E0F78C6E60812DC27DEF912DC4B12F3
:1074820077BA400122DF012275F00080CEC23B12A2
:10749200484FD2AC12DBB2204C3CB440F712DBB7FF
:1074A200B4400312DBB7B4412DF53812DBB7B45345
:1074B2002512DBB7FA12DBB7E538701A12DBB7B464
:1074C2000D1412DBB7B40A0EC3E5169A4003027715
:1074D2009FC2ACD23B22C2ACD3221277FE12484FDB
:1074E200D2AC1000F112DBB2204CEBB440F412DB50
:1074F200B7B4400312DBB7B441DCF53812DBB7B4E2
:1075020042D47E1078C612DBB7F608DEF9E5387091
:10751200C512DBB7B40DBF12DBB7B40AB9C2ACC334
:10752200220273567F0A120E9E121E1912DD3F129C
:1075320075B5124868D2AC1000E712DBB7B440F55B
:10754200F53812DBB7B46EED12DBB7E538600A121C
:107552004868744F12DC3380DC124868744012DCD5
:107562006AE51612DC3312DC3D7568F975160012F5
:107572004868D2AC10003912DBB7B440F7F53812C4
:10758200DBB7B44EC07E1078C612DBB7F608DEF960
:10759200124868E5386007744F12DC3380D11276E6
:1075A200780516745112DC3378C6B6F7C212761516
:0C75B200027356751500751603127D67F4
:1075BE0075B901E5BC30E70205160515E515242061
:1075CE0050EB227B007515F9127D7075B901E5BC83
:1075DE00B481010B0515E515240450EC7515011247
:1075EE007D6775B901E5BCB481010B0515E5152460
:1075FE002050EC227F1C120E9E121E5C400675154A
:10760E00F9127615027356E51560372404401A24D4
:10761E001E5019E515240740028027127D70127640
:10762E00510515E515240450F2751501127D677587
:10763E00B901E5BC30E7031276510515E515242096
:10764E0050EA22127666124EE605C6124EE605C6C0
:10765E00124EE605C6024EE674FF800574048001E4
:10766E00E4F5BCF5BDF5BEF5BF22E568606AF5151B
:10767E000515E5152404501D751501127D6775B9A4
:10768E0001E5BC30E70280190515E515242050EB05
:10769E00751500800C241C60F750E0E5152406508B
:1076AE0037E56875F004A485F0C7F5C675BC81E5AD
:1076BE0015F5BDF56878C6B6F70375BD00081276E8
:1076CE00DB1276D51276D586BC0886BD0886BE0836
:0976DE0086BF08124EE605C62223
:10C0880012AEC412C18712828112C10C12828912A7
:10C09800C11902AEC812AEC412C1871282817F5A7A
:10C0A800C23C12816312835F783F79437F607EEAE6
:10C0B80012C17B1282897F6512816312835F783D8A
:10C0C80079417F207E4E12C17B303C2012C33D1245
:10C0D800C198783F794312C0F7783D794112C0F78B
:10C0E80012C33D78D7E65480F675370002935BC3D8
:10C0F800E796FF1819E796FE0809C3E69FF718198F
:10C10800E69EF7227F5B7E0690A5321277351F8068
:10C118000A7F667E14745912D4CF1F127FEC7E39C1
:10C12800E402D4EE7866E620E73418C3E694720891
:10C13800E694045029C318E6941F08E69404401EA8
:10C148007869E620E71818C3E6940E08E6940150CB
:10C158000DC318E6947508E694004002D322C32262
:10C16800E67D0030E7011D08E62BFB18E63CFCE401
:0EC178003DFD22C3EB9FF6F71819EC9EF6F77B
:10C186002212C12C400CE47842F608F67840F608F4
:10C19600F6227864C3E6946AF55708E6944CF55699
:10C1A6000808C3E69458F55B08E694AEF55A753967
:10C1B60000AC56AD57EC12B271784C12B2FFAC5AC5
:10C1C600AD5BEC12B271785012B2FF7F2B7E867D8A
:10C1D600777C1812B236785012B2F312B14212B20C
:10C1E60036785012B2F312B14212B236785012B209
:10C1F600F312B14212B2367F367E847D257C6412FC
:10C20600B236785012B2F312B14212B236784C12EC
:10C21600B2F312B14212B2367F3F7EA27D607C8BB2
:10C2260012B236785012B2F312B14212AF3012AFD8
:10C236003012B30B7F3F7E807D057CE6053912B157
:10C2460042784812B2FF7F2C7E937D477C7F12B2E4
:10C2560036785012B2F312B14212B236785012B298
:10C26600F312B14212B236784C12B2F312B1421244
:10C27600B2367F357EB47DF87CDF12B23678501246
:10C28600B2F312B14212B236785012B2F312B14280
:10C2960012B2367F3F7EED7D227CCD12B236784CCF
:10C2A60012B2F312B14212AF3412AF30784412B266
:10C2B600FF7F317E397D9D7CE712B236784C12B213
:10C2C600F312B14212B236784C12B2F312B14212E4
:04C2D600B2367844C0
:10C2DA0012B2F312AF3412B2367F2C7E377D0C7C49
:10C2EA00A312B236784C12B2F312B14212B23678B5
:10C2FA004C12B2F312B14212B236784C12B2F312A5
:10C30A00B14212AF3412B30B7F3F7E807D027C9F15
:10C31A00053912B142784412B2FF784812B2F312C8
:10C32A00B2A88E428F43784412B2F312B2A88E405A
:10C33A008F4122753900AC42AD43EC12B271784894
:10C34A0012B2FFAC40AD41EC12B271784412B2FFA6
:10C35A007F2B7E537D507C0912B236784812B2F395
:10C36A0012B14212B236784812B2F312B14212B284
:10C37A0036784412B2F312B14212B2367F347EF2E8
:10C38A007DCD7CA312B236784812B2F312B14212B2
:10C39A00B236784812B2F312B14212B2367F3F7EF9
:10C3AA000A7D2E7CAE12B236784412B2F312B14232
:10C3BA0012AF3012AF30784C12B2FF7F2B7E4F7D16
:10C3CA00AF7CB212B236784812B2F312B14212B24C
:10C3DA0036784812B2F312B14212B236784812B223
:10C3EA00F312B14212B2367F357EB17D4B7C951283
:10C3FA00B236784812B2F312B14212B23678441207
:10C40A00B2F312B14212B2367F3F7E497DCD7C45EE
:10C41A0012B236784812B2F312B14212AF3412AFE6
:10C42A0030785012B2FF784C12B2F312B2A88D557E
:10C43A008E568F57785012B2F312B2A88D598E5A6F
:04C44A008F5B786428
:10C44E00E557246AF608E556344CF608E5553404EB
:10C45E00F608E55B2458F608E55A34AEF608E435DE
:03C46E0059F6225A
:1091A90012AEC412983A12AEC87F6690A51412770F
:1091B900331292177F5A78C41291F31291FB78C631
:1091C9001291F31291DE7F6578C81291F31291FB27
:1091D90078CA1291F37E2DE51B12D4EE7E33E51A7F
:1091E90012D4EE7E39E51902D4EE8604088603020C
:1091F90053397E15E51C12D4EE7E1BE51B12D4EE05
:109209007E21E51A12D4EE7E27E51902D4EE7F5AA3
:109219007E01E53A12D4047E0B909C2EE53B930225
:10922900D501E6FF08E6FE08E6FD339217E4500192
:10923900F4FC12B31C75130A75390112B51A78D7E3
:10924900E6C2E775F00A84F9303D02A9F012B31CB1
:109259008913053912B4F330170A053912B5060511
:109269003912B506A80302B2FF12AEC412983AC267
:109279003C7F5A7E0312851012921712DD3F1000AF
:109289000810011510022080EFE53A146004153A20
:109299008003753A3CD23C80DFE53AB43C05753A27
:1092A9000180F2053A80EE7E0312850B7E0B128552
:1092B9001012921712DD3F1000081001151002203C
:1092C90080EFE53BB40205753B158002153BD23CA6
:1092D90080DFE53BB41505753B0280F2053B80EE66
:1092E9007E0B12850B7F5A78C41291F31291FB12EF
:0792F900936412836F78C437
:109300001293BC78C61291F31291DE129396751CDB
:109310000012836F78C61293BC7F6578C81291F3F0
:109320001291FB12936412836F78C81293BC78CAAF
:109330001291F31291DE129396751C0012836F78CE
:10934000CA1293BC303C14E53B24F4500B78C9E6B8
:109350002410F618E63427F61293C212AEC8127E15
:10936000F102DD3FC2247E15E51C128460F51CD29B
:10937000247E1BE51B128460F51B1023E77E21E58C
:109380001A128460F51A1023E67E27E5191284600C
:10939000F5191023E822C2247E2DE51B128460F506
:1093A0001BD2247E33E51A128460F51A1023E77E5F
:1093B00039E519128460F5191023E622ECF608EB62
:1093C000F622129C4678C8E6FE0886073395E0FD33
:1093D000FC12B2367FE87E037D007C0012B51A12C3
:1093E000B23678CAE6FE0886073395E0FDFC12B473
:1093F000F312B2367F807E697D677CFF12B4F3EC96
:1094000012B26D12B2367F3F7E807D0D7C1D12B18F
:109410004212B2367F3D7E407D007C0012B236782B
:10942000BC12B2F312B14212B2367F3E7E807D0092
:109430007C0012AF3412B23678BC12B2F312B142D1
:0994400012B2367F3F7E807D00F0
:109449007C0012AF3012B23678B412B2F312B142C4
:1094590012B1BA783C12B2FF7F407E807D007C0059
:1094690012B236783C12B2F312B14212B39912B267
:10947900367F3F7EA87D007C0012B23678B812B2E2
:10948900F312B14212B14212B2367F407E007D0022
:109499007C0012B236783C12B2F312B14212B3997F
:1094A90012B2367F3F7EC07D007C0012B14212AFFE
:1094B9003412B23678B812B2F312B14212B2367817
:1094C9003C12B2F312AF34785412B2FF12B383785C
:1094D9005812B2FF12B23612B14212B23678C01225
:1094E900B2F312B142784412B2FF785412B2F312B5
:1094F900B399783C12B2FF12B23612B14212B236A7
:1095090078BC12B2F312B142783C12B2FF7F3E7EB0
:10951900C07D007C0012B236783C12B2F312B1421F
:1095290012B2367F3F7E007D007C0012AF3412B24A
:1095390036783C12B2F312B14212B2367F3F7E80C6
:109549007D007C0012AF3412B23678B412B2F31235
:10955900B142787012B2FF78C4E6FE0886073395E7
:10956900E0FDFC12B2367FE87E037D007C0012B577
:109579001A12B23678C6E6FE0886073395E0FDFC76
:1095890012B4F312B2367FE07E5E7DF87CFF12B42E
:10959900F3EC12B26D12B2367F3F7E7F7DE57CC956
:0595A90012B2367870DB
:1095AE0012B2F312B14212B1BA785012B2FF7F3F2B
:1095BE007EF07D007C0012B236783C12B2F312B10E
:1095CE004212B2367F3F7EC07D007C0012AF341255
:1095DE00B236783C12B2F312B14212B2367F3F7EEF
:1095EE00807D007C0012AF34783C12B2FF78BC1242
:1095FE00B2F312B2367F3F7E807D007C0012AF3018
:10960E0012B236783C12B2F312B23678B412B2F30A
:10961E0012B14212B142784012B2FF785412B2F334
:10962E0012B3D1783C12B2FF12B23612B142787434
:10963E0012B2FF7F417E107D007C0012B23678C0E0
:10964E0012B2F312B14212B2367F407E807D007CA0
:10965E000012B236784412B2F312B14212B2367F11
:10966E00417E207D007C0012AF3012B2367844125B
:10967E00B2F312B14212B2367F407E407D007C00C2
:10968E0012B236787412B2F312B14212B2367F4071
:10969E007EA07D007C0012AF3412AF3412AF3012B8
:1096AE00B236785012B2F312B14212B2367850126C
:1096BE00B2F312B14212B2367F3D7E2A7DAA7CAB46
:1096CE0012B14212B2367F3F7E007D007C0012AF97
:1096DE003012B236783C12B2F312B236787012B241
:1096EE00F312B14212B236784012B2F312B1BA127C
:1096FE00B236785012B2F312B14212B2367850121C
:10970E00B2F312B14212B14212B236785412B2F31F
:0C971E0012AF3012B2367F4A7E517DD26D
:10972A007CCB12B14212B2A878AC12B2FF7F407E53
:10973A00007D007C0012B236787412B2F312B14284
:10974A0012B2367F3F7E807D007C0012AF3412B2A7
:10975A0036784412B2F312AF3412B236785012B2DB
:10976A00F312B14212B236785012B2F312B1421267
:10977A00B236785012B2F312B14212B2367F3E7E3E
:10978A002A7DAA7CAB12B14212B236785012B2F3D9
:10979A0012AF3012B236785812B2F312B1BA12B20C
:1097AA00367F4A7E517DD27CCB12B14212B2A812C8
:1097BA00B236AF3AEF3395E0FEFDFC12B2367F4087
:1097CA007E7E7D057C0012B51A12B2367F607E75E8
:1097DA007D587CFF12B4F312B4F378B012B2FF785A
:1097EA00AC751B641298118F1C78B0751B671298A0
:1097FA0011E51C75F00AA42FFF249C50027F007803
:10980A00D7E654802FF62275390012B2F312B23617
:10981A007F0A7E007D007C0012B5C6A81BE513F600
:10982A0008E512F608E511F6335004EFF404FF22B6
:10983A00C23D78647BAC12922BD23D78677BB01222
:10984A00922B129C467F007EE47D577C0012B23632
:10985A0078AC12B2F312B4F312B2367F007E537DA3
:0E986A00077C0012B5C612B25585133B7F80F5
:109878007ECB7DA47C0012B23678B012B2F312B45B
:10988800F312B2367F407E7E7D057C0012B5C6128B
:10989800B255E513F56F04F53A85126E85116D859D
:1098A800106C7F407E7E7D057C0012B236786C128B
:1098B800B2F312B51A12B2367F607E0C7DA27C001C
:1098C80012B23678B012B2F312B4F312B506786C4D
:1098D80012B2FF78AC12B2F3EC12B26D12B2367F4C
:1098E800347E9C7D2B7C5F12B142785412B2FF12F9
:1098F800B383785012B2FF786C12B2F3EC12B26DE7
:1099080012B2367F347E9C7D2B7C5F12B14212B23C
:1099180036785012B2F312B142784012B2FF7F404B
:109928007E007D007C0012B236785412B2F312B178
:109938004212B39912B2367F3D7EC07D007C001280
:10994800B23678BC12B2F312B14212B2367F3E7E02
:10995800C07D007C0012AF3412B23678BC12B2F36C
:1099680012B14212B14212B2367F3D7E407D007C78
:109978000012B23678BC12B2F312B14212B2367F7C
:109988003E7E807D007C0012AF3412B23678BC1265
:10999800B2F312B14212B2367F3F7E807D007C0066
:1099A80012AF3012B236785412B2F312B14212AF7B
:1099B8003012B2367F407E807D007C0012B236784D
:1099C8005412B2F312B14212B39912B2367F3D7EED
:1099D800707D007C0012B23678BC12B2F312B1422C
:1099E80012B23678BC12B2F312B14212B14212AFBF
:1099F8003412B23678B412B2F312B142785812B2B5
:109A0800FF785412B2F312B399783C12B2FF78542B
:109A180012B2F312B3D1785412B2FF783C12B2F3F7
:109A280012B23612B14212B23678BC12B2F312B187
:109A380042783C12B2FF7F3E7EC07D007C0012B2AD
:109A480036783C12B2F312B14212B2367F3F7E0032
:109A58007D007C0012AF3412B236783C12B2F31299
:109A6800B14212B2367F3F7E807D007C0012AF3457
:109A780012B23678B412B2F312B142787012B2FF51
:109A8800785012B2F312B23612B14212B23678C01E
:109A980012B2F312B142784412B2FF785412B2F300
:109AA80012B23612B142787412B2FF784012B2F391
:109AB80012B23612B142783C12B2FF7F407E807DEE
:109AC800007C0012B236784412B2F312B14212B2DC
:109AD800367F417E107D007C0012AF3412B236789A
:109AE8004412B2F312B14212B236787412B2F312BF
:109AF800B2367F407EA07D007C0012AF3012AF34BA
:109B080012B236783C12B2F312B14212B2367F3D2D
:109B18007E2A7DAA7CAB12B14212B2367F3F7E000C
:109B28007D007C0012AF3412B236785412B2F312B0
:109B3800B236787012B2F312B14212B236783C12D1
:109B4800B2F312B14212B14212B236785812B2F3DD
:109B580012AF3412B2367F3F7E7F7DE57CC912B1E9
:019B680042BA
:109B690012B2367F4B7E187D967C8012AF3412B2CA
:109B7900A812B2367FE87E037D007C0012B5C612BA
:109B8900B25578C8A61208A61308A60608A607782B
:109B99007412B2F312B2367F3F7E807D007C0012D0
:109BA900AF3012B236784412B2F312AF3412B23671
:109BB9007F3E7E2A7DAA7CAB12B14212B236784032
:109BC90012B2F312B14212B236783C12B2F312B1A8
:109BD9004212B236784012B2F312AF3412B2367F63
:109BE9003F7E7F7DE57CC912B236787012B2F312DE
:109BF900B14212B14212B2367F487EF47D247C0014
:109C090012AF3412B2A812B2367FE87E037D007C0F
:109C19000012B5C612B25578C4A61208A61308A632
:109C29000608A607223F3F4344454647484A4B4C4E
:109C39004D4E5051525354555657583F3FE4F539FC
:109C4900F5A7909C5A791078B4E493F6A308D9F94A
:109C59002232A5C24A4A19DC3A885CDB3BFFD6DCD2
:019C69003BBF
:10AEC400D2D58002C2D575A70490040078107F0BF8
:10AED40012AEF078267F0512AEF0783C7F2212AED7
:10AEE400F0786A7F0F12AEF075A7002230D506E61F
:10AEF400F008DFFB22E0F608DFFB22D2D58002C295
:10AF0400D575A7049006FA78737F0612AEF075A77C
:10AF14000022DA0CD902800BD906303701B3500570
:10AF240002B0A3923702B08FD9F680F9D2368002EC
:10AF3400C23612B0D4303606C86002B237C8923670
:10AF4400DAD0D9E4B8000A12B11BA236923702B0A3
:10AF54007860FBB51300400F12B11BA23692F7A222
:10AF6400379236A2F79237C398F40424E740DF24DB
:10AF740019AD29AC28AB277A00C394084008CDCC7E
:10AF8400CBCAE4CD80F424086010F9C3ED13FDECC2
:10AF940013FCEB13FBEA13FAD9F1A236303701B3F1
:10AFA40040308A17E5102BF518E5113CF519E51228
:10AFB4003DF51A501A13F51AE51913F519E5181386
:10AFC400F518E51713F5170513E5137002051402B8
:03AFD400B02EE4B8
:10AFD700C39AF517E5109BF518E5119CF519E512CD
:10AFE7009DF51A500DB237C378177F04E496F6081B
:10AFF700DFFA7A047019E513C39408F513500215A4
:10B0070014E4C517C518C519F51ADAE802B0CF2038
:10B01700E7BAE5137002151415137817C37F04E612
:10B0270033F608DFFA80E8E51A20E7137817C37FBD
:10B0370004E633F608DFFAE513700215141513E575
:10B04700173378187F03E63400F6500E08DFF775DC
:10B057001A800513E51370020514E51420E75470F0
:10B0670027E513604E046020851A1285191185188B
:10B07700105326F0AC10AD11A237E51313FFE512FC
:10B0870092E7FEA81302B255E4F512F511F510F593
:10B09700147513FF5326F043260580D8E5FFF512F4
:10B0A700F511F510751400F513D2375326F0432622
:10B0B7000980C15326F0432603E4F512F511F51074
:10B0C700F514F513C23780AC5326F080EC79017A7A
:10B0D700018512F0E513A2F7339237751400F513C3
:10B0E7006002D2F785F012A813B8FF0809E512C26B
:01B0F700E771
:10B0F8006001098C278D288EF0A2F7EF3304700ABF
:10B108000AC2F705F00AD5F0011A146002D2F785D1
:10B11800F02922C88813C512C529C512C511C5282A
:10B12800C511C510C527C51022DA03B8000302B03F
:10B13800A3D9028002D9F702B08F12B0D4303701F8
:10B14800B392377004D9E78005DADEB8000302B09D
:10B15800CFD9E2C3947E500215142513F51350027B
:10B1680005147815760008B81BFA78277915E608CB
:10B17800FAE8FC78108AF0E608A427F709E5F03722
:10B18800F7500989F00907E760FBA9F0B813E61939
:10B1980019ECF8B82AD802B02E02B0BAB8FFFA02F1
:10B1A800B0A3D9FB02B08FDAF6B800F002B0CF1224
:10B1B800B30B12B0D4303701B392377007D9E3B864
:10B1C80000E280DBDAE1B8000280E1D9D5C8C39893
:10B1D80050021514247F50020514F513781A7600CE
:10B1E8007A1A7B80C3E5109527E5119528E5129515
:10B1F800294016C3E5109527F510E5119528F51196
:09B20800E5129529F512E64BF65A
:10B21100DA0302B02EEB03FB30E703187600C3E537
:10B221001033F510E51133F511E51233F51240CA6B
:10B2310030E7DD80B6E53905396010D0F0D0E0C0E7
:10B2410010C011C012C013C0E0C0F08F138E128D58
:10B25100118C1022E539146010D0F0D0E0D013D059
:10B2610012D011D010C0E0C0F01539227920800C25
:10B271007910800479087D007E007F003392D550DB
:10B281000312B2E5EC33400FEF33FFEE33FEED3343
:10B29100FDEC33FCD9EE22EECCF5F0747E29A2D57B
:10B2A10013FF92F7AEF022EF8EF0A2F7D2F73392AE
:10B2B100D5C3947F5006E4FFFEFDFC229420400498
:10B2C10074FF80F304CCFEE4FFFAE5F0CC6012C316
:10B2D100CC13CCCD13CDCE13CECF13CF0450EEDA99
:10B2E100EC30D5D7C3E49FFFE49EFEE49DFDE49CD2
:03B2F100FC22E656
:10B2F400FC08E6FD08E6FE08E6FF22ECF608EDF69B
:10B3040008EEF608EFF622CFC513CFCEC512CECD88
:10B31400C511CDCCC510CC22E4F513F512F511F509
:10B324001022E493FCA3E493FDA3E493FEA3E4932B
:10B33400FFA322C0E012B23612B14212B36A12B3B2
:10B3440026D0E0C0E012B23612B36112B14212B29A
:10B354003612B32612AF34D0E0D5E0E722AC48ADC4
:10B3640049AE4AAF4B228C488D498E4A8F4B22748A
:10B37400FF7809FFFEFDFCE52654F048F52622126D
:10B38400B42A04A2E1927F1420E01590B4AB7404B3
:10B3940012B337802912B42A30E102B27F20E0EBE5
:10B3A4008C4C8D4D8E4E8F4F90B4BF740412B337B6
:10B3B40012B236AC4CAD4DAE4EAF4F12B142307FEF
:10B3C40004EF6480FFEE33EF337001FF2212B42ADE
:10B3D400C0E08C4C8D4D8E4E8F4F90B4E3740312AD
:10B3E400B33712B236AC4CAD4DAE4EAF4F12B14284
:01B3F400EC6C
:10B3F500C54CFCEDC54DFDEEC54EFEEFC54FFF90AE
:10B40500B4D3740312B337D08212B236AC4CAD4DFF
:10B41500AE4EAF4FE58230E00712B1BAB27F809DE4
:10B4250012B1B78098EE33EF3324605007D0E0D0E7
:10B43500E002B373EFA2E7547F927FFF12B2367C2E
:10B44500837DF97E227F3E12B142EE33EF332481B4
:10B45500501012B23612B2A812B26DEFB2E7FF1257
:10B46500AF34EE33EF33602A2403F8C313FFEE92B3
:10B47500E7FEE82481E4501A12B23612B2A8EF04AE
:10B48500C2E0FCF58212B275EFB2E7FF12AF34E508
:10B495008203FAEE33EF33600B148FF0A2F713FF3C
:10B4A500EE92E7FEEA2283FA703AE4E9AABCF8E0F4
:10B4B500813EE6E99DBF0000803F1A3C2839666958
:10B4C50099BBE335A33DE75D25BFDB0FC93FCCDB6A
:10B4D5008D41EE3649C43F91C9453DF8B0C50000E0
:10B4E500803F34F517C373FA2F45DDFD0AC6EF25F6
:10B4F50013FFEE3512FEED3511FDEC3510FC02B2F1
:10B5050055C3EF9513FFEE9512FEED9511FDEC95E4
:10B5150010FC02B255EFF88513F0A4FFE513C5F052
:0AB52500CEF9A42EFEE435F0CDFAB5
:10B52F0088F0E512A42EFEED35F0FDE433CC851343
:10B53F00F0A42CFCE5128AF0A42CFCE51189F0A4F0
:10B54F002CFCE51088F0A42CFC89F0E512A42DFD4D
:10B55F00EC35F0FCE51188F0A42DFDEC35F0FC8AFC
:10B56F00F0E513A42DFDEC35F0FC02B255E4CCF858
:10B57F00E4CDF9E4CEFAE4CFFB75F020C3E5133345
:10B58F00F513E51233F512E51133F511E51033F527
:10B59F0010EF33FFEE33FEED33FDEC33FCEF9BEE9C
:10B5AF009AED99EC98400CFCEF9BFFEE9AFEED990B
:10B5BF00FD0513D5F0C622C2D5EC30E705B2D51282
:10B5CF00B2E5E51030E70DB2D512B5E912B57C1230
:10B5DF00B2E5800312B57C30D515C3E49513F5138E
:10B5EF00E49512F512E49511F511E49510F510227A
:10A6A900E57124885002D2191256DC8E4712D21451
:10A6B900129189125A98305E0F125A3612887812FE
:10A6C900596712C01A12425412393A1247FB10360E
:10A6D90029201F1C301219E412A82F12A84412A90C
:10A6E9004412A96630510302A9F012ACC1205109E4
:10A6F900C251E4F552F545F5442275A70075830763
:10A70900E559C454F0F582E0F538A3E0F518A3A3A0
:10A71900A3E0F51E74FF12A82F1256DC8E1C8F1BA6
:10A729007510DF751100E51164B4700612A7FA758A
:10A73900111012A7C74028AE1CAF1B125764203254
:10A749001EAC03AB027A0C125371ED701275A7009F
:10A75900758304851182ECF00583E510F00511D5A8
:10A7690010C412A7FA75C70375C6E075A70490054A
:10A77900007F0412A7B5DFFB75A700122B83125ABD
:10A7890036E4F5A7F8F559758307E8C4F582E0655D
:10A79900387011A3E06518700BA3A3A3E0651E70C0
:10A7A9000388592208C3E5589850DC22E0F5BCE03B
:10A7B900F5BDE0F5BEE0F5BF124EE605C622E5108F
:10A7C90075F004A4F5C685F0C775B901E5BC334039
:0BA7D9001F05C605C675B90185BE64EA
:10A7E40085BF6505C675B90185BC6685BD6785BE2F
:10A7F4006885BF69C322E51124FE502E75A7007F2A
:10A8040010AE111E7583048E82E0FD1582E0CDB575
:10A8140005005012F00582CDF00583E0FD1582E0BD
:10A82400CDF00582CDF0DEDCDFD72275A75490048D
:10A834000005A79005007FB4F0F0DFFC75A70022A7
:10A8440012BE6EC2517B077AFFE4FFF5A7900400A5
:10A8540012A92AED244C4035EC603075A7008D8296
:10A8640005A712A8F07583058D82E02410401CF022
:10A8740005A7E02CF0500505A7E004F0BA000CBBD6
:10A884000009D251EF24DC50027F23DFC3EA6005C4
:10A8940012A8A38006EB600312A8DB75A700223080
:10A8A400E0047553082230E1047553182230E204A1
:10A8B4007553282230E3047553382230E404755369
:10A8C400482230E5047553582230E6047553682253
:10A8D40030E7037553782230E0047553882230E161
:10A8E400047553982230E2037553AA22ED54F0C440
:10A8F400232390A8FA735302FE225302FD2253022B
:06A90400FB225302F722C2
:10A90A005302EF225302DF225302BF2253027F2255
:10A91A005303FE225303FD225303FB225303FB225C
:10A92A0012BDA612BC34E4F5F7C2B2C2B2ADF7F555
:10A93A00F7C2B2C2B2ACF7D2B22290050078B4E044
:10A94A006015FD54F0C4CD7C00540FFE1583E0FF62
:10A95A0012546FEFF005830582D8E42275830478D8
:10A96A00FF088882E060FAF5D38812E512244C5079
:10A97A00012285D3D288D4881279FF0512E51260A4
:10A98A00F00908E875F0B484A8F08882E060ECF574
:10A99A00D3B9000280D5B9230050D0C395D292D141
:10A9AA005002F40409FEE4FFFCAD0112547C740168
:10A9BA00FA25D475F0B484A8F0AC06AB0712536339
:10A9CA00EB30E7010CE5D22C30D1029C9C8882F056
:10A9DA000AEAB501DCE512244C50012285D3D2855E
:10A9EA0012D4A812809390040012AAAF8C068B0589
:10A9FA0012AAAFE4FFF512F5118C148B13C3ED9B69
:0EAA0A00F9EE9CFA4012E51199E5129A500AF5
:10AA18008C148B138A1289118F528F82E0F9C3ED3F
:10AA280099FDEE9400FEE582245A5002244C75F0FC
:10AA3800B48485F082E0FA2DFDEE3400FEEB9AFB3B
:10AA4800EC9400FCE92BFBEC3400FC0FBFB4B0E540
:10AA58005224D3400224B4F552C3E51333FBE51462
:10AA680033FCE511FE2BFBE512FF3CFC1254D1E947
:10AA7800F890AAC193F511FDEBF513FFECF514FE60
:10AA88007C0012546F8F44E890ABC193FAAB13ACBF
:10AA98001412539AAF03AE04AD117C0012546FEF39
:10AAA8007002F552F545227C007B007F5AE02BFBB3
:10AAB800EC3400FC0582DFF522B4B4B4B4B4B4B409
:10AAC800B4B4B4B4B4B4B4B4B4B4B4B3B3B3B3B343
:10AAD800B3B3B3B3B3B3B3B3B2B2B2B2B2B2B2B246
:10AAE800B2B1B1B1B1B1B1B1B0B0B0B0B0B0B0AF56
:10AAF800AFAFAFAFAEAEAEAEAEAEADADADADADAC71
:10AB0800ACACACACABABABABAAAAAAAAA9A9A9A995
:10AB1800A9A8A8A8A8A7A7A7A7A6A6A6A5A5A5A5C2
:10AB2800A4A4A4A4A3A3A3A2A2A2A2A1A1A1A0A0F9
:10AB3800A0A09F9F9F9E9E9E9D9D9D9D9C9C9C9B33
:10AB48009B9B9A9A9A999999999898989797979672
:10AB580096969595959494949393939292929191B5
:10AB680091919090908F8F8F8E8E8E8D8D8D8C8CF5
:10AB78008C8B8B8B8A8A8A8989898888888787873A
:10AB88008686868585858484848383838282828180
:10AB980081818080807F7F7F7E7E7E7E7D7D7D7CC3
:10ABA8007C7C7B7B7B7A7A7A797979787878777705
:10ABB800777676767575757474000203050608094C
:10ABC8000B0C0E101113141617191A1C1D1F212215
:10ABD800242527282A2B2D2E303133343637393A7D
:10ABE8003C3D3F404243454648494B4C4E4F5052EE
:10ABF80053555658595A5C5D5F606163646667686F
:10AC08006A6B6C6E6F707273747677787A7B7C7E01
:10AC18007F80818384858688898A8B8D8E8F9091A9
:10AC2800929495969798999B9C9D9E9FA0A1A2A46B
:10AC3800A5A6A7A8A9AAABACADAEAFB0B1B2B3B444
:10AC4800B5B6B7B8B9BABBBCBDBEBFC0C0C1C2C338
:10AC5800C4C5C6C7C7C8C9CACBCCCCCDCECFD0D047
:10AC6800D1D2D3D4D4D5D6D7D7D8D9DADADBDCDC6D
:10AC7800DDDEDEDFE0E0E1E2E2E3E4E4E5E5E6E7AD
:10AC8800E7E8E8E9EAEAEBEBECECEDEEEEEFEFF003
:10AC9800F0F1F1F2F2F3F3F4F4F4F5F5F6F6F7F770
:10ACA800F8F8F8F9F9FAFAFAFBFBFBFCFCFDFDFDF4
:10ACB800FEFEFEFEFFFFFFFFFFC251E4F544F8145D
:10ACC800FB900400A9007C0FC2D112ADDCE824057A
:10ACD800F8B8B4F08B13E5122403FA244C5001FAA7
:10ACE800BBFF012275112C8A1912AE138F16203D55
:10ACF80012AA1975112312AE138F15751600303D5F
:10AD0800E2801175112312ADBB751500303D05E8C1
:01AD18002F0B
:10AD190013F51575111212ADBB751400303D05E818
:10AD29002F13F514EA2404F552244C5002F552E489
:10AD3900F51AF51BF51CE516600AFB7A00AF137EC0
:10AD4900FF12AD81E515600AFB7A4FAF137EFF1242
:10AD5900AD81E516600DFB7A00E5146006FF7ECF34
:10AD690012AD81AE1CAF1B7C00AD1A12546F8F451A
:10AD7900EF2513F544D25122EFF5F0A4FCADF0EB29
:10AD8900F5F0A49CFCE5F09DFDEB8AF0A4FAABF08C
:10AD9900EF8EF0A49AF8E5F09BF9E833F8E933F976
:10ADA9007B00125515051AE51B2BF51BE4351CF51F
:10ADB9001C22EA2511F9244C5001F9C2D112ADDA4D
:10ADC900303D428F00C3EA9511F9500324B4F9D2FA
:10ADD900D17C09E4FDFEFF8982E060062FFFE43E95
:10ADE900FE0D09B9B4027900DCEDED20D118F51E8C
:10ADF90024FE923D500F12547CEFB5030050068596
:10AE09001E1FFB881222F51D80E612ADBB203D43B3
:10AE1900740212AEB212ADBB203D38740412AEBA40
:10AE290012ADBB203D2D740612AEB212ADBB203D52
:10AE390022740812AEBA12ADBB203D17740A12AEC5
:10AE4900B212ADBB203D0C740C12AEBA12ADBB20D0
:10AE59003D0122C3E89F605088148F158A16400867
:10AE69001ABAFF0A7AB380060ABAB4027A0012AD96
:10AE7900BB303D34C3E89FF9602EC3E5149515FB3B
:10AE89006930E7D4E930E703F404F9EB30E702F479
:10AE990004C3995002AA16E5142515C82F28FFE402
:10AEA900FC33FE7D0412546F222AFA244C5001FA15
:0BAEB90022C3CA9AFA500324B4FA2204
:10BBFB00758000C2B212DE35D2B275F83022758074
:10BC0B0000C2B2F5F7C2B2C2B2D2B222758000C284
:10BC1B00B2F5F7C2B2C2B2856CF7C2B2C2B2856BD3
:10BC2B00F7C2B2C2B2856AF722758000C2B275F74D
:10BC3B0003C2B2C2B2856FF7C2B2C2B2856EF7C28F
:10BC4B00B2C2B2856DF72212BC8B740612BC09749A
:10BC5B000212BC178FF7C2B2C2B2D2B222909F6E41
:10BC6B007F631276F012DD3FD214120E9412766EB1
:10BC7B00124EE612BC8B740612BC0974C712BC09B7
:10BC8B0012BC9140FB22758000C2B275F705C2B29F
:10BC9B00C2B2C2B2C2B275F705C2B2C2B2C2B2C2AE
:10BCAB00B2E5F7D2B2A2E022120E9485BF6C85BE2C
:10BCBB006B756A00E56B7015E56A701112BC8B74BD
:10BCCB000612BC0974D812BC17D2B2D21F22E54B94
:10BCDB000475F03C8485F04B12BF96852E72E55FA0
:10BCEB00030354C0F8E55E543F28F57C3055012220
:10BCFB0012BD3012BC9140F7E54C60F312BC8B12B5
:10BD0B00BD4712BD1580F112BC8BC21F740612BC4D
:10BD1B0009740212BC17787086F708B880FAD2B291
:10BD2B0012BD64808F787075A704758304E54CC4CD
:0CBD3B00F5827F10E6F0DFFC054C80195B
:10BD4700787075A704758304154CE54C30E701E45A
:10BD5700C4F5827F10E0F6DFFC75A700227410257A
:10BD67006A54F0F56AE4356BF56BE4356C540FF5FE
:10BD77006C22E54B75F010A4256A54F0F56AE5F0DE
:10BD870080E4E56A24F054F0F56AE56B34FFF56B5F
:10BD9700E56C34FF80D7E56A24FF80ECC380EBE5D0
:10BDA7006D24F054F0F56DE56E34FFF56EE56F34F4
:10BDB700FF540FF56F2212BE1512BE3DC22DC2549D
:10BDC700C255E57F7002D255147002D254E54A304D
:10BDD700E00122B4061C20540D12BD8912BEE512E3
:10BDE700BF7512BFAD2212852F7E0412DE2D754A54
:10BDF700012220550D12BD6412BF5412BF9612BE08
:10BE0700BE2212852F7E0412DE2D754A0522740389
:10BE170012BC177870E4F5F7C2B2C2B2A6F708B839
:10BE270080F3D2B222740312BC17E4F5F7C2B2C290
:10BE3700B2E5F7D2B222E575F8541F30E40244E0C8
:10BE4700F57585722EA2779226E57C543F30E50280
:10BE570044C0F55EE57C54C02323F55FE57FC2E768
:10BE670079BCF709A77E22856C6F856B6E856A6D35
:01BE770022A8
:10BE7800856F6C856E6B856D6A22E4FEFF740775AD
:10BE8800A704F5838E8274FFF0DFFD75A700227486
:10BE9800067E007FB012BE87E4F55AF55B2275A7CF
:10BEA80004758306E55A600A75F00A84E5F07002A5
:10BEB800740AC4F58222307720E55A24024002052C
:10BEC8005A12BEA6E55AF0E573F0E574F0E575F090
:10BED800E576F0E577F0E578F075A700223077F998
:10BEE80012BEA67F1074FFF0DFFDE55A24F550035B
:10BEF80012BF10155AE55AB4FF02055AC3E55A9500
:10BF08005B50D6755B0080D112BE6E7F0A056D0549
:10BF18006D12BC34E4F5F7C2B2C2B2E5F7D2B23062
:10BF2800E704DF02800512BDA680E2056D12BC346D
:10BF380012BEA6E55A24F6F07F06E4F5F7C2B2C2AF
:10BF4800B2E5F7F0DFF4D2B275A70022053FE53F6E
:10BF5800B43C17753F00053EE53EB43C0D753E0008
:10BF6800053DE53DB41803753D00024ABB153FE5A4
:10BF78003FB4FF17753F3B153EE53EB4FF0D753ED8
:10BF88003B153DE53DB4FF03753D17024ABB05422D
:10BF9800E542B43C0F7542000541E541B43C0575E6
:0CBFA80041000540221542E542B4FF0FA5
:10BFB40075423B1541E541B4FF0575413B154022EF
:10BFC400AC40AB41A842EC75F03CA42BFBE435F04B
:10BFD400FC7A3C125363EB28FBE43CFC22AC3DAB03
:10BFE4003EA83F80E178AE8604AB3EE53FC313F83C
:10BFF400800C7800120E5DE5BE75F005A4FBE5BF6C
:10C0040075F03CA42BFBE435F0FC7A1E125363EB71
:10C0140028FBE43CFC2212BFF6AE04AD0312BFE9D8
:10C024008C148B13120E67E5BFFF24F650027F01B8
:10C03400E5BE75F096A4AAF0F9C3ED9513FBEE9551
:10C0440014FC924E4B701120110E30480B75364B78
:10C054003003037536FFD22E304E02DF1F7A0212F0
:10C06400536375A7009004EEECF0A3EBF0C3E5BFB7
:10C074009F04BF0102D2E79005CBF022ED29FDEE2B
:04C084003AFE80B54B
:10DE1A0012DE2312DE2312DE237E0480067E0280B7
:10DE2A00027E017F0080087F6480027F017E00EF0E
:10DE3A004E6012E4FD0D1D0DEDC394AD40F7EF1FCA
:10DE4A0070ED1E80EA22753500C200C201C20222AC
:10DF0100F5D8D2DCE5F520E7FBE5DA540FFEAFD911
:04DF110075D800229D
:10DB08007F767E06909C7E127702740412DF017C79
:10DB1800007D5212546FEFF875F00A84C0F07F76DA
:10DB28007E2312D4EE7E29742E12D5017E2ED0E0EB
:10DB380012D4EE7E35745612D5017F6B7E1190DBC0
:10DB48007112D52DE824E04001220423F824E7507F
:10DB580002781812DB61D8FB227F6CE82411FE7969
:10DB68000512DE5A0E0FD9F922071DFFFFFFE080CC
:10DB7800000020C0000038E0000008F0000038F87D
:07DB8800000020FFFFFFE099
:10DB8F0012DBB730E6022409540F75F00AA4F5151D
:10DB9F0012DBB730E6022409540F25152212DBB72A
:10DBAF00540F2275F000800875F044800375F0075C
:10DBBF00E4206D09D5E0FAD5F0F7D24C229247C296
:10DBCF00ACE54F623885504FA26E926D859950C269
:10DBDF006FD2ACC24CA2472212DBF1C4FA12DBF1B6
:10DBEF002A2212DBB720E603540F225407240922FE
:10DBFF00E612DC0618E608FAC412DC0CEA540F44ED
:10DC0F0030F924C6E950112407800D75F00A84C03D
:10DC1F00F012DC25D0E0443030530975F00085E078
:10DC2F00E0D5F0FA3099FDC299F599623822E538BE
:10DC3F0080F2E53812DC06800812DC27E53812DCAA
:10DC4F0027740D12DC27740A80CE744012DC2774FF
:10DC5F004080C5742C80C1742E80BD75380080B88B
:10DF270085A0835383FE438380858384F0758400B3
:01DF370022C7
:10D9B60074A212DF2774A112DF2774A612DF277460
:10D9C600A412DF2774C012DF27742512DF2712DAAC
:10D9D6004675C70375C6FC75B90112B5FF74081202
:10D9E600DF01EE75F020A4FEEF54F80303032E24A6
:10D9F60092C313FE24EA50027E16EE90DA2F932588
:10DA0600BCFE24E6501F24E8401B748112DF27EE7B
:10DA160012DF2712DA53744012DF27742F12DF2722
:10DA260074AF02DF277E2680E1F7F7F8F8F9FAFBF4
:10DA3600FCFDFEFF000000000101020202030303D9
:10DA4600A8BCA9BDAABEABBFACC7ADC62288BC895F
:0ADA5600BD8ABE8BBF8CC78DC622AF
:10DD3F00C006C007C5F075A7019000007EB7E58C3F
:10DD4F00240340FA12DD611EBEAFF3C5F0D007D039
:10DD5F00062275A700EE12DF27741012DF27740456
:10DD6F0012DF2785A08343838185838475A7517F25
:10DD7F0020E0F0E0F0E0F0E0F0DFF6E4F5A7F58466
:01DD8F002271
:10DF150075A711900000E4C583F0C58330E2F8F5DC
:02DF2500A72231
:10DE5A00EF20E723EE20E71F20E61C05A7C45403A2
:10DE6A00F583EE5408C42FF582EE5407240983F58E
:10DE7A00F0E045F0F005A7228040201008040201D6
:10DE8A00EF20E723EE20E71F20E61C05A7C4540372
:10DE9A00F583EE5408C42FF582EE5407240983F55E
:10DEAA00F0E055F0F005A7227FBFDFEFF7FBFDFE9C
:10D4AE00FDA42582F582E5F03583F583ED229060AB
:10D4BE00AC7A0475F00512D4AE7D05805E7A0580D7
:10D4CE00027A04547FC0E0C083C082C3942050010E
:10D4DE00E490605C12D4C1802E9061BA7A0580050A
:10D4EE009062777A0675F00712D4AE7D07802C7A9B
:10D4FE000580027A06C0E0C083C082C3942050012A
:10D50E00E490620712D4F3D082D083D0E022905FF1
:10D51E00D075F00A12D4AE7D0A7A07C2D18002D23B
:10D52E00D1C0A7C082C083C007C006C0E030D109F9
:10D53E0075A704E493FDE493FAEEFB75A704EBFEE6
:10D54E00EAFC7901D9067908E493F5D4E5D423F5FC
:10D55E00D420E01612DE8A0EDCEA0FDDE1D0E0D038
:10D56E0006D007D083D082D0A72212DE5A80E89050
:10D57E005F1075F00E12D4AE7D0E7A0812D529907A
:10D58E005FB875F00212D4AEE493FDE4A393FACE25
:10D59E002408CE7C0812D5AA7C06AD02ED23FD2010
:0ED5AE00E00712DE8A0FDCF42212DE5A80F74C
:10D39900F5D2C2D58036F5D2D2D58030F5D224F671
:10D3A90050090E0E24A650030E0E0EE5D2F5D275C5
:10D3B900F0648485F0D3C2D57009D2D5742012D512
:10D3C90001800312D4EECE2406CEE5D375F00A848B
:10D3D90085F0D3700A30D507742012D50180031265
:10D3E900D4EECE2406CEE5D312D4EEE5D222F5D280
:10D3F90075F0648485F0D3C2D58022F5D2C2D58078
:10D4090025F5D2D2D5801FF5D275F0648485F0D385
:10D41900C2D57009D2D5742012D501800312D4E780
:10D42900CE2405CEE5D375F00A8485F0D3700A3091
:10D43900D507742012D501800312D4E7CE2405CE76
:10D44900E5D312D4E7E5D222F5D2C2D58035F5D29B
:10D45900D2D5802F30E70DF404C0E0742D12D4CF5B
:10D469000E0ED0E0F5D275F0648485F0D3C2D57084
:10D4790009D2D5742012D4CF800312D4BCCE24048F
:10D48900CEE5D375F00A8485F0D3700A30D50774D8
:10D499002012D4CF800312D4BCCE2404CEE5D312FB
:05D4A900D4BCE5D22215
:1076E700909F6E1276F002DD3F7E00800E7405FEDD
:1076F700F51EE4FFF51DF51F203C3375A700E49345
:10770700700122A3B40204051D8003B4010A051FFA
:10771700EF2409FFAE1E80E612D5017D06B44002B4
:107727007D03B421027D02EE2DFE80D27E0075A777
:1077370000E493700122A3B40204051D8003B40181
:107747000F051FEF2407FFAE1E80E612D4CB80087B
:10775700B45B0050F612D4CF0EB4210280D30EB41E
:10776700400280CDB42C0280C80E0EB45F0280C1E7
:10777700B45B0040BC0E0E80B8E60812D501EE24BB
:1077870006FED513F422909CAC307409909CB0305F
:107797007303909CB502770275F019D5E0FDD5F01B
:1077A700FA12484F12DC59744F12DC6A744B12DC20
:1077B70048C322C2501277FE12484FD2AC12DBB236
:1077C700304C1212DBB2304C0C12DBB2304C06D20A
:1077D70050C2ACD322B440E512DBB7B4400312DB8E
:1077E700B7B44FED12DBB7B44BE712DBB712DBB719
:1077F70012DBB7C2ACC32230530975F008D5E0FDE0
:10780700D5F0FA227F0575F019D5E0FDD5F0FA120B
:10781700484F12DC59745712DC6A745012DC277413
:097827008112DC27E56312DC2765
:10783000E56212DC2778D0E612DC2708B8D7F8E634
:10784000F8795F30E702792FE912DC2712DC271282
:10785000DC2712DC27745812DC27744312DC27E47F
:1078600012DC27E8C2E775F00A84C425F012DC2791
:107870007864E612DC2708B869F8E612DC4812776B
:10788000BA400122DF02800A20508B75F000808010
:10789000D250C2ACD3221277FEC25012484FD2ACA3
:1078A0002002EF12DBB2204CE7B440F412DBB7B495
:1078B000400312DBB7B457DAF53812DBB7B450D255
:1078C00012DBB712DBB7F56312DBB7F56278D012C3
:1078D000DBB7F924A0500353015FE924E0400279AB
:1078E0005FA60108B8D8E8780612DBB7D8FB12DB30
:1078F000B7FC53040FC4540F75F00AA42CFC249C4D
:1079000050027C0078D78601E4B92F02D2E72CF62A
:10791000786412DBB7F608B86AF812DBB7E53860AE
:107920000302789212DBB712DBB7C2ACC32290A37A
:107930006D8003909FB37F2012773312DD3F02DE0C
:107940002B753400C26B1279FD12DE2B127DADE572
:1079500016600312795902025912800F121E461244
:10796000DD3F10002010010280F8127E1850131223
:107970001E5112792E10000D10010280F8121DF315
:0579800080D7127B9D81
:1079850022C26BD22775480A122B77753400127EF6
:10799500E5C26A1233CF106A0512024A80ED12025F
:1079A5004A127D3F127E97127EF178D0E6642660FA
:1079B5004412800F121E4612DD3F100038100102DE
:1079C50080F8127E18501BE965156018121E5112B9
:1079D500792E12DE2310001D10010280F8121DF30E
:1079E50080BCD26B127EC3751607855917122BF012
:1079F5007535008096020259127DAD127A1F127EEE
:107A0500F17F19127A3990A39B7E121277357E2366
:107A1500E51602D46D90A4E780EF7862E4127A301F
:107A250078D0745F127A3018E4F6227F08F608DF02
:107A3500FC227F7B7E007810742012D4CFCE2404E4
:107A4500FED8F5227F197E081277357E28909F95FE
:107A5500305303909F9A027735C26B127A1F127AC0
:107A650069020259C251127EF190A393127A49120A
:107A75001E19127DAD7F20127A0812DD3FE51670C2
:107A85000512DE20803675A6FF3051031277A81245
:107A9500484FD2AC200025306DFA127899400C126F
:107AA5007E184011127B9DD25180BB105003127974
:107AB50033C25180D1D25112792E80CAC2AC22D2A2
:107AC5002775480A122B77753400C26B127EE5C202
:107AD5006A1233CF106A0512024A80EB12024A126B
:0D7AE5007D3F127E97127EF1127AF550DA85
:107AF200020259909FAE127A49121E2B12DD3FC329
:107B020010001310010510020E80F412780B4001D0
:107B12002212793380DDD3C2AC22D227C26B7548E0
:107B22000A122B77753400127EE5C26A1233CF1027
:107B32006A0512024A80EDD26B127D3F127E9712C5
:107B42007D6775B901E5BCB2E7F5BC124EE6751664
:107B520007855917122BF080CB127DADE516601FF9
:107B620078D0E53D127B8EE53E127B8EE53F127B9F
:107B72008E765A08765F12C832127EC3027D7E7FED
:107B82003E7E11909F8512770202DD3F75F00A84D6
:107B92004430F608E5F04430F60822D26B127EC378
:107BA200127D7EE51775F01084240AF54824E8500A
:107BB2000375480A122B838558592275320012BE6A
:107BC2008275A704900700751500127D6775B901CB
:107BD200E5BC20E705E515F0801004600D648260C5
:107BE2000975BCFF75B90575B9020515E51524209F
:107BF20050D8E58224FE4003027C96A882187F00BA
:107C020075A7007583078882E0FE75F004A4127DD3
:107C120012A9BCAABDABBEACBF1582E0FD75F004D3
:107C2200A4127D12C3E995BC404C7052EA95BD4046
:0D7C320045704BEB95BE403E7044EC95BF95
:107C3F004037703DEE75F004A404127D12A9BCAA62
:107C4F00BDABBEACBFED75F004A404127D12C3E949
:107C5F0095BC4015701BEA95BD400E7014EB95BE98
:107C6F004007700DEC95BF5008EEF00582EDF01552
:107C7F0082E5826009C3EF95825003027C0A0FC32D
:107C8F00E89F4003027C0275A70490070075C703A5
:107C9F0075C6A8E0F5BCE0F5BDE0F5BEE0F5BF7533
:107CAF00B90575B90205C6E58224204006E5C6244C
:107CBF002050E00875C70375C68075B901E5BC1281
:107CCF007CFCF5BCE5BD127CFCF5BDE5BE127CFC71
:107CDF00F5BEE5BF127CFCF5BF75B90205C6E5C65A
:107CEF00245850D6E5320470FB75A70022B4FF016B
:107CFF0022F975A704900700E582686005E06970B6
:107D0F00F7E922F5C685F0C775B901E5BC645F7068
:107D1F000375BC27E5BD645F700375BD27E5BE64C1
:107D2F005F700375BE27E5BF645F700375BF2722C1
:107D3F0075C703E54875F004A42480F5C6E55975A9
:107D4F00F00484A8F00825C6F5C675B901A9BCAA28
:077D5F00BDABBEACBF8615F1
:107D660022E515242050037515DFE51575F004A4EA
:107D760054FCF5C685F0C722E51724204028E517F0
:107D860075F00484A8F00824A8F5C675C70375B96C
:107D960001A9BCAABDABBEACBFA61589BC8ABD8B6A
:107DA600BE8CBF124EE622E4F516F51579FF127D5C
:107DB6006775B901E5BCB4FF040516A9150515E5F7
:107DC60015242050E9891579FF75C70375C6A8756E
:107DD600B90109E5BC04601B09E5BD04601509E5A8
:107DE600BE04600F09E5BF04600905C6E5C6242088
:107DF60050DD09891722751600751501127D677504
:107E0600B901E5BC20E70205160515E51524205045
:107E1600EB227900E975F004A454FCF5C685F0C799
:107E260075B901E5BC20E73078D066702B08E5BD52
:107E360066702508E5BE66701F08E5BF6670190501
:107E4600C675B90108E5BC66700E08E5BD66700822
:107E560008E5BE667002D32209E9242050B6C32283
:107E6600127E86127E6EA8017F08E0F608DFFB22EE
:0B7E7600127E86127E7EA8017F08E6C7
:107E8100F008DFFB2278D0796275A704758307EBD0
:107E9100C454F0F58222127D6778D0127EB1E5BC20
:107EA100F9C23C20E702D23C127EB17862127EB167
:107EB10075B901A6BC08A6BD08A6BE08A6BF0805DF
:107EC100C622127D6778D0127ED3127ED3786212D9
:107ED1007ED386BC0886BD0886BE0886BF08124EC2
:107EE100E605C622125A3612DF1512866E02DD3FF2
:107EF10012DF157F007E0990A37F1277027F0A7E31
:107F010012E5150412D3A57F1412CA1C121DF37FAA
:107F1100277E0875130778D0127780E6793E30E71F
:107F210002792F7E34E912D5017F3D7E0190A503B0
:107F310012773520311B3030031291A9C23B1281D7
:107F4100A1127F57D23B1281A1127F691281E88071
:107F51007C12C08880E6C23B7F44745320170274B0
:107F61004E7E0012D5018017D23B7F4F74572017E8
:107F71000274457E0012D5017E06E51E12D4EE7E06
:107F81000CE51D12D4EE7E12E51C12D4EE7E1774A0
:107F91008112D5017E1CE51B12D4EE7E22E51A1258
:107FA100D4EE7E28742E302602742712D5017E2D40
:107FB100E51912D4EE7E33E51812D4EE7E3930265F
:0F7FC10007742C12D4FD7E3BE53702D4EE742DED
:107FD000201702742B7F707E1512D501127FEC7E64
:107FE0003A12D34E7E0190A52E0277027E1BE51C2D
:107FF00012D4EE7E21E51B12D4EE7E27E51A12D4B0
:10800000EE7E2DE51912D4EE7E33E51802D4EE1281
:10801000808D1280B812838F127EF11283E72017B1
:108020001E10021B1248F012C832128075121DFE7B
:108030007F347E2F12778D127F2A12DD3F80E2126D
:108040001DF3203026203128C23B1281A11280CDA1
:1080500078661282A1D23B1281A11280E278691265
:1080600082A11281E812815C02834412927280F232
:1080700012C09D80EDE57D75F01084AAF075F00AC0
:10808000A42A547FFA78D7E654802AF6227F277EE6
:108090000879D08700C001D224B9D002C22412844A
:1080A0006ED001A70010230909EE2406FEB9D7E31C
:1080B0002219EE24FAFE80DB7E3479D7E7A2E7921C
:1080C0001712841B79D7E7A21792E7F722C224C2BE
:1080D0003B751E007F447E0012842B801E1023ED12
:1080E000802AD23BC2247F4F7E00128433D2247E6A
:1080F00006E51E128460F51E1023E7D2247E0CE5EF
:108100001D128460F51D303BD41023E1D2247E1271
:10811000E51C128460F51C1023E17E1CE51B128413
:0381200060F51BEC
:108123001023E67E22E51A128460F51A1023E87EF6
:108133002DE519128460F5191023E87E33E5181232
:108143008460F5181023E87E393026027E3BE5373C
:10815300128460F5371023E3227F707E1512842387
:10816300C2247E1BE51C128460F51CD2247E21E50B
:108173001B128460F51B1023E77E27E51A12846027
:10818300F51A1023E67E2DE519128460F5191023E4
:10819300E87E33E518128460F5181023E82278D7B7
:1081A300E6C2E775F00A847866F537303B057869EF
:1081B30085F03712821130262BE53775F003A404BE
:1081C3000475F00584FBE51975F00AA4251875F00C
:1081D30006A42BFBE435F0FC125585F537125585C3
:1081E300F5188B1922E563FC339217AB6250031227
:1081F30055F6305C0A7AD21253717840125513AE99
:1082030004AF037C277D1012547C8F1C8037E6FD5E
:1082130033921718860418860350031255FE7A0901
:10822300792778C01255108B1EADD3ACD2AB06792B
:10823300EA786012550E8B1DAF06AED27C177D70A7
:1082430012547C8F1CAF05AE047C037DE812547C72
:0F8253008F1BAF05AE047C007D6412547C8F1A24
:10826200ED75F00A84F51985F01822EC3392175057
:10827200031255F6751D30301786751D2D808178D5
:10828200427B607CEA800678407B207C4E12C1688B
:108292007927781012550E8B1CAF06AED280AB3008
:1082A200262AE51975F00AA4251875F00AA42537BF
:1082B200FBE435F0FC7A051253638C068B077C00D5
:1082C2007D0312546F8E048F031281DBE51E75F05D
:1082D2000AA4251D75F00AA4251C75F006A4251B09
:1082E200FBE435F0FC7A0A125363EB251AFBE43CFB
:1082F200FC7A0A125371EB2519FBE43CFCE43DFDC8
:108302007A0A125383EB2518FBE43CFCE43DFD3072
:1083120017031255FEA60518A60418A60378D7E679
:10832200A2E7923DC2E775F00A84FCABF0303B0E47
:10833200AB37EC75F00AA42BA23D92E7F622AC37DC
:1083420080F012835F305C0A7A4012537178D21245
:1083520055133017031255F68C638B622212836F0A
:108362007A0A125363EB2518FBE43CFC22E51C75E8
:08837200F00AA4251B75F00AB6
:10837A00A4251AFBE435F0FC7A0A125363EB25199B
:10838A00FBE43CFC221283C112DE27C202C2231282
:10839A0083C110000810010510021B80F51031ED91
:1083AA0010300D102604D22680E3D230C23180DD8F
:1083BA00D231C23080D7227F3590A4EC1277339025
:1083CA00A50A20300F90A52620310990A4FB20266B
:1083DA000390A4F31F7E1712770202DD3F7F357EDA
:1083EA0001909F611277357F347E3A128510744E60
:1083FA0012D50112DD3F12DE27C2027F347E3AD245
:10840A001775115975124E802675112E751227800F
:10841A001E75113E75122F801675112B75122D803F
:10842A000E75114E75125380067511457512571245
:10843A008510E511301702E51212D50112DD3F1041
:10844A00000810010510020B80F5D23C1017E3D288
:10845A001780DF02850B4430F812846AE8540F2231
:10846A00C2218002D221A22492229223128510E8EC
:10847A0030E709D23C7430302102745FF812D5011A
:10848A0012DD3F10003410010510025D80F5D23C68
:10849A00102266102367B43909745F2021DF743013
:1084AA0080DBB45F04742D80D4B42D04744180CD74
:1084BA00B45A04743080C60480C3D23C30240610F7
:0F84CA002237102338B44104742D80B1B42D042F
:1084D900745F80AAB45F04743980A3B43009745AF4
:1084E90020219B74398097148094B48908D223E899
:1084F90012D501800DF8C223800874898001E80231
:1085090084879085258003908521C007EF2408FF83
:1085190012D52DD00702DD3F0205F8F8020500004B
:10DCDF0075A70090DD1175F02D84C2D5C2D16017E4
:10DCEF00D2D1146007D2D514600DC2D1E5F093FCE8
:10DCFF00742D95F093FB22E5F093FB742D95F09323
:10DD0F00FC220009121B242C353E474F58606870C7
:10DD1F007880888F969DA4ABB2B8BEC4CACFD4D931
:10DD2F00DEE2E6EAEDF0F3F6F8FAFCFDFEFFFFFFA8
:10DDD900D23D8002C23DED8BF0A430E70205F0C3CD
:10DDE900E895F020D50425F025F0FEED8CF0A4305F
:10DDF900E70205F0C3E995F030D10425F025F0FFDD
:10DE0900203D0B2487500122EF24CC40012202DE61
:01DE19005AAE
:10D77D00203A7A7E1C7F5312DE5A7F5912DE5A1ED2
:10D78D007F5712DE5A7F5512DE5A7E2312DE5A7FE4
:10D79D005712DE5A1E7F5912DE5A7F5312DE5A1F60
:10D7AD007E2012DE5A7F5A12DE5A7E1E12DE5A7FFC
:10D7BD005212DE5A120E67E5BD20E0143006117FBD
:10D7CD00357E1C90D839E571700390D84302D52D64
:10D7DD00E5716018E57012DCDF781F79567D09124E
:10D7ED00DDDD303A0312D80C0DBD16F3227E1C7F01
:10D7FD005390D82212D52D200CD612CA7880C0C0D5
:10D80D00060E30D5021E1E12DE5AD0061F30D10272
:10D81D000F0F02DE5A070700386C446C38000505FF
:10D82D002070D8702005057088A8887008071038FA
:10D83D007CFE383838000807102844C628283800E0
:10C8570090A5387F717E23127735120E67E5BC7E6F
:10C867003112D4BC30121AC23C120E67E5BCFB75FC
:10C87700F00AA4F904FAC23D12BE6E12CAF5303DA1
:10C887000122DAF712C9FC7C00EBF4042E4019AD43
:10C897000312546FEFA2D1203C077E237F6502D19C
:10C8A7001BAE16AF1702C99DAD0112546FEF12D21E
:10C8B70009203C077E237F6502D13FAE16AF1702E2
:10C8C700C9C17F567E0512CA287F3D12CA3B7F6FBA
:10C8D70012CA3B12CA787E0A7F4112CAAB7E227FF8
:10C8E7005912CAAB2012012212BE6E857A1D855ECF
:10C8F7001C857B1B855F1A7AC0C23D12CAF1203D99
:10C907005212C9FC7C007D1412546F74562F20D12B
:10C91700029F9FFF24CB40028037EF24885002807C
:10C9270030EA1475F00384FE12DE5AC3E51B957BCB
:10C93700FEE51A955F92D55004EEF404FEEEC3139C
:10C94700FE24E0400C741F2E30D5029E9EFE12DEA0
:10C957005ADAA8227F5212C96D7F5A12C96D75170C
:10C9670053751600802B7E0012DE8A0EBE12F92246
:10C977007F157E28742012D5017F1C7E2812DE8A3F
:04C987000EBE40F9A7
:10C98B00223012E712C97775171575162DD23C0296
:10C99B00C870C23D6002D23D92D175F080305C040C
:10C9AB00F5F08001A4A2E792D5E5F075F03284F89A
:10C9BB00E5F075F00584C0E0E5F0A2D533C0E0E802
:10C9CB00601E12D4EEEE2406FED0E0F8D0E012D4B6
:10C9DB00EEEE2406FE742C12D5010E0EE802D4EEF8
:10C9EB007420303D07742B20D102742D12D5018099
:10C9FB00D4C3ED957AFFEC955EFE92D150031255A0
:10CA0B00E6227F1512CA147F327E3E12DE5ADEFBFF
:10CA1B00227E0912DE5A0EBE36F9227E0112DE5A32
:10CA2B000E0EBE3FF8227E3312DE5A0EBE40F922A6
:10CA3B007E047D1112DE5A0E0E0EDDF81F1F7E35A1
:10CA4B0090A541305C057E3190A545027735740584
:10CA5B00305C097E32740112D4BC74067E3612D45B
:10CA6B00BC7E3A740012D4BC7E3D02D4BC7F417EA6
:10CA7B001F7D0F12DE5A0F0F0FDDF8227F687D032B
:10CA8B0080047F677D0512DE5A0FDDFA227F667DFB
:10CA9B000780F37E1F7F5012DE5A1F1FBF3EF82206
:07CAAB007D0A12DE5A0E0E97
:10CAB2000F0FDDF722203D07123C767003D23D2294
:10CAC200056D12BC34E4F5F7C2B2C2B2ABF7F5F7AA
:10CAD200C2B2C2B2E5F7FA30E411EB251DF51DE44E
:10CAE200351CF51C0519EA30E3010ED2B280157827
:10CAF2000380027801203D07123C767003D23D226A
:10CB0200D8F3056DE56D2409F56D12BC34E4F5F733
:10CB1200C2B2C2B2ADF7F5F7C2B2C2B285F71BF527
:10CB2200F7C2B2C2B2E5F7FCD2B2543F30E50244DA
:0FCB3200C0CC54C02323F51AE56D24F6F56D220F
:10D6A4007E017F0990D72212D52D2051097E037F58
:10D6B40000743F02D501E4FEFFC3E54512CF73FDBC
:10D6C400940AED403D9464ED4002746312D39F7E4E
:10D6D400017F09E552240575F02D84AAF075F00543
:10D6E400A4CA75F00B842A90D70D9312DCDFBCB862
:10D6F400027BB87D04EE2DF8EF2DF90D12DDD9DD96
:10D70400FB227E0312D4EE80C6000C1622222D3991
:10D71400444F4F5A66707C7C87939EA9A9000909DF
:10D724000800410000000000888000000000410063
:10D734000800120E7BE5BCB4F8339004C3E0602CFF
:10D74400FA24F340277F137E0012DE5A0F0F12DEF5
:10D754005A0E12DE8A1F1F12DE8A0EDAEC7F147E46
:10D764000012DE5A0E12DE8A0EBE12F5229005CC8D
:09D77400E0C3941240F60480C7E2
:10CF7300305D0A75F08AA42480E5F0340022207421
:10CF8300157F017E1190CFFB12D52D7F0A7E0AE516
:10CF93002E540702D3B67F087E1190D00B12D52DE5
:10CFA30020730C7F0A7E1712DE8A0E0E12DE8A7F32
:10CFB300007E0BE57112CF7312D3A57F0C7E11E5B2
:10CFC30071602F0EE57064B4602864B475F0328428
:10CFD300C0F012D4E7CE2405CED0E075F00584C0AE
:10CFE300F012D4E7CE2405CED0E023302D01040285
:10CFF300D4E790886A027702070FFFFFC473BDAFBF
:10D00300A463B5FBCDE7FFFF030F0100FFFE038021
:10D01300306701227F357E00748812D501E55160A7
:10D023001712CF7375F06484F87E06E5F012D4040A
:10D03300E860E07E0002D4EE7E003074D6307316D2
:10D0430079BCE7FC09E7FB12530B781D201704E6B4
:10D0530070011802D2CF909CB0027702202C0122DB
:10D0630090D06902D52D050EFFF0E01CF004F81CEA
:10D07300FFF0301201227F637E00909CC712D52DF2
:10D083007F1512CA147F1F12CA147F2912CA147F74
:10D09300177E06E53F30E00B90A555305C0390A565
:10D0A3006980132074077E01909CE7800990A54A4C
:10D0B300305D0390A55F127702307306E54E600280
:10D0C300154E205718E54EB40113120E8AC3E55CC2
:0DD0D3009560F5BCE55D9561F5BD124EE67A
:10D0E0007F217E01E53F30E021305705909E108082
:10D0F00016E54E7005909E1C800D909CF3127702F1
:0BD100007E30E54E02D40A12770222B6
:10D2710012530B7F207E05751900781DC2D5E6304B
:10D28100D51712D4E7EE2405FE18B818F17E1F74E5
:10D2910063305C02748202D5017005B8191880E20E
:10D2A100D2D5CE24FACE7484301702742D12D50152
:10D2B100EE2406FE80C8742012D4FD80C8781C803C
:10D2C1000D7F007E23AC5EAB7A12530B781DC2D565
:10D2D100E630D50C12D4EEEE2406FE18B818F12271
:10D2E1007005B8191680EDD2D53017E4CE24FACEE8
:10D2F100742D12D501EE2406FE80D5742012D501BD
:10D3010080D512530B781DC2D5E630D51612D4BC88
:10D31100EE2404FE18B818F10E745E305C02742716
:10D3210002D4CB7005B8191680E3D2D53017DACE06
:10D3310024FCCE742D12D4CFEE2404FE80CB7420B5
:10D3410012D4CF80CBC23D12D3590F0F0E0E74638E
:10D35100305C02748202D50112530B781DC2D5E6EE
:10D3610030D50C12D51CEE2408FE18B818F1227025
:10D3710005B8191680EDD2D5301716740BCE24F8E6
:10D38100CE12D51CEE2408FE80D5740C12D51C805B
:08D39100D5303DCB740A80E5A4
:10D84D007F797E24E55F30E70122AC5F1CAB7B1254
:10D85D005339E51B700E742012D501EE2405FE120E
:10D86D00D89B800C12D89BE51B12D4E7EE2405FE45
:10D87D00E51A12D4E7EE2405FE742C12D5010E0E16
:10D88D00E51912D4E7EE2405FE745E02D501742D60
:10D89D00201702742B12D501EE2406FE22E55F300F
:10D8AD00E70122AC5F1CAB7B125339E51B700E7484
:10D8BD002012D4CFEE2404FE12D8F4800C12D8F42A
:10D8CD00E51B12D4BCEE2404FEE51A12D4BCEE24E2
:10D8DD0004FE742C12D4CF0E0EE51912D4BCEE2416
:10D8ED0004FE742A02D4CF742D201702742B12D487
:06D8FD00CFEE2404FE2220
:10D10B007F097E2530040512D2058028A275E579AA
:10D11B00C23D6002D23D92D175F080305C04F5F0D7
:10D12B008001A4A2E792D5E5F075F03284F8E5F022
:10D13B0075F00584C0E0E5F0A2D533C0E0E8602AC5
:10D14B0012D51CEE2408FED0E0F8D0E012D51CEE70
:10D15B002408FE0F0FE52B5403701F746012D501CA
:10D16B001F1FEE2404FEE802D51C740C303D067420
:10D17B000A20D1010412D51C80C9205904742E80B9
:10D18B00DC205804747F80D5748080D13004051264
:10D19B00D2058028A275E579C23D6002D23D92D1BD
:10D1AB0075F080305C04F5F08001A4A2E792D5E520
:10D1BB00F075F03284F8E5F075F00584C0E0E5F029
:10D1CB00A2D533C0E07F3E7E1CE8602012D57DD017
:10D1DB00E0F8D0E07F3E7E2812D57D7F447E32740E
:10D1EB002E12D5017F3E7E37E802D57D303DE074AF
:10D1FB000A20D1010412D57D80D59005CAE075F0C7
:10D20B000A84F8E4C5F0C2D522301105E54AB40210
:10D21B0050C39006E9E0957AFB9006E8E0955EFC3A
:06D22B0050031255F6EC61
:10D23100C31360047B63800FEB13FB249C40F52434
:10D241004F4004C20480079005CAEBF0D204900657
:10D25100E6E09006E8F09006E7E09006E9F0E55E8A
:10D261009006E6F0E57A9006E7F02212D24F80DED2
:10CB4100E54424F64001227800E552206607C395AA
:10CB510070500224B40475F00384F9E928FE24C45A
:10CB61005001FE12CB8312CB8F1E12DE5AC3E998FD
:10CB7100FE5003243CFE12CB831E12DE5A08B81F5E
:10CB8100DA22EE2420FE24C250032402FE22E824ED
:10CB9100F1E8C2D55006D2D5E8F4241F23FF90CC8A
:10CBA1001193CF0493FAE545F5F0A4ACF0FB1253D1
:10CBB1009AE544F5F0A49BFBE5F09CFCEB2420FBFB
:10CBC100EC3400FC12CBF2FAE5458FF0A430E70219
:10CBD10005F0E5F020D502F4042A75F005201903CB
:10CBE10075F00384FF24DF50027F20C374329FFF5E
:10CBF10022EC24F0500BEB2460EC340090CC6193D8
:10CC010022EB33FBEC33FCEB33EC3390CC3193224E
:10CC1100FF00FF03FA0BF318EA2ADE40CF58BE7378
:10CC2100AB8D96A880C068D64FE835F51BFD00FF97
:10CC310000080B0E101214151718191B1C1D1E1FAE
:10CC410020212223242526262728292A2A2B2C2D78
:10CC51002D2E2F2F303131323333343435363637B0
:10CC6100373839393A3A3B3B3C3C3D3D3E3E3F3F0C
:10CC71004042444648494B4D4E50525355565859DF
:10CC81005B5C5D5F60616364656668696A6B6D6E5C
:10CC91006F7071727374767778797A7B7C7D7E7F21
:10CCA100808182838485868788898A8B8B8C8D8E0F
:10CCB1008F9091929394949596979899999A9B9C19
:10CCC1009D9E9E9FA0A1A2A2A3A4A5A6A6A7A8A936
:10CCD100A9AAABACACADAEAFAFB0B1B1B2B3B4B465
:10CCE100B5B6B6B7B8B9B9BABBBBBCBDBDBEBFBF9F
:10CCF100C0C1C1C2C3C3C4C5C5C6C7C7C8C8C9CAE4
:10CD0100CACBCCCCCDCECECFCFD0D1D1D2D2D3D431
:10CD1100D4D5D5D6D7D7D8D8D9DADADBDBDCDDDD87
:10CD2100DEDEDFDFE0E1E1E2E2E3E3E4E5E5E6E6E2
:10CD3100E7E7E8E8E9EAEAEBEBECECEDEDEEEEEF44
:10CD4100EFF0F1F1F2F2F3F3F4F4F5F5F6F6F7F7AB
:10CD5100F8F8F9F9FAFAFBFBFCFCFDFDFEFEFFFF1A
:10CD6100E54524FD400122E552206607C395705038
:10CD71000224B40475F00384241FFE24C25003244A
:01CD810002AF
:10CD8200FE12CDBCEEFD241EFE24C250032402FE80
:10CD920012CDBCE544240275F00520190375F00399
:10CDA20084F4042432FF24EE500F12CDB1AE051EDE
:10CDB2001E7C0512DE5A0EDCFA227F1512DE5A0F95
:05CDC2000FBF2DF82257
:10D5BC007E00206615E5700475F0B484E5F075F016
:10D5CC000384FE6004C3743C9EFE745312D5E7744E
:10D5DC005712D5E7744E12D5E774457F2F12D4CF6E
:10D5EC00BE00077E3C12D4CF7E00EE240875F03CC2
:10D5FC0084AEF00F0F0F12DE5A0E12DE5A0F12DE2F
:10D60C005A1E12DE5AEE240775F03C84AEF022301E
:10D61C00745C301259E54AB4040122B4060122E5C7
:10D62C007112CBDB8F057C037E1E30662AE57004FD
:10D63C0075F00384241EFE24C6501C24FB500424C5
:10D64C00038013C00612D663D0E024C67C016006AA
:10D65C000C1460020C14FE12D66F0EEE24C14002A4
:10D66C00DCF5228D0712DE5A0FEF24CE50F722E59F
:10D67C0053206607C39570500224B40475F00384DC
:10D68C00241FFE24C250032402FE12D69A0E7F23BE
:08D69C0012DE5A0FBF2DF92226
:10DD9000AF177E00E53C12D3997E0C742E12D5018C
:10DDA0007E12E53B12D3997E1E742E12D5017E247D
:10DDB000E53A02D3997E0E78ADE612D4047E18744B
:10DDC0002C12D5017E1B18E612D4047E25742C1269
:09DDD000D5017E2818E602D404F6
:10CDC7007F797E00E54012D4047E0A743B12D4FDBD
:10CDD7007E0CE54102D4047F797E16743B12D4FDA4
:10CDE7007E18E53F12D4047F797E0078AEE612D430
:10CDF700047E0A743B12D4FD7E0CE53E02D4043057
:10CE07005EE52043E27F6D7E0078AEE612D4047EB5
:10CE17000A743B12D4FD7E0CE53E12D4047F757E66
:10CE27000075F00A84E5F012D51C0F0F7E08743ADE
:10CE370012D4FD1F1F7E0DE53F75F00A84C0F01266
:10CE4700D51CEE2408FED0E002D51C851C1E851BD0
:10CE57001FAB1BAC1C305D0A7A1B12537178321260
:10CE67005513C3EB33FBEC33FC923D125342303D79
:10CE7700087409F51DF51CF51B7F75E51D60157E0A
:10CE87002412D51C7E2CE51C12D51C7E34E51B1202
:10CE9700D51C803D7E22E51C601912D51C7E2AE533
:10CEA7001B12D51C7F787E31742E12D4FD7F75E559
:10CEB7001A8019E51B12D51C7F787E29742E12D48F
:10CEC700FD7F757E2DE51A12D51CE5197E3512D525
:10CED7001C7F777E3C125CCC851E1C851F1B227F26
:10CEE700397E1F12DE5A0FBF40F9781F79567A0034
:10CEF7007D1A12DCDF12DDDDEA2406FABAAEF3781A
:01CF07001B0E
:10CF0800C3E5119570500224B4FA604214603E14CF
:10CF1800603A2450603A146036EA24A540278A1EF5
:10CF2800751D007D1912CF380D30740312CF380DDE
:10CF3800781F7956AA1DEA12DCDF12DDDD0AD3EA72
:10CF4800951E40F2228A1D751EB380D7080808086E
:10CF58007F367E1C90D839E571700390D84312D57E
:0BCF68002D7F3CAE0090852102D52DEE
:10DA6000787512DAB07453201702744E207406E5EC
:10DA70002E54074430AF1712DADA7E3BE57DC454EA
:10DA80000F12D4EE2074077E07742012D501787827
:10DA900012DAB0E5172409FF7457201702744520E5
:10DAA0007402742012DADA7E3BE57D540F02D4EE64
:10DAB000E6FD3392171886041886033017031255B3
:10DAC000FE7917787012550E8B13AF06AED27C001C
:10DAD0007D6412547C8F148D15227E0012D5017E38
:10DAE00007E51312D3B67E19748112D5017E20E5A5
:10DAF0001412D3997E2B742E2073030E742C12D51E
:08DB0000017E2FE51502D39907
:10DC6F00E54A602E7A2420E00E7A26141460087A92
:10DC7F0028141460027A297F667E01EA12D50120EA
:10DC8F005505205406800B745B8002745C7E001275
:10DC9F00D50120110778A9B60007802130261EC2B2
:10DCAF0026909D867F681276F07F66A85AE54AB463
:10DCBF00060108E875F06484E5F012CE4020080FE5
:10DCCF00E537640260097F367E2E744112D4CF226D
:10D9030020144F740512DF01EF33EE33F9EF0303F5
:10D91300541FF5F090D956E993A4C5F013C5F0133D
:10D92300C5F013C5F013C5F0135403FCE5F013FB66
:10D93300E9242093C9244093C39BC4540FFBE99C5F
:10D94300C4FC540FF9EC54F02B2446F57BE934F670
:10D95300F55F22FFFFFFFFFFE6C5AD9C8F857D7757
:10D96300726E6C6A696A6A6C6F747A828D9DB4D9BF
:10D97300FFFFFFFAE9DCD3CEC9C6C3C0BEBBB9B74C
:10D98300B5B4B2B0AFADABAAA8A6A4A2A09E9C9911
:10D9930096918C00381CE735D137246F00C5B3C18D
:10D9A300E61F66B60E68C21867AADBF4EDB94675C2
:03D9B30010A200BF
:10DEE100D2A27408D2A1D2A300C2A3C2A1D2A3001C
:10DEF100C2A3D5E0EF7405D2A300C2A3D5E0F822F6
:10DEBA00C2A3D2A2D2A1D2A300C2A375F008339200
:10DECA00A1D2A300C2A3D5F0F5C2A175F003D2A3D3
:07DEDA0000C2A3D5F0F822FD
:10C4710012DEBAD2A300C2A3C2A175F008E4D2A30E
:10C4810000C2A3A2A233D5F0F5FE75F008E4D2A351
:10C4910000C2A3A2A233D5F0F5FFD2A300C2A3220A
:10C4A100E478806608B88BFB70012274D512C471E0
:10C4B1007881C3EE13FEEF13F692D118EE2460F6E5
:10C4C10074D612C4717888EF33CE33CE33CE33CEE7
:10C4D10033A2D192E25407FCEEFB7A08125363ECCB
:10C4E100244FF608EBF674D912C471EF543F7882E9
:10C4F100F67886EF33CE33CE33CE33CE335403F6D4
:10C5010008EEF618161608E6C4FF54F0F618E6C44D
:10C51100CF540F2FF674DA12C471EF232354FC7831
:10C5210083F67884EEF608EF54C0F67880E4660866
:10C53100B88AFBF62212C4797889C3EF96FF18EE08
:08C5410096FEA2E792165010CD
:10C549001255E6740FF8F91253B0EF2CFFEE3DFEC9
:10C55900788BEEF608EFF622E6182016072CF7E698
:10C569003D19F722C39CF7E69D80F66A405E805626
:10C57900E050F04B0044803DC0384031D02BA0251D
:10C58900601F2018D014000F000AA00144015801AF
:10C59900680178018801A001B401D001EC02100200
:10C5A90038026802A002DA030C034D78BE802085A8
:10C5B9008E8A9D8F4D95BA9A97A0BEA631AC53B27B
:10C5C9002AB801BD6AC1EDC4D1C78812C479788D72
:10C5D900EEF608EFF67887798C1253B07883799064
:10C5E90012C5617885798C1253B07881799212C518
:10C5F90061788DE624E4FE08E63392D13392D5546E
:10C60900FCFFEEA2D133A2D533FE780F79921253F3
:10C61900B078947990C3EC97F61819ED97F6799458
:10C6290090C5747F1F7D11EF93C3971F19EF9397DF
:10C639001F091DED600240EF0F90C594798DEF93AE
:10C64900F7090FEF93F7788E79941253B090C5B428
:10C65900EF93C39BFB1FEF939C2420FC7897E62B59
:10C66900F618E63CF618E436F6740612DF01D237FE
:09C67900EE24F7400624025002F1
:10C68200C237EEFCEFFD740712DF01C3ED9FFFEC32
:10C692009EFE78B7E6FD337C0050011CEF2DFFEEC5
:10C6A2003CFE789CEF26F618EE36F6222014122075
:10C6B200370F789DE6B4050912C76612C79B12C7E9
:10C6C200E42220145E7897799A12C81512556EC327
:10C6D200EE9420FE924550031255E67C007D051231
:10C6E200547C3045031255E6E531B40C3612DA4675
:10C6F200120E80E5BC2FF560E5BD3EF56120E71125
:10C7020024F8500DFAC3E5609AF560E5619400F5EE
:10C7120061120E8AE5BC2560F57AE5BD3561F55EEC
:10C7220012DA537897799AC3E697FB1819E697FCC1
:10C732007A0212536330370B7A02125363ECFEEB28
:10C74200FF800312C76612C79B20140312C7E47846
:10C75200957998E6F776000809E6F776000809E683
:10C76200F7760022799CE77700FB19E77700FC78DF
:0CC772009DE6B40506EB33FBEC33FCEC59
:10C77E00A2E792D550031255F67A32125371ECFBA2
:10C78E00EDFC30D5031255F6ECFEEBFF22EE24083D
:10C79E00FE74042037167406307511789DE6B405C4
:10C7AE0004740C8007F42406C323540FFD7C00127E
:10C7BE00534F789FE6FC08E6FBC374109DFA1253A4
:10C7CE0071EFF8EEF912556EE878A02FF6FF18EE1D
:10C7DE0039F62480FE22927540031255E678BBE6A8
:10C7EE00F5F02438400375F0E1EF33EE3378A8F618
:10C7FE00A485F07930E7020579C276307508E579BF
:10C80E0024F15002D27622E627FB1819E637FC18DF
:10C81E0019E637FD2212BE157F087871793A12C8D3
:10C82E003E024ABB855E63857A62787379647F06C1
:10C83E00E6F70809DFFA227864797380F178737964
:09C84E00AF80EB78AF797380E54F
:1052E900E4FEFFFC7D0A791DE7540F2FFFE43EFE23
:1052F900B9190280061912534F80ED301703125560
:10530900E622305C2BEC33921750031255F6EC244D
:10531900D950047C277B007AD2125371EB33CC33FA
:10532900CD33CC33ED33FBEC33FC3017031255F698
:10533900EC33921750031255F67919125585F7096E
:10534900B91DF8A70322EFF88DF0A4FFEDC5F0CE43
:10535900A42EFEEC88F0A42EFE22EB8AF0A4FBE535
:10536900F0CC8AF0A42CFC22EB8AF0A4FBE5F0CC6B
:105379008AF0A42CFCE435F0FD22EB8AF0A4FBE5CD
:10538900F0CC8AF0A42CFCE435F0CD8AF0A42DFDF4
:1053990022EB8AF0A430E70205F0E5F0CC8AF0A40C
:1053A9002CFBE435F0FC2286F0E7FDA4FAABF019FA
:0653B900E786F0A42BFBC7
:1053BF00E435F0FC18E68DF0A42BFBEC35F0FCE4A3
:1053CF0033FDE687F0A42CFCED35F0FD22EB89F0E0
:1053DF00A4CBAEF08AF0A42EFEE5F03400FDEC89EC
:1053EF00F0A42EFEE5F03DFDE433CC8AF0A42DFDB4
:1053FF00E5F03CCEFC22EB89F0A4CBAFF08AF0A411
:10540F002FFFE5F03400FEEC89F0A42FFFE5F03E0E
:10541F00FEE433CC8AF0A42EFEE5F03CFCED89F0DF
:10542F00A42EFEE5F03CFCE433CD8AF0A42CFCE581
:10543F00F03D8E058C068F04FF22C2D5EC30E705B8
:10544F00B2D51255EEEE30E70DB2D51255E6125425
:10545F007C1255EE800312547C30D5031255E62290
:10546F00C3EC13C0E0ED132FFFD0E03EFEBC000BEA
:10547F00BE0029EF8DF084FFADF022E4CCF975F07A
:04548F0008EF2FFFF4
:10549300EE33FEEC33FCEE9DEC994005FCEE9DFEF5
:1054A3000FD5F0E9E4CEFD22EDF9F5F0EE8420D23C
:1054B3001CFEADF075F008EF2FFFED33FD400799AB
:1054C3005006D5F0F222C399FD0FD5F0EA22EC3352
:1054D300EE3400FEEF3400FF7D007A007900780996
:1054E300C3ED9AFDEE9BFEEF9CFFB392D54009ED11
:1054F3002AFDEE3BFEEF3CFFA2D5E933F9ED33FD88
:10550300EE33FEEF33FFD8D92279007A00C380153A
:1055130079007A00C3EA13FFE913FEE8132BFBEECD
:105523003CFCEF3DFDE4F5D2F5D333FE7F19C3EE2A
:1055330098FEE5D299F5D2E5D39AF5D3B392D54047
:105543000DEE28FEE5D239F5D2E5D33AF5D3A2D54F
:02555300EB3338
:10555500FBEC33FCED33FDDF0122EE33FEE5D23308
:10556500F5D2E5D333F5D380C3EDC454F0FEECC4D6
:10557500FF540F2EFEEF54F0FFEBC4540F2FFF2204
:10558500EC75F00A84FCEB54F025F0C475F00A8440
:10559500C4CBC454F025F0C475F00A842BFBE5F0A8
:1055A50022AC10AB11125585A904AD03FA7C197B09
:1055B50099125363AE04AF03EA75F006A4F8AC1272
:1055C500AB131255852875F00A8485F014F8EF2B76
:1055D500FFEE3CFEEF28FFE43EFEE43DFDE439FC32
:1055E50022C3E49FFFE49EFE22E4C39DFDE49CFCF0
:1055F50022C3E49BFBE49CFC22C3E49BFBE49CFCF0
:10560500E49DFD2275D4107B807A0079807800EACC
:0A561500F5F0A4FCADF0EBF5F0A4F5
:10561F00FEAFF0EB8AF0A4C333C5F033C5F092D5DB
:10562F002DFDC5F03EFEE430D501043FFFB5150D4D
:10563F00EEB51409EDB51305ECB51201224006EADB
:10564F0098FAEB99FBD5D40ABB0001220ABA0001E4
:10565F000B22C3E913F9E813F8EA28FAEB39FB80B8
:10566F00A478087B807D807C00EDF5F0A4FAE5F04E
:10567F008EF0B5F007EA8FF0B5F001224003ED9BF5
:10568F00FDD827BDFF0122EDF5F0A4F9A8F0ED0438
:10569F00F5F0A4C399FAE5F09813CA1329F9E83A7B
:1056AF00F8C3E99FE89E50010D22C3EB13FBED2BCE
:1056BF00FD80B6C374689511FB74019510FC8004CE
:1056CF00AC10AB117A0B79B81253DC80177473F8E6
:1056DF00F9E627FB0809E637FC0809E637FD30E74E
:0556EF00031255FEEB63
:1056F40033FBEC33FCED3323FD242083F8ED241C31
:1057040083FFED241883FAED241483F9EF99F9E863
:105714009AFA1253DCEF9DFFE89EFE22FFFFFFB6CC
:10572400FED7FD63FB5DF8C4F59BF1E3ED9EE8CF86
:10573400E379DD9ED743D06BC919C153B91CB07945
:10574400A7709E06943F8A237FB674FF6A045ECBDB
:10575400535B47BB3BF1300423FB17DE0BB2FF80E6
:10576400C21DC232532CF8C3E5679576FBE56895F4
:1057740077FCE5699578FD30E705D2611255FE2482
:10578400F05003125838AA06A907125405EC2480D5
:10579400E43DFBF9F51AE43EFCFAF519E43F600236
:1057A400D2321253DC8B128C138D148E15C3E56424
:1057B4009573FBE5659574FCE5669575FD30E70525
:1057C400D2621255FEEBF9F51FECFAF51DED6002FD
:1057D400D232303201221253DCEB2512F512EC35B1
:1057E40013F513ED3514F514EE3515F51540E102F6
:1057F400560912576420323BEB242E40D3EA24018D
:10580400CB3400FC7A07793D1253DCC010C0118EF2
:10581400108D118C128B13E4FCFD7E077FD012B522
:0E5824007C851203851302D011D010BB000545
:10583200BA0002D21D22B261C374809BFB74F59C34
:10584200FC74209DFD22204D69204866303F637F15
:10585200697E0112CA287E1F12CA9875A700900499
:10586200EDE0A2E792171392E7FC1582E013FB30FA
:1058720017031255F6BC003AEB603720E73420E6F6
:105882003110E513201707C3741F9BFE80027E1F91
:1058920012CA8D0EDBFA22FB2017097E00C3742088
:1058A2009BFB8008EB241FFE74209BFB12CA870E11
:1058B200DBFA2275A700758307E559C4440FF58208
:1058C200E0A2E792522212C84B1258B5C2E775F015
:1058D2000A84FEAFF075A7045382F1786412593E30
:1058E200AE07786712593E75A700E57DC4540FFED6
:1058F200E57D540FFF7873125932AE07787612594C
:105902003274AF1256DE1257F68B148A1312092024
:10591200ACCCAB017A0A125363E5139B9004ECF012
:10592200FBA3E5149CF0FCA2E7923DD23F02C851D2
:10593200860308860408860518188006E0FBE0FC4A
:0A594200E0FD7A0A12538320E70CFF
:10594C00EB2EF608E43CF608E43DF622C3EB9EF69B
:10595C0008EC9400F608ED9400F622204D0920483E
:10596C0006C23F302A0522C23380F6E54824F640B1
:10597C00F5E5580460F075A700758307E559C42454
:10598C0008F582E0FEA3E0FF1209207437125A2AB0
:10599C00500B30381BC23878C586468013743212CF
:1059AC005A2A400C203809D23878C5A646754600CC
:1059BC00740D125A2A404A1258C8303D3820112210
:1059CC00204D1F20481C204019BCFF16EB243250E0
:1059DC0011D240120E62E5BF75F019A4F536D22E25
:1059EC00D22F205238E55965586032204D2F20486F
:1059FC002CD2338028201109204D062048037536FF
:105A0C0000303319204D1220480F1291460559C30E
:105A1C00E55895595003855859C233C2402229FB89
:105A2C00E435CCFCC3EB9FEC9E22E558B4FF01227D
:105A3C0085581175A704758307E54824F650028034
:105A4C005C201259202905202A02805112C84BE4EF
:105A5C00F516F517751000125AC2E510700312C82E
:0B5A6C0045125ADB302910E51B2517FE
:105A7700F517F51BE51C3516F516F51C125AE81235
:105A8700C8450510C3E511951050D175A70002C888
:105A970051E55AF51124F6500375110A75A70475D7
:105AA7008306751000125AC2125ADB125AE8051003
:105AB700C3E511951050EE75A70022E510C4F582D5
:105AC700E0E0F564E0F565E0F566E0F567E0F568C8
:105AD700E0F5692275A701125ED4123ED775A704B7
:105AE70022E9F0E51CF0E51BF022E510C454F0F5BF
:105AF70082E0F512E5822406F582E0F511E0F51C57
:105B0700E0F51B22E512B426157F757E34740D125D
:105B1700D51C20442575110012CEE6025C397F6D35
:105B27007E3BE012D501E5137E3512D501E5127EE5
:105B37002F12D50120440312CEE612CE52025C3951
:105B4700202852E558B4FF012275A704758307E59D
:105B570059F51030330965586005204802051012C1
:105B67005AF1E0F513305E07204304E5376095E00E
:105B77007F797E3D12D4CFE5137E3912D4CFE5125B
:105B87007E3512D4CF30480B7F7F7E3512DE5A0E1A
:105B9700BE40F980392012012275A7047583068556
:105BA7005B10125AF1305E0A204307E53770030293
:025BB7005D5B34
:105BB900E512700B7E3A7F79745D12D501800D75FF
:105BC900F06484E5F07E397F7A12D451E537B40266
:105BD90005128FDE8045B403028040E51C7006E59E
:105BE9001B24FB5036E511F964B4602F20062CE51F
:105BF90037600D200C0AC3E99570F9500324B4F9F4
:105C0900E912DCDF781D79547D1D90D82BE53F2002
:105C1900E00390D83212DDDD12D52D75177975168E
:105C29001930280375161DE51264266003125C7C81
:105C390075A7009006E3E511F0A3120E7BE5BC758C
:105C4900F01970040475F014A4951BFBE5F0951C7C
:105C5900FC922450031255F6ECF0A3EBF0C24FC2AC
:105C690063EC700EEB24E64002D24FEB24C84002ED
:105C7900D26322E51C24ED402BAE1CAF1B125E9EA5
:105C89007C007D3212547CC005EFAF17AE1612D4DA
:105C99000ACE2405CE742C12D5010E0ED0E02312A3
:105CA900D404801B125E95125CD6CE2405CE742CCA
:105CB90012D501CE2402CEE875F0058412D4E7CEC0
:105CC9002404CE7422305D02748302D4FDEE243D97
:0D5CD90050047EC37F4B7C017DF412547C8F
:105CE600C004C005EF6007AF17AE1612D40AD0077E
:105CF600D0067C007D3212547CA805EFAF17AE1695
:105D0600CE240ACE02D4E7125E95EE2450305D030F
:105D1600EE24A150047EC37F4B7C017DF412547C9B
:105D2600C004C005EF6007AF177E2F12D457D00707
:105D3600D0067C007D3212547CC005EFAF177E374B
:105D460012D4BC7E3B742C12D4CF7E3DD0E075F0CD
:105D5600058402D4BC7F6D7E2F746312D501E512D3
:105D660075F06484E5F07E3512D39912CEE602CE44
:105D76005230480320740122E4FCF5A79006E3E0C4
:105D8600F9A3E0FE24FE40EFA3E0FF7D78E537604F
:105D960008304FE3200C2A800B120E67E5BD20E089
:105DA60010304F0DD206E57124FE5015125E8B8021
:105DB600107D3CE546600A7D141460057D0A14706A
:105DC600B6891112534F7D6F12546FBE00A9EF248E
:105DD600E240A4AD07E51112DCDF202404B2D5B2FF
:105DE600D1781F795612DDDDA806A907E511242D05
:105DF60075F0B484E5F012DCDF7407304F02740EE0
:105E0600FDFA12DDDDB2D5B2D112DDDDB2D5B2D1E9
:075E1600DDF0AD0212DDDD3D
:105E1D00850616850717B2D5B2D112DDDD85061EB2
:105E2D0085071F7A03304F027A06E511241675F0A7
:105E3D00B484E5F012DCDFA816A917AD0212DDDD82
:105E4D00DDFBE51124EA400224B412DCDFA81EA913
:105E5D001FAD0212DDDDDDFBE5377021304F1E90E9
:105E6D00A60D305D0390A6097F3C7E331277351267
:105E7D000E67E5BD20E00612CA9E12D7CC22C3E9FB
:105E8D009570500224B4F922E51B2402FFE4351C61
:105E9D00FE305D1ABEC305BF4D028012AC06AB07C6
:105EAD007A1B1253717832125513AE04AF03227858
:105EBD007379641256E01257F6751CC3751B4B208F
:105ECD0032048B1C8A1B22125EBC30320122AC19AB
:105EDD00AE1AA91DAF1FB90005BC00028010C3E9A1
:105EED0013F9EF13FFC3EC13FCEE13FE80E8BF298B
:105EFD00005006BE2900500122C3EF13FFC3EE135D
:105F0D00FE80EB3E7FE3E3E3E3E3E3E3E3E3E37F01
:105F1D003E0C1C3C7C7C1C1C1C1C1C1C1C7F7F3EDA
:105F2D007FE3E3E3070E1C3870E0E3FFFF3E7FE302
:105F3D00E3030F0E0F03E3E3E37F3E070F1F3F77EE
:105F4D00E7E7FFFF0707070707FFFFE0E0E0FEFFBA
:105F5D00030303E3E37F3E1E3F73E0E0E0FEFFE358
:105F6D00E3E3E37F3EFFFFE3E30303070E1C383853
:105F7D003838383E7FE3E3E37F3E7FE3E3E3E37FBF
:105F8D003E3E7FE3E3E3E37F3F030303E77E3C0015
:105F9D000000181818FFFF18181800000000000066
:105FAD00000000FFFF0000000000003FF00000387F
:105FBD001C38F00180C1F020F0FC0038F03FE0000B
:105FCD000000007CC6C6C6C6C6C6C6C67C183878D4
:105FDD001818181818187E7CC6C60C183060C0C664
:105FED00FE7CC6C6061C0606C6C67C0C1C3C6CCCCC
:105FFD00FE0C0C0C0CFEC0C0C0FC0606C6C67C3CDC
:10600D0066C0C0C0FCC6C6C67CFEC6C6060C18302F
:10601D003030307CC6C6C67CC6C6C6C67C7CC6C6FD
:10602D00C67E060606CC78000018187E7E1818006D
:10603D0000000000007E7E00000000000000000057
:10604D000000000000C6E2E2D2D2CACAC6C6C20033
:10605D000000000000000000008080A0C0A0003003
:10606D004020C08080C0A0A0000060A0600000A003
:10607D0040A05098D090882050A850888850A850A3
:10608D002060806000000040E040000000000080C3
:10609D000000E000000000000040002040800040B3
:1060AD00A0A0A04040C04040E0C02020C0E0E020C3
:1060BD004020E02060A0E020E0C02020C06080E013
:1060CD00A0E0E020404040E0A0E0A0E0E0A0E02023
:1060DD00C0004000400000800080002060E0602093
:1060ED0000E000E00080C0E0C080E0E0E0E0E00023
:1060FD000000000040A0E0A0A0C0A0C0A0C040A033
:10610D0080A040C0A0A0A0C0E080C080E0E080C022
:10611D0080806080A0A060A0A0E0A0A0E0404040F2
:10612D00E0202020A040A0A0C0A0A080808080E022
:10613D00A0E0A0A0A0A0E0E0E0A040A0A0A040C0F2
:10614D00A0C0808040A0A0C060C0A0C0A0A0608002
:10615D004020C0E040404040A0A0A0A060A0A0A072
:10616D00A040A0A0A0E0A0A0A040A0A0A0A0404062
:10617D0040E0204080E02020A870202070A8202042
:0D618D0008F030D0100000F0A8A8000000BD
:10619A00E0000000902048708898984000E0E0E015
:1061AA0000A0E0E0E04060301030604040E0404055
:1061BA0060909090909060206020202020706090E5
:1061CA0010204080F06090102010906010305090A5
:1061DA00F01010F080E010109060609080E09090D5
:1061EA0060F0102020404040609090609090606085
:1061FA00909070109060C0E0F0F8F0E0C0000000ED
:10620A000000000000000000000000506050007014
:10621A007050000078807008F000F8888888F800CC
:10622A00C0C8102040981800C0B098B0C0006020C4
:10623A0040000000000090D8FCD8900000246CFCBC
:10624A006C24000020A870A82000002020F820203C
:10625A000000000000000080000000F000000000C4
:10626A0000000000606000081020408000708888EC
:10627A00888888702060202020207070880810206C
:10628A0040F8F810201008887010305090F810105C
:10629A00F880F008088870304080F0888870F80824
:1062AA00102040404070888870888870708888788C
:1062BA0008106000606000606000000080000080DC
:1062CA0000002040F84020000000F800F80000001C
:1062DA002010F8102000708808102000200000000C
:1062EA000000000070888888F88888F08888F0881C
:1062FA0088F070888080808870E09088888890E034
:10630A00F88080F08080F8F88080F0808080708843
:10631A0080B8888878888888F888888870202020BB
:10632A00202070381010101090608890A0C0A090A3
:10633A0088808080808080F888D8A8A88888888803
:10634A0088C8A898888870888888888870F088881B
:10635A00F080808070888888A89068F08888F0A08B
:10636A00908870888070088870F82020202020206B
:10637A00888888888888708888888888502088884B
:10638A0088A8A8A85088885020508888888888506B
:10639A00202020F80810204080F800CCAC9CACCC1F
:1063AA000000CCD4E4D4CC0004781828C800FC40FF
:1063BA00A04018202018000000000000F80000008B
:1063CA0000A040A05000788888986870884030887B
:1063DA0070200000F0A8A8A8A878484848487888FB
:1063EA0070888080887020A88898A8C8888880507B
:1063FA0048FC485080304C5C6060603C00E0F0082B
:10640A000808F88044485C484480F880808080808E
:10641A008078484848484888B8A8A8E8A8A8B8880A
:10642A0088888888F808500070888888708080F08A
:10643A0088888888F8888888888888F090909090DA
:10644A0090F0A8A8A8A8A8A8F8888888F808080832
:10645A0050008888888878A8A8A8A8A8F808000002
:10646A000000000000000000000000008888888802
:10647A00E8A8E8A8A8A870A8A8A80000000000003A
:10648A000000000000000000000000000000000002
:10649A000000000000000000006000606000600072
:1064AA0060006060205020000000005090B890D03A
:1064BA0090886050500070705000882020887000CA
:1064CA000080C0A090F8003048B4B448300030488A
:1064DA00B4B44830FC0098D02058C800F8E8D880F6
:0A64EA00D8E8F8404050F850404058
:0300000002005E9D
:03000B0002B60C2E
:0C000E00206E06859950D26E32D26F32FF
:0E00230010990AC298206DE385994FD26D3274
:10003800E4F537F534F52F12DE50C229C22AC2681A
:09004800C227C214C215022D9C4E
:03005B00022B2A4B
:10B5FF008530F0C5F065308530F060F722C0D0C0DF
:10B60F00E0C0F0C0A775A700C083C08275D00875D1
:10B61F008A00300503758A7A758CEA0532E5327037
:10B62F000215320530E530640A6026201520E53119
:10B63F00B40C0BE530B4010612BA8712D903E53109
:10B64F00B4180BE530B4060612BA8712D90302B844
:10B65F0026C2AFD2C075C07AD2AFF5300531E53111
:10B66F0064197040F531201529C225C22C7D0A744A
:10B67F000412DF01EF33EE339005CCF0EE24F540EA
:10B68F00112402400B24014005DDE4022B2AD225B0
:10B69F00D22CE5A6600215A678B5E660011678B63D
:10B6AF00E6600116302E0BE5367007C22FC22E1240
:10B6BF00B9B4E5367004C24B8002153678A9E6603E
:10B6CF00011678D8E66001160535E5357002153597
:10B6DF00E590307B0B30E008D278C27BC200801A35
:10B6EF00307C0B30E108D279C27CC201800C307DF6
:10B6FF000930E206D27AC27DC202E59044F8F470B6
:10B70F0003753500304A09E53324FA5003753305C4
:10B71F00E5336005153302B7CBE590F4540770039A
:0DB72F0002B7CBA2E09200A2E19201A2E2DB
:10B73C00920230100320143D75330820001B20109A
:10B74C000C2011098013E59030E10E8006E53724BA
:10B75C00FC40F3E543541FF53320100375A6FF207E
:10B76C002E5D301004E536705620100C201109E5C2
:10B77C003524F55003753304D21BD2A5D2A612B9C9
:10B78C00B475B44075B24078D8E670020534202701
:10B79C002E20682B202928202A25A2107211501F38
:10B7AC00E52054076019E53424375004C24A800F51
:10B7BC002401400B200026200119D27D7534C820AD
:10B7CC001558E531702412DEE174E812DEBA802AD5
:10B7DC0002B8F9E53724FC40E6D27C80DF3011DF7B
:10B7EC00E53724FC40D9D27B80D275F00384E5F098
:10B7FC0070DE12C53674E812DEBAE531B4060512F5
:10B80C00C6AE8016B40C0512C6C4800EB412051256
:10B81C00C6AE8006B4180312C6C4E59030E10530FC
:10B82C00E202800620100820110520103C807D20AB
:10B83C0027F82068F52029F2202AEFE5342430403F
:10B84C00E9240750E5600B205E088590F020F20299
:10B85C00740190B86E93D2A5201002C2A512B99FA4
:10B86C00806FC8A08269554646202F12E536603C91
:10B87C0024AA500AE53675F01984E5F06040D2A68A
:10B88C00201002C2A6D2A5202F0C7418304B0274C3
:0EB89C006412B99F803BE53675F00C3048030E
:10B8AA0075F00684A2E0744640E9743780E5E52B1A
:10B8BA005403600C20100E301106E54A640260053C
:10B8CA0012B9BA800312B911101B08A25892A5A284
:10B8DA005992A675A700D082D083D0A7D0F0D0E025
:10B8EA00D0D0201009C5A67003022B2AC5A632C2E1
:10B8FA0018B40202D21812C5D430180874E412DE41
:10B90A00BA02B80602B80178A7E5B4600924E04093
:10B91A0005760002B9BAE534702920412220751F44
:10B92A00300D1CE57924CE40167AFFE5B110E70107
:10B93A000A2325B3F5B3EA35B4F5B4C313F5B2E671
:10B94A0060021622C2412075028075E579FF6058AF
:10B95A0020120424FD5051206502C21CD265FF2426
:10B96A00B050027F4FEF90BA379375C70375C6FC84
:10B97A0075B90185BFF0A4E5F0F624F44002760C0F
:10B98A00301C2DE5BEC39FF5F0A4E5F024E040038A
:10B99A0075F020E5F0C21C79AA770375B300F5B4F7
:10B9AA00C31375B100F5B222C26578A77680D24179
:10B9BA0079AA7703D21CE4F5B3F5B4F5B1F5B2224E
:10B9CA00C26579A1E57924CE500DE720E7E2762811
:05B9DA00301CDD743299
:10B9DF0080BE7680E720E7D3E5799740CE79AAE756
:10B9EF00FAE5792323B4C500400274C42437300E1E
:10B9FF0031F42437300D15F7BA0302FA0AC39AF55A
:10BA0F00B175B300EAF5B4C313F5B222101C07D217
:10BA1F001C76C802B9A1763274FF200E02749B0205
:10BA2F00B9A1C313247E80CCFFF3E8DDD3C9C0B81E
:10BA3F00B0A9A29A948F8A85817D7975716E6B6892
:10BA4F0065625F5C595653504E4C4A4846444240DB
:10BA5F003E3C3A383634333231302F2E2D2C2B2AB0
:10BA6F00292827262525242423232222212120208B
:10BA7F001F1F1E1E1D1D1C1CD2B5C28EAE8DAA8D82
:10BA8F00AF8BAB8BE4F58DF58BD28E301401227812
:10BA9F00B6BE0007EF24E24002800806E624EC5011
:10BAAF00027614206705E624F64005E4FEFAFFFB54
:10BABF007C007D0A12534F7C007D5E12546F8F51B4
:10BACF00EE60037551FFEAFC7A33125363EBF5F026
:10BADF00A4E5F0CB8CF0A425E0C5F035E0CB92D5F2
:10BAEF0025F050060BBB0002D2D530E7060BBB008A
:10BAFF0002D2D5ECF5F0A42BFBE5F03400FC30D5E9
:10BB0F00010C78A6E6C39BFF18E608F6EB18F618AB
:0EBB1F00E69CFE18E608F6EC18F6301401223B
:10BB2D007A0050040A1255E67C007D6E12546F8F18
:10BB3D00F078A2E6A4FBACF0125585EBBA0002F446
:10BB4D0004FAE4F8FFEA30E70118E579600620759C
:10BB5D00031FF4042AF579EF38D27520E708600346
:10BB6D007579FF02C807C2750470F5E579F40460B4
:10BB7D00EFF57980EE120E5D78BBA6BC120E7BE55B
:10BB8D00BE78A2F624F65007E4F5BEF6124EE61284
:10BB9D000D46E5BEF54824F65008E4F5BEF548120D
:10BBAD004EE6E5BFF54324F3503924F34035120E2C
:10BBBD007178A1A6BCE5BF789DF61424FB500874DE
:10BBCD0003F6F5BF124EE678B7A6BE120E67E5BDB9
:10BBDD00A2E39266A2E49267035403C253B4010236
:0EBBED00D25322740DF5BFF543124EE680C010
:10005E0078FFE4F6D8FDF4F5A6D2B4D2C075C07A16
:10006E0075D75075AE1375AF017581D87590F8754B
:10007E00EFBC75FDFFD2A412DE27C2A47450122B62
:10008E0042758951D28C75A882D2BC12BBFB12DE8E
:10009E00E112C4AC12BB8212D9B6122A087F407E7E
:1000AE0001909C73127702124D4A12DE2712DB0862
:1000BE0012DD3F12DE507C1412DE31300003022BB3
:1000CE002ADCF512489F753A001248EDE53A701693
:1000DE0012DF157F437E0690A3F012770212DD3FEA
:1000EE003000FD022B2A75A6FF12489F12BB82120A
:1000FE002A0812DD3F12DE2312DE5078B5761E126C
:10010E00D9B612C4A1C215C214122A08909CBA7F85
:10011E00781276F0205E0A7F767E12909CC712D5FA
:10012E002D7F4012DDB57F497E0978AEE612D39958
:10013E007E15743A12D5017E1AE53E12D3997E26AB
:10014E00743A12D5017E2BE53F20E00805A6E5A600
:10015E00700215A6E53F12D3997F5312CA1C7F5722
:10016E007E0B12D2C612D34E7F602073030202089A
:10017E007E0BAC5DAB5C12D2CA12D34E7E311277BF
:10018E008D7F697E1212D8513025087E1290DB7158
:10019E0012D52DE5A60303543FFDFE0D7F7312DE2F
:1001AE005A0F12DE5A1EDDF478B5E57124F64002C0
:0801BE00761E307419E660564C
:1001C6007F727E16744012D4CF7E17E612D4577E05
:1001D6001F745312D4CF12DD3F10003710013710B1
:1001E600023712483FD2AC75369612DBB7B4E0053B
:1001F600124935800AE53670F112488D12DE20026A
:10020600010D2074097E2BE52E540712D4EE7E17BD
:1002160002018C022B2A022D628072E53524C85019
:1002260049E59020E244D0E0D0E012027102735614
:10023600E53524D25034E59020E22FD0E0D0E0120C
:10024600DF158038E53524D25020E59020E21BD01A
:10025600E0D0E012DF15306B0B7F091276E7124F04
:100266001E127BBD1202710206BE2212DF1590A479
:10027600A87F001276F012DD3F02DE2012DF159015
:10028600A4A87F001276F012DD3F12DE23C215C24B
:1002960014C227C26812DE50753701909DA3121C46
:1002A600FF9002AB730200F70217C2020B56021F41
:1002B60012021F0E0206BE0206FB0273560202C699
:1002C60012DE5075370790A140121CFF9002D673BC
:1002D60002029302096B0209A50209D90202FA0277
:1002E60005AD0202C60202C60203180202FF024B55
:1002F600B30203261248F0805A7F517E00747212B0
:10030600D4FD121E5C40B9124E3512D9B612BB820C
:1003160080AE7F49A25E120D31925E120D5080A012
:100326007F64120E9E121E5C401DE5352480F47516
:0C033600F0198460157F727E1F12D4EE57
:1003420012DD3F1001E810000280E30202C612BC77
:10035200680202C6124EE612DE5075370290A319E9
:10036200121CFF900369730202C6020EA8020F0D4F
:10037200020F61020FB6020FFA02100902035902BC
:10038200051302038980D0D21412DF157F147E0573
:1003920090A362127702121E1912DD3F124868758D
:1003A200A6FFD2AC1000DE12DBB7204CF2B405EF90
:1003B200E4F511F514F5151204411204D51248683A
:1003C20075A6FFD2AC1000BD12DBB7204CF2B415FB
:1003D200051204C880E7B406E712047FE51424FC82
:1003E20050D5E4F56FF56EF56D12048B1204D5123B
:1003F200486875A6FFD2AC10004212DBB7204CF25F
:10040200B415051204C880E7B406E71204B5E56F17
:1004120024F050D5124868743B12DC337A47909C22
:100422006A1224C9742A12DC27909C731224C9749C
:100432002A12DC27DAF912DC5012DE31020359AC3F
:1004420014AB157A0412536375A704900400E4F008
:10045200ECF0EBF08514C78515C67F08120467DF40
:10046200FB75A7002275B901E5BCF0E5BDF0E5BE5C
:10047200F0E5BFF005C6E5C6700205C722E5152402
:1004820008F515E43514F5142275A704900400E567
:100492006F4410F0E56EF0E56DF0740312BC347F2A
:0404A20020E4F5F766
:1004A600C2B2C2B2E5F7F0DFF4D2B275A700227489
:1004B60020256D54E0F56DE4356EF56EE4356FF587
:1004C6006F2205117F287E00E51112D41080069058
:1004D6000402E070177F287E15900400E012D41005
:1004E6007E2A900401E012D41012DD3F124868748F
:1004F6003A12DC6A75A7009004007F23E0A312DCA1
:1005060006DFF912DC413099FD2202035912DF158C
:100516007F0F90A69C1276F0121E1912DD3FC214B0
:10052600C21512DE207510651000DFE53170F9E5A1
:10053600106465700D855E14857A15E4F512F51361
:10054600800C78A8E51326F513E43512F5127F1E04
:100556007E19E51012D3B6C3E57A9515F517E55E53
:100566009514F5167F287E0BAC16AB1712D2CA125D
:10057600D34E12DD3F12DE31D510ADAB17E516FCBA
:1005860030E7031255F67A0A79001253DCA912A84D
:1005960013125515EBF510243840037510C8120ECA
:1005A6005D8510BC02035612DF15909CFE7F017E0E
:1005B60009127702909D067F0A7E091277027F1341
:1005C60012CA14751700120E6CE5BC12068DE5BD35
:1005D60012068DE5BE12068DE5BF12068D909D565C
:1005E6007F5F7E06127702121E9E12DD3F75170090
:0605F60012066D10000862
:1005FC0010011510024880F20517E51724F7500377
:10060C0075170075100080E2E51764087015120E5E
:10061C006C75BC0175BD2375BE4575BF67124EE682
:10062C000205ADE51012069F12DD3F12064D0510B6
:10063C00531007E51724FE400353100380AC02024D
:10064C00C6A9BCAABDABBEACBFE5171304F8E64007
:10065C00085407C42510C4800454702510F6027D7C
:10066C00A17800E875F009A42417FF7E3B7D20E8F3
:10067C00651770027D89ED12D50108B809E502DD18
:10068C003FF8C4120693E812069F7E030517E51780
:10069C0002D4EE540775F009A4909D0E2582F582C4
:1006AC0050020583E51775F009A42417FF7E0C0290
:1006BC007702C26812DE50753705909EE6121CFF59
:1006CC009006D073020293027941027986027B1C58
:1006DC000206BE0206F4027A5E027AC402178B028C
:1006EC0006BE021771020C627F2E12168680C31290
:1006FC00DE50753706909FC4121CFF90070B7302D7
:10070C0002930217C802182A0218A30219700219C0
:10071C00A2021A19020750020749021A62021B07A9
:10072C0002072F7F64120E67E5BDA2E7120D31128E
:10073C000E67E5BD92E7F5BD124EE680B27F491219
:10074C00168680AB12090C122B6912DF15121DF3E1
:10075C00E55804607790A0951207F912871E12DDF8
:10076C003F10000810011310021C80F50559C3E559
:10077C0058955950D575590080D01559E55930E721
:10078C00C985585980C4E559B40F02802FB51F0292
:10079C00802A75F007A42408F51775162774B82558
:1007AC0059F987001207E712DD3F100028100128C5
:1007BC0010020280F574B82559F9A700E53524FA22
:1007CC00508878C7A64812090312DF1512DD3F12B4
:1007DC00DE230206FB1880CC0880C9E875F005A45E
:1007EC0085F01CF51BC000125C7CD000221287AF78
:1007FC00B4FF0122751000751FFF1287C6E5106447
:10080C000F6017120830401274B82510F8E675F016
:10081C0005A485F01CF51B125D0D0510C3E558955C
:10082C001050D7221211AEF8602E6404602AE8141E
:10083C00B51025F51F120E7BE5BC70060475F0147F
:10084C00800375F019A485F01CF51B125D0D7E223A
:10085C0090A63D127735D322C322E558B4FF01226E
:10086C00751000E510640F602EE51075F007A424D8
:10087C0009FF74B82510F8E61208ED75F00A84C06B
:10088C00F07E2012D4577E28742C12D4CFD0E07E68
:01089C002A31
:10089D0012D4BC1208AD0510C3E558951050C322F3
:1008AD001211AEF8603964046035E8146510702FCC
:1008BD00120E7BE5BC1208EDF8C313923D7E1C129F
:1008CD00D46D7E28742C12D4CFE4303D067405B857
:1008DD000001147E2A12D4BC7E18742312D4CF22A8
:1008ED00305D1275F036A42432FBE435F0FC125560
:1008FD0085125585EB221209151276D5DFFB2212D2
:10090D000915127EB1DFFB2275C70375C6F078B8E5
:10091D007F042275C70375C6F375B901E5BFB548E8
:10092D0031E55924F1402BE55975F00484A9F024E3
:10093D00F0F5C675B901C5F0A9BC600CA9BD146070
:10094D0007A9BE146002A9BFE975F005A4F985F0E9
:10095D00CC22120E7BA9BD75CC0022124EE612DE02
:10096D005075370390A1AD121CFF90097B730202E5
:10097D00C6020C7B02131F020C90020C9B0216E6A2
:10098D000213A6020D5C0213DA02142002173802BC
:10099D00138E021465124EE612DE5075370490A2C6
:1009AD0072121CFF9009B5730202C6020CAA020C4A
:1009BD00B50209A5020CCB020CD60210230209A523
:1009CD00020CE5020CC0020CFF124EE612DE507551
:1009DD00370B90A2C2121CFF9009E9730202C602E6
:0B09ED0010D10210D1020A6F020AAD07
:1009F800020A10020A330217CE02117602123E02D0
:100A080011E70212CF020D19120E67E5BF1470C16B
:100A18007F2E120E9E1F120E67E5BDA2E6120D3143
:100A2800120E67E5BD92E6F5BD80A37F37120E9ED4
:100A3800120E62A8BFE8120A6712DD3F1000081004
:100A4800010D10021280EE18B802EA780A80E60852
:100A5800B80BE2780380DE120E6288BF0209D67FE7
:100A6800367E2CE802D39F7F1C120E9E120E67A8BA
:100A7800BE120AA112DD3F10000810010D10021469
:100A880080EF18B800EB780B80E708E824F450E111
:100A9800780180DD88BE0209D67F1B7E35E875F0B7
:100AA80005A402D3997F25120E9E120E67A8BF12C5
:100AB8000ADF12DD3F10000810010D10021480EF4C
:100AC80018B800EB780980E708E824F650E17801C7
:100AD80080DD88BF0209D67F247E3BE802D4EE126F
:100AE8000E5DE5BF75F03CA4ACF0FDE5BE75F00504
:100AF800A42DFDE5F03CFC120E67E5BF14603675C9
:100B0800F005A485BEF0A42DFFE5F03CFE7C007D39
:100B18003C12547CC005EF75F01884E5F07F2D7EFB
:100B28002412D3997E30743A12D5017E35D0E01262
:070B3800D39902DD3F7F2D80
:100B3F007E0590A65F127702120E67E5BDA2E67FD3
:100B4F002D12161502DD3FD25712DF15121DF312AB
:100B5F000B640202937F177E02909E041277027F2E
:100B6F004C7E02909E1C127702AC5DAB5C7F577E71
:100B7F000412D346120E8A85BC6285BD63E56124DB
:100B8F00F84044909E287F371276F0AE61AF607CBC
:100B9F00017D5E12547CC3741F9FFAAC63AB62EC91
:100BAF0033921750031255F6125363AB047C003087
:100BBF0017031255F674F52BFB74033CFC125339D3
:100BCF007F377E1512D2BE909E357F697E0F1277CA
:100BDF0002E560240FFBE43561FCA25C923BD25C22
:100BEF007E1E12D2CAA23B925C7E30742012D501B7
:100BFF007E36742012D501E5602562FBE561356311
:100C0F00FC7F227E0412D346E56245637016742E74
:100C1F007E3A12D50112DD3F10000D1001151002A2
:100C2F0026020B8C742080E81562E562B4FF0C1568
:100C3F006380080562E56270020563E53524F550AF
:100C4F0003753301020B8C120E8A8562BC8563BD5E
:100C5F00024EE67F637E00747212D4FD121E5C405A
:100C6F00087F631276E7124EED0206BE120E71E593
:100C7F00BCA2E77F0A120D34E5BC92E7F5BC02096E
:030C8F00687F1C5F
:100C9200A20D120D31920D80097F25A20E120D3187
:100CA200920E120D5002096B7F0AA20F120D3192A1
:100CB2000F802A7F13A208120D319208801F7F52E3
:100CC200A20C120D31920C80147F25A20B120D3151
:100CD200920B80097F2DA209120D319209120D503B
:100CE2000209A57F49120E67E5BDA2E3120D31127A
:100CF2000E67E5BD92E39266F5BD0209A27F5B1223
:100D02000E67E5BDA2E5120D31120E67E5BD92E553
:100D12009243F5BD0209A27F6D120E67E5BDA2E006
:100D2200120D31120E67E5BD92E0F5BD0209D61231
:100D32000D468F1F9217120E9EAF1F1F7E3912840F
:100D42000BA21722120E7685BC2B85BD2122120E14
:100D520076852BBC8521BD024EE6203714120E711A
:100D620085BE12120D89120E718512BE124EE680D8
:100D7200057F3F120D7B02096B7E0390A239127729
:100D82000212DD3F02DE2075A6FF12DF1512B5FF4B
:100D9200740712DF018FF0740612DF01EF2512C310
:100DA20095F0A2E7923D4010FD24CD50027D32AC79
:100DB20005C3743F9DFD800FF404FD24C850027DDD
:100DC20037AC0574402DFD7F4012CA147E1212DE2C
:0F0DD2005A0EBE1EF91F303D020F0FEF6D70ED70
:100DE100E536700A753606EC2513F5148C13120ED0
:100DF1000712DD3F1000071001083002072215120B
:100E01008002051280827F377E28742E12D5017FE1
:100E1100347E21740A303D010412D51CE514FC24F2
:100E21009C50027C637F347E2DEC12CE407F437E4A
:100E31001E12D2C67E00E51212D45D7F057E02909D
:100E4100A2451277027F6D7E0190A2501277357F05
:100E5100747E0490A262127735021DF375C6F48088
:100E61003575C6F5803075C6F6802B75C6F78026B8
:100E710075C6F8802175C6F9801C75C6FA8017758C
:100E8100C6FB801275C6FC800D75C6FE800875C64E
:100E9100FF800375C6FD75C70375B9012274721F02
:100EA10012D4FD0F02DD3F7F0A120E9E7E2A1248E8
:100EB100F0120E7BA8BF120EDC10001210010510FB
:100EC100021580F508E824E750EC781880E818E866
:100ED10030E7E3780080DF88BF805F7F097E05907F
:100EE100A520B80C0390A51A1277027E27E53D28AC
:100EF100240C75F01884E5F012D3997E33743B12FB
:100F0100D5017E35E53E12D39902DD3F7F13120EE6
:100F11009E120D46120F3E10000810010510021717
:100F210080F2105C07205D0BD25C80E8105DE5D299
:0D0F31005D80E1D25C80DD852BBC020356A3
:100F3E00205C10205D1890A5737F127E231277021D
:100F4E0002DD3F90A587205DF090A57A80EB90A5FD
:100F5E008080E67F1C120E9E120E76A8BF120F988E
:100F6E0010000810011110021A80F2E824F250034A
:100F7E001880EA780D80E6E824E740030880DE78E2
:100F8E001980DAE8F5BFF54380A37F1B7E26E412B5
:100F9E00D4EEE82323B464087E26740112D4EEE462
:100FAE007E2E12D39902DD3F7F25120E9E120E85E4
:100FBE00A8BCE8120FF112DD3F10000810010D1051
:100FCE00021F80EEE824E050E9188006E824CF40A6
:100FDE00E108120E8588BC124EE6D21512D9B680E3
:100FEE00D180157F247E3724E202D40A7F2EA20AF6
:100FFE00120D31920A120D500203597F37120E67ED
:10100E00E5BDA2E4120D31120E67E5BD92E49267C2
:10101E00F5BD0203567F367E00747212D4FD0F7E2C
:10102E0016743F12D4CF120E71A8BD12109C12DD91
:10103E003F10000810010510021080EFE8248750C1
:10104E0004240A800224E8F880E17F377E1674209B
:10105E0012D4CF7E2C743F12D4CF12109C12DD3FCF
:10106E0010000810011410022080EF18B80904783F
:10107E007880E7B878E478E780E008B87904780AF1
:10108E0080D8B8E8D5787980D188BD0209A2E82445
:10109E0087923DE8500224917F367E30C313923BF7
:1010AE0012D40A7E3CE4303B02740512D4E77E1A59
:1010BE0090A466303D0390A46A1277027F3C7E3A7C
:1010CE0002DE5A7F127E00747212D4FD0F7E2074DF
:1010DE003F12D4CF120E5D85BE1085BF111211586E
:1010EE0010000810011110021B80F21511E511B449
:1010FE00FFEB75111780E60511E51124E850DE753A
:10110E00110080D91211587F137E20742012D4CF73
:10111E007E31743F12D4CF12DD3F10000810011142
:10112E0010021B80DF1510E510B4FFD875100B8070
:10113E00D30510E51024F450CB75100080C6120EA6
:10114E005D8511BF8510BE0209D67F127E24E51182
:10115E0012D3997E30743A12D5017E35E51075F0B2
:10116E0005A412D39902DD3F7F49120E9E1211AED5
:10117E00F81211B410000810010D10021280F218AE
:10118E00B8FF02780480EA08B80502780080E212FF
:10119E000E5D88BD124EE6B800030209D902123E5A
:1011AE00120E5DE5BD227F487E0590A48012770267
:1011BE00E8601CB4040A7E0590A475127702800CB8
:1011CE0090A48C1277027E38E812D4EE02DD3F90A6
:1011DE00A4877E2912770280F31211AE601D64047B
:0211EE00601986
:1011F0007F5B120E9E120D46121219120E7610000F
:101200000B10010810020C80EF0209D9105FE9D21F
:101210005F80E5852BBC0209D61211AE601F640405
:10122000601B7F5A7E0590A4801277027E2390A4D3
:1012300090305F0390A49712770212DD3F221211C3
:10124000AE70030209D97F527E11120E9E120E7BE0
:10125000A8BC12127E120E7B1000081001081002AA
:101260000880EF1880EC0880E9120E7B88BC124ED3
:10127000E6120E85E875F005A4F5BD0209D6121137
:10128000AE604BE875F03270040475F028A4ADF040
:10129000FC305D11ACF0FB7A8A125371EB30E7053C
:1012A0000CBC00010DAE05AF047C007D6412547CC3
:1012B000C005EF7F517E1A12D3B67E2C742C12D546
:1012C00001D0E07E2F12D3991241B712DD3F227F69
:1012D00064120E9E120E7BA8BD121300100008109F
:1012E000010F10021680F218E824CD50EC783280FD
:1012F000E808E824CD50E2780080DE88BD0209D6F7
:101300007F63E823C2E012CF7375F06484C0F07E7F
:101310002612D4EE7E2C742C12D501D0E080A47F4E
:1013200013120E9E120E71E5BCA2E7923DC2E7F8C1
:10133000E812135E12DD3F10000810010D100212BA
:0313400080EE1824
:10134300B800EA783280E608B833E2780180DEE854
:10135300A23D92E7F5BC79A1F78079547F305C0117
:10136300237F127E2375F00A84C0F012D40A7E2DE7
:10137300742C12D501D0E07E2F12D4E70F7E359066
:10138300A58D305C0390A5E90277357F64120E9E2C
:10139300120E7BE5BE7F637E2C128460F5BE79A2BC
:1013A300F780317F37120E9E120E76A8BC530003CE
:1013B3007F367E32E812D4EE12DD3F1000081001B2
:1013C3000710020780E718180880E2E5BC54FC48C0
:1013D300F5BCF52B0209687F49120E9E120E85A8F3
:1013E300BE12141112DD3F10000810011110021A71
:1013F30080EFE8240AF8242450E778DB80E3E8242C
:10140300F6F8247F40DB788180D788BE80C6E8F475
:1014130024DC75F00A847F487E3B02D4EE7F5212AF
:101423000E9E120E85A8BF12145812DD3F1000083D
:1014330010011110021A80EFE82408F8245750E72E
:1014430078A880E3E824F8F824A040DB786080D70C
:1014530088BF0213D7E8F424A923C47F517E3B023B
:10146300D4EE122C74754A00D210C211D214D27564
:1014730075791475340012DF157F007E0290A21A6D
:101483001277029041E07F087E2612D52DE52B547A
:10149300030F7E3912D4EE121E0E12D197128ED183
:1014A30012DD3F10000810011A10022480C52075B8
:1014B30004057980BE1579E579B4FF05C2757579A0
:1014C3000180B02075EB1579E57970A7D27580A3FB
:1014D300C210C21402096B120E76E5BE7F097E3A72
:1014E30002D4EE120E7BA8BF120EDC120D46120FB1
:1014F3003EA8BF120F98120E85E5BC120FF17F2D87
:10150300A20A1216157F36A267121615120E5DE592
:10151300BC7F487E3202D410120D467F1BA20D12EF
:1015230016157F24A20E121615120E71E5BC1213A6
:101533005E7F09E5BCA2E7121615A8BF121724E5C2
:101543002B54037F367E3212D4EE120E7BE5BE7F20
:10155300637E2C12D4EE120E85A8BE121411A8BFFE
:10156300121458120E67A8BC021769120D467F09A0
:10157300A20F1216157F12A208121615120E67E596
:10158300BDA2E37F48121615E5BDA2E57F5A1216E8
:10159300157F51A20C1216157F24A20B1216157F6C
:1015A3002DA209121615120E71A8BD02109C120E5F
:1015B3005D85BE1085BF11121158120E67A8BE12A9
:1015C3000AA1A8BF120ADF120AE7120E76E5BE7F50
:1015D3003F7E3A12D4EE120E62A8BF120A67120EB1
:1015E3005DA8BD1211B4120E7BA8BC12127E120E9E
:0415F3007612121941
:1015F700120E7BA8BD121300120E67E5BDA2E07F95
:101607006C800B7F098040120D467F48A25E744EA6
:10161700400274597E3A02D501127DAD7F73127A6A
:101627000B127DFC7F6C127A1A7F2D801A120E67BF
:10163700E5BDA2E77F63121615120E76E5BE7F0998
:101647007E3A12D4EE7F4812166EB40104BF090128
:10165700E4F51075F005A47E1E909F952582F5820E
:1016670050020583027702120E67E5BD035403C2D9
:1016770034C25330E103D2342230E002D253221273
:101687000E9E1F12164E12DD3FE5101000121001BC
:101697000610020280ED22045403B4030AE4800713
:1016A700145403B403011423C5BD54F925BDF5BD76
:1016B700124EE680CE1275D1EBF516F5147F6C123B
:1016C7007A1A1275B57F647E23E51612D46DC3E5C9
:1016D700169514F5167F73127A0B7F2D02164E7F1F
:1016E7002E120E9E120E71A8BFE824FA400330375F
:1016F70002780312172412DD3F10000810010D10A5
:10170700021280E518B800E1780580DD08B806D92F
:10171700780180D5799DE8F7F5BF0209687F2D7EAE
:101727002C7420B80502742E12D5017E32E802D43B
:0C173700EE7F5B120E9E120E67A8BCE84D
:1017430012176912DD3F10000810010D10021280FC
:10175300EE18B800EA780380E608B804E27801805E
:10176300DE88BC0209687F5A7E2CE802D4EED26878
:1017730075480A1248F0D214122B77127EE5123301
:10178300CFC26B12024A80F3D214751501127D6722
:1017930075B901E5BC20E71C127E9775A6FF127E82
:1017A300F1121E1912DD3F12780B10000F500512B3
:1017B300793380E70515E515242050D10206BE12C2
:1017C30017D40202931217D40206FB1217D402098C
:1017D300D91217E0120E768548BE024EE6122B6927
:1017E300122B83125A3612DF1590A03FD24912876B
:1017F3004B128704121DC912DD3F1000141001059E
:1018030010021B80F50548E548640A7002F548801C
:10181300CF1548E54864FF700375480980C28548C1
:1018230049122B83E558221248F0122B6985484947
:10183300C250E558B40F02D250125A36803AD2271A
:1018430075480A122B77125A3612DF1512866E90DC
:10185300A43720290390A442121E8BC26A1233CFED
:10186300106A0280E1C227127D3F854948121C3667
:10187300122B83D229125A3612DF15909F511287E9
:101883004920500E121E7512DD3F1000101001AEDC
:1018930080F8121E1912DD3F10000280FB0206FBC6
:1018A300122B69E55830E7137F1B90A4217E0512A4
:1018B300770212DD3F12DE230206FB122B83125A3C
:0A18C3003685594912DF15121E0385
:1018CD0090A44212874912870E12DD3F10000810B6
:1018DD00010A10020C80F512193B80DB12194880A9
:1018ED00D612DF15121E0390A05012874912870ED3
:1018FD0012871212DD3F10000810010A10020C8031
:10190D00F512195480DB12196280D6121BFC122BB2
:10191D0083125A3612DF1590A389128749121E4180
:10192D0012DD3F10000510028880F80206FB0559F4
:10193D00C3E55895595003755900221559E5596459
:10194D00FF7003855859220549D3E5491495584030
:10195D0003754900221549E54964FF70058558490D
:10196D00054922122B69E55830E7057F240218AD91
:10197D00122B83125A3612DF1590A05B1287491273
:10198D001E8012DD3F10000A10010280F8121CA506
:10199D0080DE0206FB122B69E55830E7057F2D022C
:1019AD0018ADC26B7559FF125A3612DF15121DF3A1
:1019BD00E55930E703121E0E90A06D12874912876C
:1019CD001E12DD3FE55820E706100008100111102A
:1019DD00021B80F00559C3955950CF7559FF80CA28
:1019ED001559E55964FE70C285585980BDE55920D9
:1019FD00E711D26B75A700758307C4F582E0B2E7D6
:101A0D00F080A7306B03121C530206FB122B69E505
:101A1D005830E7057F360218AD122B83125A361255
:101A2D00DF1590A077128749121E5C4009121C9A8F
:091A3D00121CCF121A460206FB2E
:101A4600120E7BE5BD75F00584F5BCF5BDF5BEF55A
:101A5600BF120915124EE605C6DFF922122B69E5FB
:101A66005820E7087F5190A0800218B012DF159029
:101A7600A44D128749121E1912DD3F12484FD2ACEF
:101A860010001FE55830E7F8306DF5121B9C7E20DC
:101A96007F00501390A49E12773512DD3F12DE238D
:101AA60080CAC2AC0206FB1B8B13909F6E12773561
:101AB60012DD3FC26B7B007514B8121C8F127E6656
:101AC600127E185025A814E824384004A6010514EF
:101AD6000BC3E5139B50E678B8121CD1306B03128A
:101AE6007BBD122B83125A368082127DADE51660BD
:101AF600E6D26B127EC3C003127D7ED003A9158089
:101B0600C4122B69E55830E7057F5A0218AD122B2F
:101B160083125A3612DF1590A08B128749121E3691
:101B260012DD3F10003510010280F8754605121BC4
:101B36006450157F007E357407954612D46D12DD0C
:101B46003F12DE23D546E7D390A458500390A49EB7
:101B560012874912DD3F12DE2380B30206FB1248CC
:101B66004F12DC59745212DC6A745412DC27E558A1
:101B76000475590012DC481277BA4016127D3F12DE
:101B86007E9712780B400B0559C3E558955950ECD2
:101B9600C322C2ACD32212484FD2AC12DBB2204CC5
:0D1BA600F1B440F712DBB7B4400312DBB717
:101BB300B452E2F53812DBB7B454DA12DBB7FA6089
:101BC300D424EF40D012DBB7E53870C912DBB7126B
:101BD300DBB712779F7B007E03127896501020505C
:101BE300B412DBB7204C03B440F7DEED80A7127EBE
:101BF300760B12779FDAE0C322121CE0E55924C862
:101C0300F88602E54924C8F9986013146010500F50
:101C130018E608F618E86970F7A702121CCF22E548
:101C230059640F60F91908E618F608E86970F7A710
:101C33000280E8121CE078C8C250E6B4FF028007B5
:101C430008B8D8F6D25022B8D702D250A615807C55
:101C530078B8121CE2E4F9F5A7758307E9C4F582A5
:101C6300E030E70AE924B8F82438400276FF09C3D4
:101C7300E5589950E7121C9A78B879C8E6B4FF0280
:101C83008002F70908E8243850F2804079B877FFDA
:101C930009E9243850F82279C877FF09E924285044
:101CA300F822121CE0C23D78D7B6FF04A900D23D4A
:101CB30018B8C7F5203D0279D81978C8B6FF0122B4
:051CC300C3E899500781
:101CC800C6C7C6081980F478C8121CF1127ED31250
:101CD8007ED3127ED3027ED378C8121CF1127EB155
:101CE800127EB1127EB1027EB175C703E54875F068
:101CF80004A42480F5C62212DF15C23C1276F4E54E
:101D080037605314604D14604514603D14603514F9
:101D1800602D14602514600E14600B14600D14609F
:101D28001414600C803012160E802B1216BC8026FC
:101D38001215B1802112160A801C1216348017124F
:101D48001620801212156E800D12151B80081214B1
:101D5800E680031214DA12DD3F12DE27121DF31299
:101D6800B9C0A81F08E814C23BB51D02D23B75F0E4
:101D780007203C0375F009A4FF7E00303C0C74205A
:101D8800303B02743E12D4CF800A740B303B02748D
:101D98000A12D4E7D8CF12DD3FE51D100008100164
:101DA8001010021880B9651F7003751DFF051D808E
:101DB800AE7005851F1D80A7151D80A375F003A4AF
:101DC800227F7B7E0090A3A1127735E54824F64058
:101DD800087E0A90A40312773522127A377E05749A
:101DE8005B12D4CB7E1D745C02D4CB121DE27E3410
:101DF80090A3B2027735127A378003121DE27E3142
:0E1E080090A3B6027735121DE27E3190A4A998
:101E1600027735127A377E008005127A377E2D904A
:101E2600A4A9027735121E367E31909FA902773516
:101E3600121E197E1A909FAE027735121E1980C0A7
:101E4600121E197E18909F5B027735121E197E1A94
:101E560090A4AE027735121E197E1A90A4B312779B
:101E66003512DD3FD3100006C310010280F62212A0
:101E76001E197E1A90A04A027735121E197E1890F6
:101E8600A0660277357F007E2012773502DD3F128D
:101E96007A3790A4B9027733127A3790A4CA0277B8
:101EA6003312BE82120E94E5BDF55EF56CE5BCF507
:101EB6005FF56B756A007561FF75A70490070012E0
:101EC600BE2CB4FC23E582C313F561E56CF0E56B2B
:101ED600F0E582600F12BDA3E56C655E70E1E56B0F
:101EE600655F70DB75A700223024EA0460E7240FE3
:101EF60040D380E1E560758307C333F582E0A3F53F
:101F06006CE0F56B756A0022D2248002C224D214DA
:101F1600C21F121EA7756000E561B4FF1612DF1519
:101F2600909E387F0A7E0512773512DD3F12DE203D
:101F3600020293C210C21112DF15121DF3301F0ADE
:101F46007F07909E4612773380647F007E01C3E54B
:101F56006012D46D7E0E742812D4CB856048740747
:101F6600F51FFF7E00743E12D4CFE548121EFC1208
:021F7600C8237E
:101F78001224D80548C3E5619548FD401CE51F2497
:101F880007F51F24C850E17F387E01ED0412D46D97
:101F98007E0E742912D4CB800DE51F2407FF7E0125
:101FA80090A4A8127735201F0312251B12DD3F10BD
:101FB800001910012C10020280F5120236301F3D64
:101FC800020282101F02D21F021F39E56160F4E588
:101FD8006065617005201FF080E9201FE6056080BC
:101FE800E7E56160DEE56065617005201FD5800961
:101FF800201FD5E560700280CA156080CB121EA72D
:10200800121EFA12C82312260F756A1012BE151274
:1020180026C6909E4ED23C1276F4121D649020295A
:1020280073021F3902330F022049022035121E5C49
:1020380040CB121EFA12BE2CC2E2FF12BC52021F83
:102048001212DF157F6490A6821276F07F7990A62F
:102058008F1276F012DD3F75160010000A10010984
:1020680010020280F505160516C253121EFA12C890
:102078002375370A909E6A121CFF902086730220EF
:10208800050220AD02227C0222810220710220B4C6
:102098000220B90220710220F70220FB0220FF0271
:1020A800210602210A7F0A12168680BD124868801E
:1020B8000312485D780A1221D9740912DC2512220C
:1020C8001812DC4112225312BE1512BE3D12BD6415
:1020D80012BF54122362D5150C75150A1222661206
:0C20E800248912DC41100204E57F70DB4B
:1020F400022005780A800678048002780112486874
:102104008009780A8002780112485D1221D9740985
:1021140012DC1A122218E54812DC06E516540344B0
:102124003012DC27742A12DC2712DC2712DC41125D
:10213400225312BE1512BE3D12BD6412BF541223A7
:1021440062D51548854815122266E51C12DC06E5A1
:102154001B12DC06E51B2548F51BE4351CF51CE4C5
:10216400A27792E7A27492E0A27392E112DC06AD28
:1021740075AC74AB73E57DC412219AAD78AC77ABC2
:1021840076E57D12219A1224A712DC41100204E59F
:102194007F709F022005540F2375F00584F8C3EB6C
:1021A40033FBEC33FCED33FDC3EB33FBEC33FCEDE1
:1021B40033FD20E713EB28FBE43CFCE43D12DC0692
:1021C400EC12DC06EB02DC06C3EB98FBEC9400FC9F
:1021D400ED940080E88848121E20E4F54AF549751C
:1021E4006A2075150112BE1512BD64D5150E8548F9
:1021F40015E5492401F549E4354AF54AE57F70E5DA
:10220400744012DC6A747812DC27746312DC27745D
:0F2214002102DC1A122464E56012DC06121EFAA5
:1022230012C823E53A12DC1AE53B12DC1AE53C122C
:10223300DC1AE53D12DC1AE53E12DC1AE53F12DC3E
:102243001A740112DC06E54A12DC06E54902DC06D3
:10225300121EFA756A20E4F51CF51BF514F51375C7
:10226300150122753800E51412DC06E51312DC06AD
:102273000513E513700205142212486880031248FF
:1022830052121E201223BC12DE2B756A2075150113
:1022930075A6FF754A0112BDBD12BD6412BF54126B
:1022A3002362D5150975151E12238612DE351224F5
:1022B30089E57912DC06E412DC06E5711223471284
:1022C300DC06E57012DC06E57B24ACFFE55F340930
:1022D30012DC0CEF12DC06E51520E033857D56E4B5
:1022E30012DC06E52EC412DC0C12DC5012DE3510B3
:1022F300021A30559B744012DC27744512DC277494
:102303004F12DC27744612DC2712DC50022005E54D
:1023130056122321C4FAE57D1223212A80C2FBC46D
:1023230012232E2323CB12232E2B22540FFC24F60D
:1023330050027C0090233DEC932200000101010236
:1023430002030303FA2440400A24804003EA3322B1
:10235300D2E72274FF2220E703C3132224C022E51D
:102363003F701F7F7B7E0078AEE612D457EE2404C5
:01237300FE6B
:10237400743A12D4CFEE2404FEE53E12D45112DD99
:102384003F22C015C016D21212A6DAC212D016D03D
:102394001578AEE612DC1AE53E12DC1AE53F12DCD3
:1023A4001AE54512DC06E55212DC06740A12DC0654
:1023B40074C012DC0602DC50744012DC2774541220
:1023C400DC6A744E12DC27743012DC27E5165403E1
:1023D400443012DC27122464742112DC1AE53D1205
:1023E400DC1AE56012DC06121EFA12C82378ABE68A
:1023F4000812DC1AE60812DC1AE60812DC1AE612E5
:10240400DC1AE53E12DC1A1229EFE51212DC1AE599
:102414001112DC1A740112DC0690A4DB1224C975B3
:102424006A1012BE15057F057F787F12DBFF787B6B
:1024340012DBFF787D12DBFF787712DBFFE4FEFF0F
:10244400780712DBFF12DBFFE57412DC06E5751278
:10245400DC06E412DC06E412DC0612DBFF02DC50CC
:1024640075C70375C6FF75B901C217751D0085BC14
:102474001C85BD1B85BE1A85BF191252E9EE12DCFC
:1024840006EF02DC06E57512DC06E57412DC06E5EF
:102494007312DC06E57812DC06E57712DC06E576D5
:1024A40012DC06E51664016011E55E12DC06E57ACD
:1024B40012DC06E516640260012278BCE612DC0632
:0A24C40008E602DC0675A700E493A9
:1024CE00700122A312DC271A80F4AF1F7E0478ADB0
:1024DE00E612D4517E0C742C12D4CF7E0E18E61256
:1024EE00D4517E1A78AEE612D4517E22743B12D4A9
:1024FE00CF7E24E53E12D4517E2FE54012D4577E76
:10250E0037743B12D4CF0E0EE54102D45175320012
:10251E00121EFA12C823857946787A796412C83C5D
:10252E0074641256DE8E4712260F756A20D23D1243
:10253E00BE1512BE3D122646303D09307406C23D10
:10254E008E1E8F1FE57F602BE54C24FFF54CE54D6D
:10255E0034FFF54D454C600512BD7980D2751D3C9A
:10256E0012BE1512BE3D12BD64122646E57F6003F3
:10257E00D51DED1226A79026BF12D52D203D0DAEEE
:10258E001EAF1F1226A79026B812D52DE546FD7058
:10259E000B90A611305D1190A60D800C047010905A
:1025AE00A60D305D0390A6097F381241B2804BE430
:1025BE00FFFC7E05305D047E027FB312546FAC06C5
:1025CE00AB071253397F38C23DE51C6007D23D7E02
:1025DE002C12D4BCE51B203D026007D23D7E30128A
:1025EE00D4BCE51A203D026007D23D7E3412D4BC25
:1025FE00E5197E3812D4BC1241B7E53224C850FA20
:10260E0022E54075F03CA42541FFF54CE435F0FE83
:10261E00F54D7C007D1012547C0F8F4BAF4CAE4DA0
:10262E007C007D3C12534F7C00AD4B12547CEE4F20
:10263E0070010F8F4C8E4D2278647973C2D11226A1
:10264E005DFF78677976D2D112265DFE02DE5AC31F
:10265E00E796FB0809E796FC0809E796FDA2E792C4
:10266E001750031255FE75135A30D10E751320B242
:10267E0017AA47125383AB04AC05E546600B046002
:10268E000BAA4612539AEB03FBEB03FBEB543FFBF7
:10269E00E5132B2017029B9B22EE141430E701E466
:1026AE00FEEF141430E701E4FF2205057088A888B8
:1026BE007005052020F8202075320012DF157E1ED1
:1026CE007F1C12DE5ADFFB12DE5A7E1E7F1C12DECC
:1026DE005ADEFB7E1D7F1D12DE5ADEFB7F007E2141
:1026EE0078ADE612D4517E29742E12D4CF7E2D18D9
:1026FE00E612D4517E35742E12D4CF7E3918E612DE
:10270E00D4517F077E21745412D4CF7E25744F127C
:10271E00D4CF7E2D78AEE612D4517E35743A12D4D3
:10272E00CF7E39E53E12D45178AE1229EF7F0E7E60
:08273E0021744C12D4CF7E255A
:10274600744112D4CF7E2DE51212D4517E35743ADF
:1027560012D4CF7E39E51112D4517F157E257444EB
:1027660012D4CF7E2DE54012D4577E35743A12D45A
:10277600CF7E39E54112D4517F217E0190A5DC122E
:1027860077357E0EAC77AB7612D3037E2B85795FD9
:1027960085787B12D8AA7F287E0190A5E01277352E
:1027A600751D2B751E10E5741229A37E25742F1234
:1027B600D4CF751D2D751E2BE5751229A37F367E88
:1027C6000290A5CC127735E5721228501228E8122D
:1027D6001EFA756A209004E6E56CF09004E7E56B56
:1027E600F0AE4DAF4C7C007D4012547CBF00010F13
:1027F6000FAC07AD07E4FED23D12BE1512BE3D1268
:102806002891E57F602CE54C24FFF54CE54D34FF1F
:10281600F54D454C600512BD7980DE751D3C0E12E6
:10282600BE1512BE3D122896E57F600612BD64D520
:102836001DED1228667F7812CA267F767E007430D8
:1028460012D4CFE53224C850FA227E2112CF731259
:10285600D46D7E2F90A5E4305D0390A5E90277350F
:102866009004E6E0FD9004E7E0FCC3E56A9420FBF3
:10287600E56B9CFCE56C9DFD50032410FD12556E26
:0D2886009004E8EEF09004E9EFF022DD038D
:10289300AD040E7F78E55E20E72AE57A8549F0A44A
:1028A300A9F0E57A854AF0A429F9E435F0FAE55E62
:1028B3008549F0A429E435F02AFAE55E854AF0A4B7
:1028C3002ACF9FFF12DE5A103D18C3EF9B50131BF4
:1028D300EF6B600E8F018B0712DE5A1FEF6970F8E2
:1028E300AF01AB072290A591305C0390A5AA754A6E
:1028F30040754900AF76E577FE20E76B7005EF245E
:10290300105064EF24A8EE34FD401190A596305C7E
:102913000390A5AE754A1975499A8075EF2450EE58
:1029230034FB401190A59B305C0390A5B3754A0C12
:102933007549CD805CEF24A0EE34F6401190A59E3E
:10294300305C0390A5B8754A067549668043EF2449
:10295300F0EE34F1401390A5A1305C0390A5BD7552
:102963004A04754944802A8028EF2490EE34E840D5
:102973001190A5A4305C0390A5C2754A0275498FD6
:10298300800F90A5A7305C0390A5C7754A017549D0
:102993009A7F401277337F4612CA267F5F02CA2688
:1029A300AE1E75F064305C0375F03284C0F0F870CD
:1029B30004EE2404FEE51D12D4CFEE2404FEE860E9
:0129C300070C
:1029C40012D4BCEE2404FED0E075F00A305C03752A
:1029D400F00584A8F012D4BCEE2404FE742C12D4A6
:1029E400CF0E0EE8305C012302D4BCE53E2541F550
:1029F4001124C45003F511D3E63540F51224E850F0
:102A040002F5122212B9BAC21012DF157F057E092F
:102A1400909C6A1277027F137E08902A3C12D52D6F
:102A24007F2B7E01902AA412D52D20370A7F277E82
:102A340027902B1612D52D22113007FE1FE001E13D
:102A440001F80F00061B00F80C00180E007C1000A3
:102A54007006003C2000E006003E4001E004001E39
:102A64008003C004001F0003C004000F000780009F
:102A7400000F800780000017800F00000027C00FA0
:102A840000000043C00F00100083E00F002003018A
:102A9400F00700C00F01F80383007F87FE01FC00EC
:102AA4000E3E1800000300000000180000030000A0
:102AB40000003800000000000000300000000000AA
:102AC4000000FC761F0E1C6030ECFCBC3F172DF0A0
:102AD400F978613866264F619A706070C60E1EE3FD
:102AE40030E06060C60C1CC360C0E0618C0C18C789
:102AF400C0C0C0E18C1C39C611C0C4C19C993196B8
:102B04003180C8C1FF1E31E7E180F0C0EE1C31C343
:102B1400818006163091882892884924904927900C
:102B24009248A0E3C8BCC2AFD2C075C0107581D8AA
:102B340074FE122B42E4F5F9F5FBC2B480F7D2A679
:102B4400C2A512B99F12DE2702B9C075C703E548B2
:102B540075F004A42480F5C6C23C75B901E5BC0433
:102B64007002D23C22120E76E5BEF54824F65003DC
:102B7400754800753400753704C228D229D22A75E5
:102B8400C703E54824E75003754800E54875F00499
:102B9400A42480F5C6751607751700C23C122BC411
:102BA400122BC4122BC4122BC485175815587559EF
:102BB40000E548B40A09E5586005F46002055922A5
:102BC400203C1D75B90105C6AABCABBDACBEADBFEA
:102BD400EA122BE5EB122BE5EC122BE5ED122BE5BB
:102BE40022203C07F515B4FF03D23C22C0C7C0C65F
:062BF400127D6775A704C5
:102BFA00851683E517C4F8F58275B90105C6E5BCE3
:102C0A00F0C582F82406F92403C582E5BDF0E5BEC5
:102C1A00F0E5BFF075B90105C6E5BCF0E5BDF0E524
:102C2A00BFF08516838982E4F075B90105C685BCB3
:102C3A001385BD14E4F0F08882E5BEF0E5BFF075B7
:102C4A00B901E5BCF0E5BDF0E5BEF0E5BFF075837E
:102C5A0006E51723541E24B0F582E513F0E514F0B7
:102C6A0075A700D0C6D0C705172212BB8278BEA6A8
:102C7A004808E4F6F55908761808F6D23608760AAE
:102C8A0008F6060876BEC254C25512BE97122B77B2
:102C9A00C229C22AC207C227C268120E67E5BDA2AC
:102CAA00E59243C24AE4F52EF534F536F52F78B6A7
:102CBA00F678B5F678A9F6789EF678B8A65E08A6EC
:102CCA007A12D26CC26BC233C238C240C223C22249
:102CDA00122CF475460278C5A646C23AD221C21908
:102CEA00C226E4F542F541F54022E45407205E0984
:102CFA00B4040040027403801B120E6CC313A9BCF7
:102D0A00600C14A9BD600714A9BE6002A9BFE940FE
:102D1A0001C45407F53722122B69125A3612090CCC
:102D2A0012DF15121E41E55804700A7F327E0590A3
:102D3A00A42112770290A67912874B1208667F7235
:102D4A0090A66E1276F012DD3F1000051002048084
:102D5A00F8D322C3220200F7120E67E5BD20E70569
:102D6A00122D2140F0754E50122C7412852C754488
:102D7A00031248ED12AEFFD54403022B2A201EF19E
:102D8A00789F7680754A0012BCB3D210C211C21362
:102D9A00C21212483F75A60C12D9B612C4A1E5A6F2
:102DAA0024FA400612488D75A60C20250CE590548D
:102DBA00057009E53524E25003022E54E532241841
:102DCA00400D75F00C84E5F070D41233D280CFD266
:102DDA001ED2AC306DC87532F012DBBCB4E0BF1243
:102DEA004935E53124F39205201203123264122E7A
:102DFA001AC014128E17D014200A03122F3D123350
:102E0A00D212A6A91233D212852F1233D2022D9CC6
:102E1A0030122EE54024F0401C7A0AC3E53F954B58
:102E2A006013401E24E2400D305405C254757F01E0
:102E3A0012BCD9DAE679BCE7D2E7F57F09877EC208
:102E4A007722F40424E250ED80DE12DF157F2A7E19
:0C2E5A000E90A4DF12770275A6FFC210D4
:102E66001012137F367E08909F8C12770212DD3F78
:102E760012DE200200F7D22112491112BCE37F1E96
:102E86007E0B90A3FA12770212DD3F122EA77F3E29
:102E96007E0790A11E12770212DD3F12DE1A022B68
:102EA6002AD215D21412BE6E120D4675B90575B921
:102EB6000212BE78D25512BD9D7F0012BC5212BEC0
:102EC60078E56A600512BD6480F7857A62120E9411
:102ED60085BEBC85BFBD856BBE856CBF75B90575E6
:102EE600B90285BD6C85BC6B756A2012BE6E123048
:102EF600DE12BE78756A0012BE15E57064FE703487
:102F06007570FC854077854178851F797818797AC0
:102F160012C83C12BD1212DE3512BE78756A101246
:102F2600BE157F087810797212C83E85627C855E70
:102F36007D12BD12C2152212486812308A745212CE
:102F4600DC27744D12DC27744312DC2712309912E9
:102F5600DC627441207402745612DC27122FE612CA
:102F6600303012DC62E53C12DC1AE53B12DC1AE575
:102F76003A12DC1A12306612DC62744512DC271231
:102F860030CF12308A744712DC27744712DC27745C
:102F96004112DC27123099122FE612DC62E43074FB
:102FA600010412DC2512DC629004C3E012DC1A1262
:102FB600DC629004E4E075F00A84AFF012DC1A12C9
:102FC600DC66EF12DC25AC5EAB7A1230ABAC5DABE7
:102FD6005C1230AB12DC6212DC621230CF02483F68
:092FE6007875C23D122FF17878D4
:102FEF00D23D12DC62128211303D05E51E12DC2546
:102FFF00E51D12DC25123073E51812DC25E57D2066
:10300F003D01C4540F12DC2512DC62303D097445BA
:10301F0030170274578007744E301702745302DC56
:10302F0027207408123066123066802775A7049027
:10303F0004BFE0FCE0FB7A1B125371783212551378
:10304F001253391230709004C1E0FCE0FB12533977
:10305F0012307075A7002212DC62E4F51AF51980A0
:10306F000D12DC62E51C12DC25E51B12DC25E51ACE
:10307F0012DC2512DC66E51902DC25742412DC272C
:10308F00744712DC6A745002DC2712DC62E53D12D1
:10309F00DC1AE53E12DC1AE53F02DC1A12826D12D1
:1030AF00DC62E51D12DC27781CE612DC2518B81748
:1030BF00F812DC66E412DC2512DC62744D02DC27A8
:1030CF00C038742A12DC27D03812DC4102DE357882
:1030DF00107F0EE4F608DFFCF564F565F567F5681B
:1030EF007515FC751AC0751DC075664075694075FC
:1030FF004A0112BDBD30550302319412BD64E57112
:10310F00B510004002F510E4F511E512207502E547
:10311F0013C395795006207545857913D3E57A95B4
:10312F0014E5156480FFE55E64809F400C857A147A
:0E313F00855E15857B16855F173074B3C2D18F
:10314D007864797312317278677976123172D2D1CF
:10315D0078187973123172781B79761231728091E9
:10316D0085791280B9D3E7960809E7960809E664D0
:10317D0080FFE764809F20D101B3400AE7F618195C
:10318D00E7F61819E7F622E51AB4C00E7873791828
:10319D0012C83C7873796412C83C78187964C2D12E
:1031AD0012320574181256DE8E47AE1EAF1F781BF5
:1031BD007967D2D1123205C3E51F9FE51E9E5004DB
:1031CD008E1E8F1F7EFF7FFFAC1EAD1F12547C7AAB
:1031DD0004EF8AF0A4E5F0CE8AF0A42EFEE435F0DB
:1031ED00BEFF011E60051460057EFF8E1F22EE7E60
:1031FD000020E7F77EFE80F3C3E697FB0809E6970C
:10320D00FC0809E697FD1818191930E7031255FE49
:10321D00C3EB33FBEC33FCED33FDEB33EC33FBED68
:10322D0033FC30D105AA4712539A0BBB00010C7524
:05323D001E03751FFFD8
:10324200EC24FC40048C1E8B1FE627FB0809E637A2
:10325200FC0809E637A2E713F618EC13F618EB138D
:10326200F62210131978B5E624FA401AE57124F60D
:103272004008E57924F6400280360606803212DEE6
:1032820031E59030E2DF753612D22EE4F534F55A8C
:1032920012BEC91232B5C219C257122CF41291468B
:1032A200129173D212853F4B754C00205E02D228D8
:1032B200022CECD214123304E6F008DFFB857A62AA
:1032C2001232FA7570FE783A797112C83C12BD1248
:1032D2001232FA85627A855E7B120E8A85BC7E8501
:1032E200BD7F7570C012BD12123304E0F608DFFB19
:1032F20075A700D254C2142274FF7870F608B88001
:10330200FB2275A7049004F078707F1022121EFA37
:10331200122C7412DF1512DD3FC258C259754A01D0
:10332200753901756A2012BDBD1256DC8E47C21076
:10333200D211D214D21212BEC91291461291731234
:10334200D9B675A6FF753609753200E59020E206FA
:10335200E5352405400CE5905405701FE53524E25F
:103362005019C211C21212DF1512DD3FE4F535F514
:083372002F7E0612DE2DC202BF
:10337A00022005C221E54AB40202D22112BDBD12C1
:10338A00A6A930260F125A9812852F753606E536E9
:10339A0070FCC22612852C1233D2E54A20E021B4F1
:1033AA000209753900E53670F9808CE53960FAFD55
:1033BA0024E24002053912BDBD2026C9DDF880E9A4
:1033CA0075390080E475370410003A1001161002AE
:1033DA0016E52F5407600312B9B420783D20790A04
:1033EA00207A1F220235C802351CE53760091460AD
:1033FA00091460090236740235E7023645C27902B9
:10340A00369102354FE53724FC500FE537640760E3
:10341A000302370C0236D00234E62011FAE5902076
:10342A00E2028056753400201203D2132278A9E6EC
:10343A007017C226767DE5377005106B02D26BD203
:10344A0077753614D22E02BEBEE53760431460404B
:10345A00B40227200B24E6249B401F2414501C127C
:10346A00914690A3CD7F207E0812770212DD3F7528
:10347A003608D22E78A9E624ECF622241940FB2439
:10348A001450F712914612917390A3D67F2980D7D0
:10349A002028E7E54824F640E1E5580460DC7F5D32
:1034AA007E10E6249B40D324145015C2330559C319
:1034BA00E55895595005855859D22690A3BB80A93D
:0434CA00241940B6CB
:1034CE00241450B2E55960021559102606E55960CC
:1034DE0002155990A3C4808D10780122753900E52C
:1034EE003424384007754A0175340022700AE54AC3
:1034FE0030E0F2754A0280F0146008754A061291A7
:10350E00738006754A0412914675390180DA3029A6
:10351E0009C229D22A7559008005302A1BD22912D8
:10352E0086FA1286C8E53524AF400475340022753C
:10353E003700C229C22A80F3206841302703D26A9D
:10354E0022D2221238A812DD3F107A0122E534244D
:10355E00384007122CF475340022700FAA37122C43
:10356E00F46A70F27401122CF580EB04122CF5241F
:10357E00FC50E3E537B40706D22880DA8036C2283D
:10358E00E53724FC2324BEF879C4E7F9A74809A738
:10359E005979C4E8F78648088607E537B4050575F6
:1035AE004818D236122B838F59E53764067002D233
:1035BE000702356412388402382EE537601B14601A
:1035CE007614600F146009E53724F9400902378636
:1035DE000236740236BF023753D223124096107948
:1035EE000122E534243840077546017534002278EF
:1035FE00D87020304A0BC24AE624F85004B24380F9
:03360E000AD24A93
:103611007614E54624FE40DDE54660D9154680D89E
:10362100B600D5B40500500C04F54624FA50C9750E
:10363100460580C424F95005127B5B80BB100FB88E
:10364100D20F80B4D223E53464C8600312409610CF
:10365100790122E534243750097011105B32D25BB5
:10366100802E100802D2081240968024100C21D21C
:103671000C801DD22312409610790122D24BE534E1
:1036810024374010C258C259201105D22E75360771
:103691007534002224FD401524037006D258C25906
:1036A10080EEC258D2591460E7D25880E3120E71ED
:1036B100E5BCB2E7F5BC79A1F7124EE680D278B845
:1036C100A65E08A67A2011C8753605D22E80C130B3
:1036D100122B128734055BE55B75F00B84E5F0F581
:1036E1005BE55A24F64009E55A955B5003755B008A
:1036F10012873812DD3FE5346003D534D2753400CA
:1037010022D229D22A75480A0237F4C2401007F1A1
:103711003029030237F41286F612870A102A1BC2D7
:10372100330559C3E558955920E7025008755900EA
:10373100E548B41816E558B4FF0375590012871E01
:1037410012DD3FE5346003D534C122D22A1286FA54
:1037510080EE301223128734155BE55B30E70C7580
:023761005B0A01
:10376300E55A24F64003855A5B12873812DD3FE59C
:10377300346003D534DA75340022D229D22A75484D
:1037830017804CC2401007F22029441286F6128794
:103793000A102A22C2331559E55930E71C855859B6
:1037A300E558B4FF03755900E548B41802800AD2FE
:1037B3002A1286FA800E855859E558B4FF037559C5
:1037C3000012871E12DD3FE5346003D534B5222095
:1037D300106220115F7F180548E54864187008F5EA
:1037E3004830270375480A122B4F303C2DDFE88001
:1037F3002620105A2011577F181548E54830E70551
:10380300754817800A640970063027037548171234
:103813002B4F303C05DFE275480A122B83125A36D0
:10382300E532244C50051286C8800312866E753427
:103833000002DD3F12386B7F15E5486B70048A4840
:1038430080020548122B4F303CD0DFED80CC12387C
:103853006B7F15E5486A70048B4880021548122B6C
:103863004F303CB6DFED80B27A007B09E537B40414
:1038730001227A0A7B17B40601227418FAFBF54871
:103883002275A704758307E559C4F582E0E0F57353
:10389300E0F574E0F575E0F576E0F577E0F5787539
:1038A300A700025A36E59020E23EE534243750382B
:0638B3001238EC1238C9C6
:1038B900205E4F7F2C909D20123933909D29806A7C
:1038C900E534243775F009A42435FF205E0624BEAB
:1038D90050027F3EEF249B50027F627E3274891230
:1038E900D5012275A7049000317E087F3AE4F0DF04
:1038F900FDE5822446F582E43583F583DEED75A77F
:1039090000227F2C120E6CE5BD12391CE5BE12395E
:103919001CE5BFF8C4123922E8540775F009A490D0
:103929009D0E2582F58250020583EF2409FF027658
:01393900F09D
:108529000285E312DF15E53724FC40F4B4FE14207C
:10853900110EE590F45407600122E532247450EFDE
:10854900028E2312DF1512D6A412D73612CF81124A
:10855900D2C212D10B7E197F3612D05F12DC6F1294
:10856900D075C206E53760051460338053C23A12EC
:1085790086871241591242EE1245D41264F41265EB
:108589001C123E04E54864186009E54824F65003C6
:108599001246BF128DB912CE061241F48014D23A96
:1085A9001286AD1239421241C312C98C128DB91209
:1085B900CDC7125D7712D77D125848125B478012DA
:1085C90012869312C8C912D84D12C95B128DB912FD
:1085D900CDDE30101112D013800C12DF15E53724CF
:1085E900F9401E1286703022091238A8E53470024B
:1085F900C222302309124096E5347002C22302DDFB
:108609003F121DF375170012DA607F1212CA143077
:10861900124A75100075A704758306125AF1E51000
:1086290075F009A42415FFF5177E00E512602F7572
:10863900F06484E5F00F12D4511F7E0EE51112CFBC
:10864900C9751623125CAD0510C3E55A951040068D
:10865900E51024F550BF3012031287388088745D05
:1086690012D50180D5C249302905121DC9800312CE
:108679001DF3909F5112874B202A7602871E3012D4
:1086890023305E2030501D028A2F301217305E06CB
:03869900200B11A2
:10869C0002909012CA0D7F1712DDB575172002DA01
:1086AC006012D61B12D5BC30121120510512D67B8C
:1086BC00800612CD6112CB411251AB22E4FEFFE5D4
:1086CC004824F6400D90A4031277357E16E5480237
:1086DC00D4BCB40E0690A40902773590A41112777D
:1086EC00357E12E54824F702D4577D20800C7D3F5F
:1086FC00302A077D633029027D3C7F0080247D2059
:10870C0080127D3E800E7D3CE54975F007A4240661
:10871C00800A7D3FE55975F007A42409FF640270B7
:10872C0001FF7E1CED02D4CF7D2080027D3FE55BF6
:10873C0075F009A42416FF7E09ED02D4CFC24912AC
:10874C0087AFB4FF01227510001287C67920E03084
:10875C00E702792F3049171211AEFAB40408E5106C
:10876C00700C79658008EA14651070027923E97E33
:10877C001812D4CF7E20E51230E708909F8C127728
:10878C00358016E51112883C125D0D201005201164
:10879C000280063012031287EE0510C3E5589510BF
:1087AC0050A7227E207F001277351286C87E007F6C
:1087BC000690886E12D52DE5582275A7047583078F
:1087CC00125AF1E51075F007A42409FFF5177E0085
:0B87DC00E51212D4CF7805EE2404FE55
:1087E700E012D4CFD8F6221288F612890CFD7C004D
:1087F700AE1CAF1B12546FBE003A8F00C3E57A95CB
:1088070013FFE55E9514FE402B7C007D2812547CF7
:10881700C3EF98401F75F0058404FB24F950027BD1
:10882700067E2CAF170F12DE5A0F12DE5A0F12DE1A
:108837005A0EDBEF2264B4602464B475F03284C04E
:10884700F012D4BCCE2404CED0E075F00584C0F07D
:1088570012D4BCCE2404CED0E02302D4BC90886AC4
:108867000277352D2D2D000140FFFFFFE0FFFFFFB1
:10887700FFC25030123F20283CE558F460372048AB
:1088870003200931D250E559F51030330665586099
:108897000205101288C012891C75A7049006DCE532
:1088A70012F0E511F0E517F0E510F075A704900652
:1088B700E0ECF0EBF075A7002275A70475830712AB
:1088C7005AF17813E0F608B819FA9006D07811E64D
:1088D700F008B819FAE51CF516F0E51BF515F012C6
:1088E70088F69006DAE514F0E513F075A70022750F
:1088F700A704758306E51023541E24B0F582E0F51E
:1089070013E0F51422120E71E5BD2487E5BD923BF5
:0289170050020C
:1089190024912212890C75F005A485F012F511E451
:10892900F519FEF51CF51D12BE6EC23DC2567F3CFF
:1089390012CAB7303D05751900807DDFF3E5596529
:1089490058700A301007EE24D35002D2568C1B8D72
:108959001AE519FD24E250DEAE1CAF1D7C0012544D
:108969006FEFF51924F650CEAC1BAD1A12C9FC20D5
:10897900D1108E048F05E51975F0A7A4AEF0FF128A
:10898900546FAC12AB117AA012539AEB33FBEC3350
:10899900FC20D11AEF9BEE9C5014C3E51213FCE5A1
:1089A9001113FBC3EF9BEE9C4004AC06AB072048B8
:1089B90007203B048C128B119006E2E519F0128A0C
:1089C90004AC16AB157AC8125371A912A811125525
:1089D90015ED7005EC249E50057C807B0822C3E5CB
:1089E9007A305602E55C9513FFE55E305602E55D87
:1089F9009514FEC3EF9BFBEE9CFC22AE16AF157CD3
:108A090000E519FD24F6501A12546F7C007D0612F8
:108A1900534F7C007D0512546F8F10EEF51724E932
:098A290050037517FF2212CA0D5B
:108A3200128A4C128A8F12D271128AB520480912F8
:108A42008BA3128BD3028C3680747F177E20204832
:108A52000E748A204D101258B5500E742F80077470
:108A62006A305F02746712D50175A7049006D07848
:108A720011E0F608B819FA7F177E00781275190509
:108A8200E60812D501EE2406FED519F42275A704D4
:108A92009006D8E0F516E0F515E0F514E0F513E0E0
:108AA200F512E0F511E0F517E0F510E0FCE0FB75DA
:108AB200A700227F187E26AC14AB1302D3039006C4
:108AC200E4E0F51CA3E0F51B7F2A304E13120E677B
:108AD200E5BF90A46EB4010390A6681276F08042BE
:108AE2000F7E00745312D4CF9005CBE0F830E70527
:108AF200E53F30E0091F7E00E8540F12D4E79004EE
:108B0200EEE0FEF51EA3E0FFF51F128B4BE51E24DF
:108B1200E9500C7E06742B12D5017E0C12D501127F
:108B22008B7BC20375172A751627125C7C202415CD
:108B3200205F15D2037F2A7E1E908B69304E0390F0
:108B42008B7202D52D205FEB227C007D3C12547C7F
:108B5200A805EF7F2A7E0812D40A7E12743B12D433
:108B6200FD7E14E802D4040707384C9EBAF264383A
:0F8B72000707387CE6C2E67C38AC1CAB1B7A48A0
:108B8100305D027A27125371A91EA81F125515EDE7
:108B91004C60027BFF7F207E28EB12D4107E3902CD
:108BA10091237F2B90A417127733E517F46022AE3F
:108BB10017AF107C007D3C12547CA805EF7F2A7E04
:108BC1000C12D40A7E16743B12D4FD7E18E812D41E
:108BD1000422AE12AF117C007D0A12547CA805EF6D
:108BE1007F207E3012D40A7E3A742C12D5017E3C4D
:108BF100E812D4E70F7E29744502D4CF748580072B
:108C0100748720560274867E2912D50130170774A5
:108C11002D7E3A12D501227C007D0A12547CA805D2
:108C2100EF7F2A7E3012D40A7E3A742C12D5017E4F
:108C31003CE802D4E7128D67E54824F65005128C12
:108C41001880B9E559046558600D128C18128BFD16
:108C5100E559655860AA22A217923D8E1E8F18858C
:108C610015179006D0E0F51185581015101245B46E
:108C7100C3E51195105002F404F924A65005C374FC
:108C8100B399F9E975F00584F924EE500279119050
:108C91008DA7E993F5F0120920E5CC7004E930E7DE
:108CA10002747F23A4A9F0E51B2517FDE51C3516E9
:108CB100FEC3ED99F515EE9400F51675A7007583C1
:108CC10006E55823541E24B0F582E0A3F513E0F520
:108CD10014128D67203D2C201729120E71E5BD2439
:108CE10087E5BD5002249175F007A4FB9518E5F0C6
:108CF100951E400FEB9FE5F09E4008EF9518EE950D
:108D01001E500EA23D9217AE1EAF18128C18028B88
:108D1100FD306B10128D04E53F20E00774867E2242
:108D210012D5012275A7009006E0E516F0A3E5151E
:108D3100F0128C18128C0174857E2312D50185588E
:108D4100101288C0128A4C128A8F8C168B15128AC7
:108D5100B51289CA1288B212D2719006E2E0F519F1
:108D6100128A04028BA3C3E57A305602E55C95139F
:108D7100FFE55E305602E55D9514FE921750031231
:108D810055E6AC16AB157AC8125371A906A807129D
:108D910055157E037FE7ED700CEB2418EC34FC4095
:108DA10004AE04AF032200172E43576C8092A4B681
:108DB100C5D3DFE6EDF3F8FD305E4F30504C75A7BB
:108DC100009006E0E0A3FCE0FBECA2E79217402054
:108DD10024FE50047F3B8022AE04AF037C007D144F
:108DE10012547C74542F2017029F9FFF7462800CD1
:108DF1001255F6EC24FE50E07F6D743D7E0012D4D6
:108E0100CF7E017D197C03128E0C227F3D12DE5A2A
:108E1100EF2DFFDCF822E537B40206E534243750A4
:108E2100292212DF1512D6A412CF81128FA312C8E4
:108E31005712CDEE128FFB125B477F207E2B12D093
:108E41005F12D73612DC6F1238A812D197128ED169
:108E510012514502DD3F20041EE579FD24A0500298
:108E61007D5FED24CD401E744520750C2DFFF5125C
:108E7100128EA61FBF44F922C39DFFF512128EA6C2
:108E81000FBF46F92220750EED2413FFF512128E45
:108E9100A60FBF78F922C374779DFFF512128EA633
:108EA1001FBF12F922EF24BA40082433FCC37432E5
:108EB1009C1404FC24D750047C238009EC2375F016
:108EC10005842413FC7E0512DE5A0EECB506F82249
:108ED100E59020E206E53424374003128E577F45A2
:108EE1007E047D1212DE5A0EDDFA7F437E00746429
:108EF10012D4CF7F4F7D12128F8C7F3B7D12128F48
:108F01008C7F597D16128F8C7F317D16128F8C7F4D
:0F8F1100637D1A128F8C7F277D1A128F8C7F6DD4
:108F20007D1E128F8C7F1D7D1E128F8C7E057F19FA
:108F300012DE5A0FBF72F97804E57924CD50027819
:108F400009E8305C0123F87F1B128F7B7F6B128F47
:108F50007B18305C01187F25128F7B7F61128F7B1D
:108F600018305C01187F2F128F7B7F57128F7B1870
:108F7000305C01187F39128F7B7F4D7E00E875F0E1
:108F80000A847004E802D4BCE802D457EF6512608A
:108F90000C7E04EE20E00712DE5A0EDDF62212DE11
:108FA0008A80F790A52E7F287E2C1277357E3B1283
:108FB000D31AAC5EAB7A7F307E19C23D12D3599082
:108FC000A41B7F5D7E2D12773578B9C3E57A96189C
:108FD000FBE55E96FC7F507E19D23D02D359E51128
:108FE00064B4700122E51112DCDF7831790F7D0B5A
:108FF00012DDDD1F1E90908B02D52DE5716012E50C
:109000007012DCDF7831790F7D0412DDD90DBD0AD5
:10901000F97F011290637F1D1290637E2312906D81
:109020007E3F12906D7E247F171290777E397F02EB
:109030001290777E247F071290817E397F1C1290D8
:10904000817E317F0212DE5A7F1C12DE5A7F0F7E34
:109050002412DE5A7E3E12DE5A7F0C7E2E90D822DB
:1090600002D52D7E2A12DE5A0EBE39F9227F081251
:10907000DE5A0FBF17F9227D0612DE5A0E0FDDF9F8
:10908000227D0612DE5A0E1FDDF9220303E0A0E066
:1090900012CA0D7F18909D5E1277337F217E017476
:1090A0004112D4CF7F2A7E01745312D4CF9005BED3
:1090B000E0F51AA3E0F519A3E0F51EA3E0F51D8580
:1090C0001A1C85191B751720129140E519251DF5ED
:1090D0001BF51DE51A351EF51CF51E751729129195
:1090E000409005BA129130AC1AAB19751720129046
:1090F000FE9005BC129130AC1EAB1D751729EC70AB
:1091000006EB24CD4001227A48305D027A271253C3
:1091100071125515ED4C600122AF177E07EB12D38B
:10912000B67E1A0F90A5F1305D0390A5F402773555
:10913000E0FEA3E0FD12BFC4C3EB9DF8EC9EF92254
:10914000751627025CAD12BFC475A7049005B478EC
:10915000737F06E6F008DFFBECF0EBF0E0E0E0FC0C
:10916000E0FDE0FEE0FFEF2DFFEE3C9005C0F0EFEC
:0B917000F0801275A7049005BAE0FB28
:10917B00E0CBF0EBF0E0E0E4F0F075A7002275A790
:10918B00049005B478647F06E0F608DFFB75A70052
:0E919B00125EBC9005BEE51CF0A3E51BF022A1
:10393A00D23C799E77008002C23C12BE6EE4F5103A
:10394A00F511F512F513F514F515F516F517C23D2F
:10395A00123C8A203D1F123C8A203D19E51F30E5A2
:10396A001130E40E1239B1303C08799EE724F55043
:10397A000122D510DBAE14AF157C00AD12125449EA
:10398A008F55AE16AF177C00AD1312546F125670D6
:10399A007E00E55530E7011E2DFFE43E30E7027F49
:1039AA0000740A2FF55622C235E51CAF1DBFFF056C
:1039BA000FD235F404FABF003F532CF8E518AF19BB
:1039CA00BFFF050FD262F404BF002D20E72A205B57
:1039DA000123FF24AA4021E51AAE1BBEFF050ED221
:1039EA0061F404BE00128547F0A4E5F020E709203F
:1039FA005B0123FE24AA5001227C807B8030516621
:103A0A00302163C006C0078AF0E545A4AEF0FFE5A1
:103A1A0056205B011375F009A4ACF0FD12546F74C3
:103A2A00FFBE0001EFFA24C050027A3FD007D00649
:103A3A00E55212DCDF303504B2D5B2D1EA8CF0A4FB
:103A4A0030E70205F0748025F020D10495F095F056
:0A3A5A00FCEA8BF0A430E70205F04F
:103A6400748025F030D50495F095F0FBC3EC2F203D
:103A74006203C39F9FFFEB2E306103C39E9EFE2013
:103A84003C64200C05123B1E4064123B00405F1254
:103A9400DE5AE51EFD24FB50550E12DE5AED24F6C7
:103AA400504C1E1F12DE5AED24F150421E0F12DE3E
:103AB4005AED24EC50380F12DE5AED24E7502F1F34
:103AC4001F0E0E12DE5AED24E250231E0F0F12DEDB
:103AD4005AED24DD50180E12DE5AED24D8500F1E74
:103AE4001E1F1F02DE5A123B004003799E0722E983
:103AF400242AFFE82461FE123B1E401DEF2460408F
:103B040018243F5013EE2460400F243F500AEF2442
:103B1400D6FFEE249FFEC322D322532CF8432C0459
:103B2400EE10E706D2E7F404D261FE24D340EAEFB4
:103B340010E706D2E7F404C262FF24D340DBEFB5FA
:103B440006005003CED26070057480FE8062FF24AC
:0D3B5400FD5060903C0A938EF0A4AAF0335F
:103B6100CA33CA33CA33CA33CA33FA903C34938F47
:103B7100F0A433C5F033CA903C5593FB123BD29568
:103B810070500224B412DCDFEA8BF0A430E70205A6
:103B9100F0C3748095F020D50425F025F0FEEA8C61
:103BA100F0A430E70205F0C3748095F030D104250C
:103BB100F025F0FFC3227A01EE6F70097B16BF0278
:103BC100BB7A0380B7BF01047B0080B07B0D0A8004
:103BD100ABE52C540723C3903BDC73800E800E8031
:103BE10024801E8010800A80108012EB22742D9B8D
:103BF10022742D2B22745A9B22745A2B2274879B78
:103C01002274872B2274B39B22FFFFCCAA9280716E
:103C1100665D554E4944403C383533302E2C2A28B8
:103C2100272524232221201F1E1D1C1B1A1A1918A7
:103C31001817178181818282838384858687898A87
:103C41008B8D8F90929496989B9D9FA2A4A7A9ACCF
:103C5100AFB1B4B400010203040405060708090A60
:103C61000A0B0C0D0D0E0F0F10111112131314145A
:103C7100151516161612BDA612BC34E4F5F7C2B21C
:103C8100C2B2E5F7D2B264C022203D07123C767081
:103C910003D23D22056D056D12BC347D008DF7C246
:103CA100B2C2B285F71F8DF7C2B2C3E5F79573F5BE
:103CB100188DF7C2B2C2B2E5F79574F5198DF7C246
:103CC100B2C2B2E5F78DF7C2B2C3E5F79576F51A40
:023CD1008DF76D
:103CD300C2B2C2B2E5F79577F51B8DF7C2B2C2B295
:103CE300E5F78DF7C2B2C2B2E5F7F51E8DF7C2B2A2
:103CF300C3E5F7957AF51C8DF7C2B2C2B2E5F78D2D
:103D0300F7C2B2C2B2E5F7D2B2543F30E50244C0C3
:103D1300955EF51D156D156DE51024784001227E25
:103D230000AF55EF30E7011E0512E51FA2E592D55E
:103D3300400EE515951EF515E5149400F514800B5A
:103D4300E515251EF515E43514F5147800E51E6018
:103D53000620D50318F404C39FF5F0E89E30E7016D
:103D6300220513E5F0A42517F517E5F03516F5162A
:103D730022303D03D23D22123C7660F8123C76603D
:103D8300F3E546600A123C7660EA123C7660E5058C
:103D93006D056D056D12BC347D008DF7C2B2C3E5B0
:103DA300F79573F5188DF7C2B2C2B2E5F79574F5BE
:103DB300198DF7C2B2C2B2E5F78DF7C2B2C3E5F708
:103DC3009576F51A8DF7C2B2C2B2E5F79577F51B72
:103DD300D2B2156D156D156D2230742412BE6EC2EC
:103DE3003D75101E123D74203D167902123E484067
:0A3DF3000CA806A907123AF34003DA
:103DFD0012DE5AD510E422200F4030123D2006CF9E
:103E0D00304806200C03204FC6E546790260147930
:103E1D000614600F791614600A79361460057976E8
:103E2D0014701712BE6EC23D7896123D74203D0A75
:103E3D00123E48400312DE5AD8F022532CF8AB182C
:103E4D00E519FC339262123E9ABC002BEB89F053BC
:103E5D00F00784FF24DF401FAB1AE51BFC33926192
:103E6D00123E9AAA4712539ABC000CEB89F053F0FC
:103E7D000784FE24DF5002D32274562F2062029F46
:103E8D009FFF741F2E3061029E9EFEC322500312AF
:103E9D0055F6E920E40122C3EC13FCEB13FBE920FA
:103EAD00E50122C3EC13FCEB13FBE920E60122C371
:103EBD00EC13FCEB13FB2274542F2062029F9FFF27
:103ECD00741D2E3061029E9EFE2279B4203249204F
:103EDD001D46EFB506009260AC06AB074004AC077B
:103EED00AB06903F26EC2304938BF0A4A9F0EC23B2
:033EFD00938BF0B4
:103F0000A429F9903F8693C9904086E52C540793E5
:103F100013E95001F490408EF9E52C54079329756C
:103F2000F0B484A9F022FFFFFFFF7FFF55553FFF4C
:103F300033332AAA24921FFF1C711999174515556E
:103F400013B1124911110FFF0F0F0E380D790CCC60
:103F50000C300BA20B210AAA0A3D09D8097B0924BF
:103F600008D30888084207FF07C107870750071CC6
:103F700006EB06BC06900666063E061805F405D15B
:103F800005B005900572000000000001010101016B
:103F90000101010102020202020202020203030302
:103FA00003030303030304040404040404040405D6
:103FB00005050505050505050606060606060606A9
:103FC000060607070707070707070708080808087E
:103FD0000808080808090909090909090909090A55
:103FE0000A0A0A0A0A0A0A0A0A0B0B0B0B0B0B0B2A
:103FF0000B0B0B0C0C0C0C0C0C0C0C0C0C0C0D0D02
:104000000D0D0D0D0D0D0D0D0D0E0E0E0E0E0E0ED9
:104010000E0E0E0E0F0F0F0F0F0F0F0F0F0F0F0FB4
:10402000101010101010101010101010101111118D
:10403000111111111111111111111212121212126A
:104040001212121212121213131313131313131347
:104050001313131313131414141414141414141426
:104060001414141414151515151515151515151505
:1040700015151515151616161616161616161616E5
:1040800016161616161600FFFF00FF0000FF002E82
:10409000B5875B2D5A88E537607414603EB40258CA
:1040A0007F347E12E5342437400810644B90A3EC33
:1040B000801AF89041E012D52DE824FD501179A125
:1040C000E77E0590A22520E70390A22F0F803A24D7
:1040D000040F7E2312D4EED26480627F357E02E527
:1040E000342437401410641090A11530081B127747
:1040F000027E1A90A3EB801122700590A1278009FF
:10410000909D8B200C03909D9712770280C97F357C
:10411000E5342433402A2404501B7D0F600C7D1E9F
:104120001460077D3C1460027D78ED305D02C3139E
:104130007E2B12D3B67E0090A12812770202DD3FBB
:104140007E0524FE5005909F798009909D6E200F7A
:1041500003909D7A12770280E4E546604A14603C41
:1041600014602E14602014601290A625205D4190EA
:1041700041D97F367E3412D52D803C90A625305D06
:104180000390A621802A90A621305D0390A61D8071
:104190001F90A61D305D0390A619801490A61930BB
:1041A0005D0390A615800990A611305D0390A60DC1
:0241B0007F3658
:1041B2007E331277357E3C7422305D02748302D5E1
:1041C20001305D0890A5FD305BE4800690A60520D5
:1041D2005BDC90A60180D70508B28D8DB5BA0910B7
:1041E20006000A10F248922492249224F2480A10FD
:1041F2000600305E5220434F20284CE55864FF6091
:1042020046E54824F640407F3FE55804F9C23D1296
:10421200424A1211AE601AB404047401D23D75F020
:1042220003A4243CB5070A7E3A303D027E36124290
:104232004C0F0F0FD9D7E55975F003A4243EFF1296
:10424200424A0F0F12424A227E3D12DE5A0EBE40F1
:10425200F922C248C249305E56202853E55864FF0D
:10426200604DE54824F640471211AE6042D249B48F
:104272000402803B1465597036D248304E31E559FC
:104282006558602B3074281242B7120E67E5BFB42E
:10429200011DE5BD20E618202416205F129006E4D9
:1042A200E0700CA3E024CE400624255002055922DA
:1042B200305FFC80E820113375A7009006E4E070BF
:1042C20028A3E0302402F404305F02F4042404F949
:1042D20024F74015E924FC4003D26C2270012230FD
:1042E2006C097536A7D22ED22FC26C22305E0830EE
:1042F2007405E558B4FF0122C244C24D780075A787
:0B4302000475830712463688188A1ED7
:10430D008E168F17C23EC23BE54824F6500302437A
:10431D00C7D23EE55860F7E8655970F22048EF12B4
:10432D00447C30D13BAE16AF17A818E54670551238
:10433D000920E5CC49604DD244E5CC7033E924CD5C
:10434D00402EE975F038A4ACF0FB12558512558559
:10435D00EBFDF5111243DD304D2CC206C23B8043FF
:10436D00E546705C120920E5CC7005E924CD50506E
:10437D00124F7C75A704758307A8181246368A1E3E
:10438D008E168F178037120E67E5BDA2E0B3923BF4
:10439D005011307428123AF34026A907A806D20608
:1043AD0012CA9E1243F91243F01244398907880646
:1043BD001E1F90463112D52D800630D103124411A7
:1043CD00A81808C3E55898400302430075A70022BA
:1043DD0074562F2062029F9FF9741F2E3061029E2A
:1043ED009EF822E51865586001227D057A00EA12D3
:1043FD00DCDF12DDDD0A0AED24F240020A0AEA24AE
:10440D004C50EB22AE16AF17123EC41E303E021EAC
:10441D001EE51E12D4CFEE2404FEE51212D4CF30C9
:08442D003E09EE2404FEE51334
:1044350012D4CF22E5186558603CC001C000C012F7
:10444500C0138518101245B4D013D012D000D00176
:10445500E510303B07C39570500224B412DCDF2011
:104465003B07AE16AF171243DDE5112402FD7A06B0
:1044750012DDDD1DDAFA221211AEB40457E87054CC
:10448500120E85E5BD604D78C6A61308A61208A6CE
:104495002C12C84B75A704758307751001125AC2F3
:1044A50012C8451510125AC21256DC8E628F63125D
:1044B50057648B1C8A1B12C85120320E124564208A
:1044C5003B08D24D1266FF1244DA78C68613088679
:1044D5001208862C22120E85AABD7C027BB31253CC
:1044E5009A8C128B13AA1DA91F1253DCA91CA81B99
:1044F5001255158C1D8B1FAC12AB13AA19A91A12D4
:1045050053DCA91CA81B1255158C198B1AE56E25B1
:104515001AF9E56D3519F8C3E56E951AFBE56D9544
:1045250019FAC3E554951FFDE56F951DFCE5542566
:104535001FFFE56F351DFEE52C23652C30E206ECEB
:10454500CEFCEDCFFD75A7049005C2E8F0E9F0ECCF
:07455500F0EDF0EAF0EBF0DD
:10455C00EEF0EFF075A70022D23BC3E5649573C56E
:10456C00659574F564E5669575600404600822E54C
:10457C006424E0500822E5642420400122C3E5674E
:10458C009576F567E5689577F566E5699578600940
:10459C0004600122E566F48002E5668562F0A4748D
:1045AC00E025F04002C23B2212C84B75A70475836C
:1045BC0007125AC212C8450510125AC2C02C125A00
:1045CC00DBD02C891002C85130125120064E7800D5
:1045DC0075A70475830612463630D139123EC4E5F0
:1045EC004624FE500A0E0F90462C12D52D8026EA3A
:1045FC007007745D12D4CB801C75F06484ADF070C0
:10460C000FED75F00A847008E5F00E12D4BC80052D
:10461C001EED12D45108C3E55A9850B475A7002268
:10462C00030340A040030340E040D2D1E8C4F5822C
:10463C00E0FA797312468F30D146AF06532CF8ED61
:10464C00BFFF07F40460390FD262BF00331247C3B7
:10465C00402E797612468F30D126E5822403F582DE
:10466C00E0F512E0F513EEA2E713FEED13BEFF0723
:0A467C00F404600C0ED261BE0006CB
:104686001247E0400122C2D122C3E09709FDE0971C
:1046960009FEE097600904700AEE30E7068007EE2F
:1046A60030E703C2D122E546600E14600BF9EDCE69
:1046B600A2E713CE13D9F8FD227C007B44E54660C1
:1046C600207C007BCC1460197C017B981460127CE2
:1046D600037B3014600B7C067B601460047C0C7BCF
:1046E600C08C148B157AE9125371A8471255138C96
:1046F600168B1775C70075C6047510DF75B901E509
:10470600BC20E76FF51385BD1205C605C675B90150
:10471600532CF8C3E5BE9573FBE5BF9574FC05C63F
:1047260075B901E5BC9575FD5005D2621255FEC3FB
:10473600E5159BE5149CE49D40338C198B18C3E565
:10474600BD9576FBE5BE9577FCE5BF9578FD5005F2
:10475600D2611255FEC3E5179BE5169CE49D400DFC
:104766008C1B8B1A12478AE5322428401305C6E5AE
:10477600C68006E5C62404F5C6700205C7D5100135
:0F47860022024702AE19AD181246ACED1247C31E
:10479500AE1BAD1A1246ACEE13ED131247E0123EF6
:1047A500C4E54624FB50080E0F90463102D52D1E58
:1047B500E51312D4CFEE2404FEE51202D4CF75F032
:1047C500067FFDA946B9000575F0027FFF84C5F097
:1047D5002F500205F0C5F0FF24DE228547F0A430F6
:1047E500E70205F0E5F0A946B9000280050475F079
:1047F5000384FE24E022E537B4020122E537700286
:10480500D23964027002C239E53724FC799EE7602B
:1048150005640B600C22D27E20081E401C107F1000
:1048250022D27F2008134011107E01227537012204
:104835007537002039037537022275F9FF75FB00BE
:10484500800E75F9FF75FBFF801C2053F512487D1E
:10485500759E85759D2D801412487D759E84759D68
:104865002D800912487D759E83759D09C2AC75988A
:1048750052C26DC26EC26F2212166EC253E4F5F9B2
:10488500F5FB30340215FB22D2A47F3212DE37C28B
:10489500A412D9B612DD3F12DE20C214C215124889
:1048A5003F74C012DC6A74A312DC27748F12DC27F4
:1048B5001248D374C012DC6A75A7049048DD7F10D6
:1048C500E49312DC27DFF91248D375A70022E538F7
:0548D50012DC2774CA8B
:1048DA0002DC27A29494859C8080808080818380DA
:1048EA00819E8075A60A12489FD269D2ACE5A62499
:1048FA00FA500C306DF712DBBCB4E0F1124935C244
:10490A00ACC26975A6FF22D21EC274C273E4FDF559
:10491A0071F570C22D12483FD2AC12DBBCC5F070E3
:10492A0005DDF7C2AC22C5F0B4E0EFF538E4F532A4
:10493A0012DBB7A2E19273A2E2927475A704900403
:10494A00B4F012DBB7C2D1124B1C20690330740BCE
:10495A008D758E748F73E514C4F57D124B9C124BC2
:10496A001C20690330740C8D788E778F76E51425B8
:10497A007DF57D124B9CD2D1124B1CEEF0F55DEF0A
:10498A00F0F55C207303E4FEFF79BCA70609A707CC
:10499A0012DBB77D0A124B898F71EE60037571FFC6
:1049AA007D14124B89C22DED24F150010F240A50B7
:1049BA0002D22DBFB4027F008F7012DBB7F054070A
:1049CA00C52E54F8252EF52EE571700EE4F571F515
:1049DA0070C22D9004BFF0F0F0F012DBB7E538603A
:1049EA0009D21EC27412AF038005C21E12AEFF1294
:1049FA00DBB7B4E1FA75A7049004C412DBB7F0126E
:104A0A00DBB7F0F53A12DBB7F0F53B12DBB7F0F59E
:0B4A1A003C12DBB7F0F53D12DBB7F0FB
:104A2500F53E12DBB7F0F53F12DBB712DBB7B4E2A8
:104A3500FA12DBB7F07E0C12DBB7FF12DBB712DB25
:104A4500B712DBB712DBB720E1027F00EFF012DB14
:104A5500B7DEE412DBB7B4E3FA12DBB7FF12DBB75C
:104A6500CF60027F7F9004E4EFF0E4F012DBE79083
:104A750004D8124B8912DBB7B4EAFAC2AC75A704A5
:104A85009004DAE561F0E560F0E55EF0E57AF0E5E1
:104A950079F0E52EF0E55FF0E57BF0E551F0207467
:104AA50012E4F571F5709004B4F09004BDF0F0F0E7
:104AB500F0F0F075A70078ABA63A08A63B08A63C2F
:104AC500120E7BE5BF253D240C75F0188478AEA643
:104AD500F0186005640260182216E670121816E6D2
:104AE5007004760C181678ACE6904B0F9308F622F6
:104AF5000618E608904B0F930466700D76011806AC
:104B0500E6640D70047601180622001F1D1F1E1F86
:104B15001E1F1F1E1F1E1F12DBB7FC12DBB7FD1267
:104B2500DBB7FE12DBB7FFECA2E692E7921713FCA8
:084B3500ED92E713FDEE92E79B
:104B3D0013FEEF92E7301701F4F513ECA2E713FC27
:104B4D00ED92E713FDEE92E7301701F4F512ECA2AA
:104B5D00E713301701F4F510ED92E7301701F4F576
:104B6D00111255A620D10E8C1C8D1D8E1E8F1F125D
:104B7D00B30B1255A630170312B2E52212DBB7C3E1
:104B8D0013FEF012DBB792E7FFF07C0002547CAC11
:104B9D001CAD1DAE1EAF1F30170312B2E5ECF0EDCC
:104BAD00F0EEF0EFF022124BBC0202C612BC73C243
:104BBD00101248F07F5A7E0590A3FA12770212DD8B
:104BCD003FD214D215C255122CEC789F7680087600
:104BDD000012BCB31232FA7570FE853A71853B72C4
:104BED00853C73853D74853E75853F7612BD1212E9
:104BFD0032FA7570C0757B03757A54E4F57FF57ED6
:104C0D0012BD12751421751348755F01757B007502
:104C1D00750475745275780175776CE4F57DF551F1
:104C2D00757F0190DF5C85836E85826DC23D124C70
:104C3D009A851C1D75A6FF305505C221022EA7129F
:104C4D004C9AE572A2E59275A2E79277D274D2736F
:104C5D00E51275F008A4AEF0FF2075031255E612AB
:104C6D00C79B12C7E4124D1DE51C251D13F571855B
:054C7D001C1D12BC8BA0
:104C820012BCE3757F02E56A70B57F5A7E2FE5415B
:104C920012D3B612DD3F80A7856E83856D82C25521
:104CA2007873124CFE7876124CFEE493F570B4B42D
:104CB20002D255A3E493F51CA3E493F512A3203D7D
:104CC2000FA97BE493F57BC399502A20E702055F85
:104CD200A385836E85826D103D16D23DE582240543
:104CE200F582E43583F583E493F52654F0F57222D8
:104CF200E526C480F630E7D8155F80D48601E493B8
:104D0200F6A308C399500A20E70606B60002080671
:104D12002230E70616B6FF0218162230750DE5138B
:104D22002579F513E43514F514800DC3E51395794F
:104D3200F513E5149400F514AE14AF137C007D0A4C
:104D420012547C8E5E8F7A22124DDF851617203D1B
:104D520001227F5A909C831276F07F64E5166404E8
:104D6200700C909C9B12773312DD3F02DE1A909CEE
:104D72008F1276F07F6E7E0890A5ED127702121EDA
:104D82000312DD3F7515B87514047F6E7E20C224B0
:104D9200A815E82404F9C23DE7124E27203D06E695
:0A4DA20012D5018008E6128460E8D3
:104DAC00A815F60515EE2406FED514DA851716128D
:104DBC001E5112DD3F10000510018D80F878B812DD
:104DCC000E8F86BC0886BD0886BE0886BF124EE6CE
:104DDC0012DF15120E8FC23D75160078B87F4B7E10
:104DEC000890A5ED1277027E20E5BC12D501124E7B
:104DFC001E7E26E5BD12D501124E1E7E2CE5BE127E
:104E0C00D501124E1E7E32E5BF12D501124E1E0286
:104E1C00DD3FF608080808F618181824D0500524A9
:104E2C00F64001220516D23D2275C70375C6FE1247
:104E3C00766E124EE675C6FC75BC2675BD6475BEE5
:104E4C00A975BF70124EE675C6FB12766E124EE651
:104E5C0075C6FA75BC1475BD1475BE0075BF0C1201
:104E6C004EE675C6F975BC4E75BDBF75BE0075BFF7
:104E7C0019124EE675C6F875BC0A75BD7E75BE0076
:104E8C0075BF01124EE675C6F775BC0175BD23756D
:104E9C00BE4575BF67124EE675C6F675BC0275BD8C
:104EAC00AB75BE0175BF01124EE675C6F512766E76
:104EBC0075BE0275BF0A124EE675C6F412766E7593
:104ECC00BCE1124EE675C6F312766A124EE615C6B2
:104EDC00124EE615C6124EE615C675B90575B90221
:104EEC0022751500127D6775B901E5BC64816003FC
:104EFC001276510515E515242050E975C70375C6C2
:104F0C008075B90505C6E5C6241C50F5124F1E0266
:034F1C007BBDE476
:104F1F00F5C7F5C6742612766F75BD4E124F38124F
:104F2F004F35E4124F3512766F124EE605C6227FCB
:104F3F00357E00E54B12D46D7E10E54C12D46D7E9C
:104F4F0020E54D12D46D7E30E54E12D46D227F4692
:104F5F007E00E56C12D46D7E10E56B12D46D7E2051
:104F6F00E56A12D46D7E30E57F12D46D2220740174
:104F7F0022D24475A700758307E559C454F024075E
:104F8F00F582E0F51A244C40E7A3E0F512A3E0F513
:104F9F00131209208938120E67E5BDA2E0923BE596
:104FAF001A40069570500224B4F51A203B05D2061C
:104FBF0012CA9EE51A1250DFE5152437F51DE435A8
:104FCF0014F51CE5172437F51FE43516F51E85CCAF
:104FDF0012853813AC12AB137A0412536375380170
:104FEF0024FA401A05382402401405382401400ED3
:104FFF000538053824014006053805380538C3E55E
:10500F001A945A500224B4F51AC23BC23CC23D75E1
:10501F001B00A23B823C406D203B2CE51A75F0082B
:10502F00A4951BFBE5F0303D04940180029400FC35
:10503F005008EB24A0FBEC3405FC1250E6125095FF
:0A504F00923B40031250B8203C2CA5
:10505900E51A75F008A4251BF9E4303D010435F083
:10506900FAE994A0FBEA9405FC5004AB01AC0212E6
:1050790050E6125095923C40031250B8E51B253872
:10508900F51B5094203D04D23D808D22E51F251744
:10509900FEE51E35167016EE24914011E51D251505
:1050A900FFE51C35147006EF2491400122D3228EAE
:1050B900027C8A7B3B125371ED2402FE8F027C8AAB
:1050C9007B3B125371ED2439FF02DE5A1256CF8011
:1050D900311256C2804675F008A4ACF0FB75190070
:1050E900C3EB9468F9EC9401FA40080519AC02ABDA
:1050F9000180ED8C108B11531903E51920E0CD12B5
:1051090056C212513AAF05E51924FE50031255E66D
:105119008E168F17E51920E0B81256CF12513AAF03
:1051290005E5191460061460031255E68E148F15EF
:1051390022AC06AB07AA12A9130253DC125227208C
:105149003D4974857F227E0812D5017E0830173CBF
:10515900AC1EAB1FEB2418EC34FC402F125342E574
:105169001B60077F207E0812D51C7F207E10E51A60
:0951790012D51C7F237E17742E51
:1051820012D4FD7F207E1BE51B7011E519C2E012CF
:10519200D51C227F207E0E740A02D51CE51975F0FB
:1051A200058475F005A402D51C125227203D5E74B9
:1051B200857F227E3A12D501301753AC1EAB1FEB0E
:1051C2002418EC34FC4046EC7033EB249C402E7ED9
:1051D2002D125219125585C0E07F2A7E2EEB12D570
:1051E2001C7E39D0E0C2E012D51C7F347E3712DE3D
:1051F2005A1E12DE5A1F12DE5A0E02DE5A7E30127A
:105202005219125585EB7F2A7E3112CE40227F2A17
:105212007E39740A02D51C7F2912DE8A0FBF34F947
:105222000EBE40F322D23D301266120E71E5BDF57C
:105232001C75F00AA4F824E15002781EE4FCFBFE7F
:10524200FFC23D12BE6E125293203D44D8F8751D26
:10525200CEE51C146009751D9C146003751D6AC29D
:1052620017EC30E705D2171255F68C018B00E9488E
:105272007003D23D22EE7008EF251D4003D23D227D
:10528200AC06AB077A1C1253711255158C1E8B1F7C
:1052920022203D07123C767003D23D22056D12BCDE
:1052A20034E4F5F7C2B2C2B2ADF7F5F7C2B2C2B298
:0252B200E5F71E
:1052B400FAD2B230E4E3ED2FFFE43EFEE56D2408BC
:1052C400F56D12BC34E4F5F7C2B2C2B2ADF7D2B296
:1052D400EA30E508EB2DFBEC3400FC22C3EB9DFB2C
:0552E400EC9400FC2227
:0100030055A7
:10DF5C0069FC362E06FD69FC372F071169FD383038
:10DF6C0007FD69FD3931061169FE383107FD68FE80
:10DF7C003732091168FF373008FD68FF372D07115C
:10DF8C006800362909FE680036290C116801372B08
:10DF9C000CFF6801372F0A116802383009FF68023C
:10DFAC00372E08116803372C0AFE6803372E081128
:10DFBC006704373208FE67043633091167053535B7
:10DFCC0005FF6705353303116706362F02FF670619
:10DFDC00362B05116707362B07FF6707352F051101
:10DFEC006708353104FF6708332E0511670931289E
:10DFFC000700670931250A11670A35240B01670AE6
:10E00C003A240A11660A3C210801660B3D1E0B11CD
:10E01C00660B3D1E0C00660B3D200A11660C3B2165
:10E02C000CFF660C39220E11660C37231100660D9D
:10E03C0036240D11660D34260F01660E3226111191
:10E04C00660E32251401660F35251311660F37271E
:10E05C0016016610392918116610392B1502651135
:10E06C00392D11116511372E0C026512332F081141
:10E07C006512312F07026513302C0A1165132D29F7
:10E08C000E0265132A271011651429270E02651438
:10E09C002C290C1165153129080365153726071134
:10E0AC006515321F09036516411B09116516411CC4
:10E0BC0008036416461F081164164D2105046416E6
:10E0CC005922031164166425040563156A2407118B
:10E0DC0063156D23090663156C230D1163156C25EF
:10E0EC00130762146E2B151162146E2F1406621333
:10E0FC006E30161162136E30150761136F311211E9
:10E10C0061126F350F0761126F380D116011723A81
:10E11C000A086011763F0611601079420209600FFF
:10E12C007A3A0533600F7832040A5F0F742C01338E
:10E13C005F0E722B030A5F0E732E08115F0E743084
:10E14C00050C5F0D722C02135E0D6C2B010C5E0D19
:10E15C00622C05315E0D5F2B030D5D0D5E290833BE
:10E16C005D0D5F23030B5D0D5F1B01335D0D5A16B7
:10E17C00020A5D0D521B00115C0D4D26000C5C0E4D
:10E18C00462802335C0E3926040C5C0F2C2B08330A
:10E19C005C0F23320C0F5D0F172E0A335D0F0C2E04
:10E1AC0009105D0F043507335E0FB23C080F5F0F8B
:10E1BC00AB4209335F0EA43E070F5F0EA2430B3335
:10E1CC00600EA746120B600D9F490C73610C9C49A5
:10E1DC000F0C610B97460973610B8B440A0C610A97
:10E1EC008B420B336109843A080C6108823A043380
:10E1FC0061087934030C60086F2F063360086228BD
:10E20C00050C6008572505336008511F040D5F0885
:10E21C004E1B05335F08491B090D5F094120103760
:10E22C005F0938270D0D5F0A302F06335F0B2B3239
:10E23C00070F5F0B282F0A335F0B262E0E0E600C78
:10E24C0023361137600D1F3F160F600D18411277E2
:10E25C00610D0F320A13610D042B0633610D022E72
:10E26C00040E620D043A0231620E0343050D630D78
:10E27C00B1470113630DA94A000B640CA14D0511A4
:10E28C00640C9B44070E650B99490911650A944768
:10E29C00090D65098E49021365088848060D650845
:10E2AC0081400E336407793B130F6407722F187784
:10E2BC0064076D231A106407692911776407651CBC
:0DE2CC00080F63075D180B33630751190D30
:10E2D9000D630746220E336308402B110F6308387C
:10E2E900291837630932271B0D6309312B1477620B
:10E2F9000A372C0F0A620A3C280973620A441E0B6A
:10E309000C620A48150E33620B46190C0A620B4758
:10E31900260D33610B4C280C0B610B54251037610A
:10E329000B5E24170C600B63291A77600A66361492
:10E339000A600A68390B735F0A6C2C100A5F09724C
:10E349002015775F097422120A5F0873300F775F0F
:10E35900087639140A5F077D3816775F0785370F06
:10E36900095F068D3B0D735F058B4410075F048BB6
:10E37900490C735F048E3F0C075F03863604335FD5
:10E389000394280708600299300E1160029E400527
:10E39900076102A34A0C336101AA4810086201B15E
:10E3A90042127762020131150A6202062B13776362
:10E3B900020830110C63020B361277630310331114
:10E3C9000C6403182B147764032223110A640426AE
:10E3D90023107764042226110A64051C2715776423
:10E3E900051D251508640521271277640628270FBE
:10E3F9000764062F1D11776406350F140764063E5E
:10E409000A19776406401216086407431B117763DB
:10E41900074A22120663075228127763075A2713FD
:10E429000662075E2314776206612011076206649B
:10E439001E0E7362066A1E0E076206742110376289
:10E44900057828130661057A2F157761047A332038
:10E459000661047A301B7761037A281B0761037F01
:10E4690023187761028429160661028832177761B9
:10E47900018D371305610193340C7362009A2E09DB
:10E489000562009D2E043362009D370C0663FFA0D0
:10E4990040103763FFA844140564FFAF4612776440
:10E4A900FF014511056500043F12776500053E101F
:10E4B900076600073F117766000B430D07670110D8
:10E4C9003D117367011539120767021A321277670E
:10E4D900021A2C12076702192C107768031B2E0FDA
:10E4E9000668031F2C117768042729100468042E75
:10E4F9002A0F776705322F130467053330127767C0
:10E5090006362D140567063B291677670643231B34
:10E51900046706471E16776607491E150366074CEA
:10E529001B157766074C2217046607522214776574
:10E53900075B26150265066229157765066D291799
:10E549000165067529137765057D281A0265058217
:10E5590028187765047F1F160265048F2A117765CD
:10E5690003953211006602993D157766029C401C9D
:10E57900FF6602A13E1F776701A43F1CFF6701A741
:10E589004314776801AB4710FF6901B1490F7769F7
:10E5990001024911026A0207490D736A020B480C0C
:10E5A900056B030F480B336B03144A0D026B0419F7
:10E5B9004914376B051F491CFE6C06224824776CE9
:10E5C90006233F21FC6C07203023776C0721272184
:10E5D900FC6C07262420776C08292812FC6C082873
:10E5E9002C0F776C0927230CFF6C09251802316C55
:10E5F90009350F05FC6C094C1401116C09561D01F4
:10E60900FC6B095F2003136B086B2108FB6B087413
:10E619002509336B08772507FC6B0778210D336BC8
:10E62900077A1E0AFB6B077F220C336B06832E0ABF
:10E63900FA6B05853C09336B0489410EF96B048C2F
:0DE649003E10376B038D3C0FFA6B038D40C4
:10E6560013776B02904112FA6C01934110776C01AB
:10E66600984410F86C009B471A776D009F461EF879
:10E676006DFFA24519776EFFA14019F86EFFA640FF
:10E6860014776FFEAA4417FA6FFEAF4A127770FE30
:10E69600B34D18FA70FF024B1B7771FF054718FD43
:10E6A60071FF0942177772000E4012FD7200163D87
:10E6B6000C7372011B3510FA7201232E1577720244
:10E6C60029321AF872032C371D7772032F3014F88B
:10E6D600720336210F77710346190DF87103502026
:10E6E6000B33710353290EF87003572B143770033D
:10E6F600612712F870036F2911777002793017F7C6
:10E706007001803722777001843D1FF67000883FC4
:10E71600197770FF8D3F11F670FF933D0C7371FEF4
:10E72600973D0EF571FE9B3E0C3372FD9F4310F62E
:10E7360072FDA448127773FDAB4C13F573FDB14F10
:10E74600167774FD034F14F775FE074C127775FEA6
:10E756000A4510F975FE0E400F7776FF124111F843
:10E7660076001745167776001C4614F67601214288
:10E7760017777602263D17F3760229382177760336
:10E786002A3315F276032B3009737604302A07F004
:10E79600760439220A337604472110F07504512590
:10E7A60012777504552416F1750459210F777504EF
:10E7B6005F2111F0740463231477740468240EF245
:10E7C600740370230933740379270AEF74028030C7
:10E7D6000B33740185360DEF74018B3913377400D2
:10E7E600903D1BF075FF94441E7775FF984823EF04
:10E7F60075FE9B46207776FE9F4221F076FEA13F6E
:10E80600177777FDA44313EF77FDA747157778FDB4
:10E81600AA4915EF78FDAD4C157779FDB04D19EE87
:10E826007AFDB34D1C777AFD024E19F07BFD054F3C
:10E836001B777BFE094F24F37CFE0D531D777CFF6F
:10E84600114619F37CFF173F12777C001F3810EF33
:10E856007C00263613777C012B3115ED7C012F2B9E
:10E8660015777C02332513ED7C02392214777C025E
:10E87600402110EE7C0249210B737B02531F0FEBE4
:10E886007B02601E15777B026A2214EA7B017428DC
:10E8960019777B017B2D1AEA7B00833122777B0077
:10E8A6008A3320EB7BFF91371A777BFE953C1FEA74
:10E8B6007CFE983C26777CFEA74621EC7CFD9939A8
:10E8C60023777CFC9A3B1FEA7DFC9A3F1C777DFBF5
:10E8D6009A401EE87DFB9B3F20777EFA9B3F1FE612
:10E8E6007EFA9C431A777EF99E4717E57FF8A04A81
:10E8F6000E737FF8A34A0AEA80F8A548073380F822
:10E90600A94402EA81F8AE46041182F8B24C00E747
:10E9160082F80351021183F8085304EA83F90E4D75
:10E92600061183F914430CEC84FA1A400E1184FB89
:10E93600203F0AE884FC2540061384FC2B4008E6A9
:10E9460084FD3039073383FD36300EE483FE3C2BDD
:10E95600193783FE402A1EE783FE3D25187783FE7E
:10E96600371B16E783FF3114137783FF35170FE440
:10E9760083FF3E220D738200412C15E58200432C55
:10E986001A77820046251BE782004C201577810006
:10E99600552116E581005E2510778100682718E469
:10E9A60081FF72291E7780FF7A2E22E580FE7E3057
:10E9B600277780FE812B22E680FD85251C7780FD4A
:0DE9C600882618E281FC8A2F187781FC8DCD
:10E9D3003821E181FB903F287781FA924025E0813D
:10E9E300FA943D237782F9973C18E082F99A3F1510
:10E9F3007782F89E4412E083F8A347107783F8A741
:10EA03004A0CDF84F8AA4D133785F7AC5214E2851C
:10EA1300F7AF56107786F7B2580DE087F802560223
:10EA23003387F8055002E388F8094C051188F90C7F
:10EA33004E02E489F91052011189FA155004DF8955
:10EA4300FB1D45041389FB233304DE89FB292306BD
:10EA53003389FC2B1F05DE89FC2F23093389FD3302
:10EA6300280ADC89FD3B23103788FD471E0EDD880D
:10EA7300FD511E0E3388FD53200CDD88FD54210B00
:10EA83003387FD57200DDD87FD5C20093387FD5D4E
:10EA93002403DE87FD5B29013386FD592C04DE86C2
:10EAA300FD5D2C093385FD622F0CDC85FD652D0B87
:10EAB3003385FC672908DF85FC6722093385FC6BF6
:10EAC300210CDD84FC72280A3384FB783005DD8455
:10EAD300FA7C37073384FA7E390ADC84F9813B06F2
:10EAE3003384F8843F05DB84F8873F023384F78A55
:10EAF3003C04DB84F78D390A3384F6903908D985D1
:10EB0300F5923F113785F595430FD985F498440A5B
:10EB13007386F49B440AD986F39C440C3386F39C96
:10EB23004507DA87F29C47063387F19E4C0AD9885A
:10EB3300F1A251103788F1A65516D989F0A7571FAE
:10EB4300778AF0A9541BDA8AF0AA4D12778BF0ACBE
:10EB5300460DDB8BF0AC4906338CEFAB4D05DB8CFC
:10EB6300EFA95002318DEEA85209E28DEEA7530EA4
:10EB7300118EEEA75316E58EEDA44A20118FEDA05A
:10EB83004423E28FEC9C4821118FEB9A4A22E090B8
:10EB9300EB95411D1190EA8E391DDF90EA893621EC
:10EBA3001190E9873223E590E9852C2C118FE87DBC
:10EBB3002A26E08FE8762124118FE8662122E08F50
:10EBC300E856221F118EE947201DE08EE9392116F0
:10EBD300118EE9302518E28EEA2D2917118EEB30BC
:10EBE3003213E18EEB333711118EEC373C10E18E8B
:10EBF300ED393E07138DED3B4203DD8DEE3B3E09C0
:10EC0300338DEE3B310DDE8DEE392812378DEF3823
:10EC13002319DC8DEF382A18778DF0372A12DC8D13
:10EC2300F0382214778DF0361B0EDC8DF1361B0C79
:10EC3300338CF1371F0DDB8CF136250E378CF23414
:10EC4300270CDC8CF22A270D338DF31F2A0CDC8D65
:10EC5300F3173409338DF4143A08E48EF4123A0CA2
:10EC6300338EF4103D11EA8FF50E411A778FF50CB0
:10EC73004917EA90F50A50157790F5054F13E79178
:10EC8300F5B24F107792F5AD5408E492F4AB5A0104
:10EC93003393F4AB5C05E893F4A9500A3394F3A4DB
:10ECA300450CE094F3A041093394F29A3A05E295B6
:10ECB300F29734043395F1913208DC95F19E310DCE
:10ECC3003395F08A320CDA95F0872D0B3395EF806C
:10ECD300250EDE94EF73220C3394EF6C2412DD9433
:10ECE300EF6928157794EE6B2812DF93EE69280EEF
:10ECF3007393EE64270DDF93EE5C260B3392EE578E
:10ED0300270EDB92EE5828123792EE5E2610DB9226
:10ED1300EE64240D7391EE6C2108D991ED722304F6
:10ED23003391ED782904D991EC7C320A3391EB7F4E
:10ED33003A08D891EB833D093391EA883C0CD7918B
:0DED4300E98D3B103791E9903E12D792E820
:10ED50009143137792E794420ED792E7993E073397
:10ED600093E7A03901D993E7A63B0A1194E6A83F9F
:10ED70000CD794E6AB490E1195E6AE4F07D695E653
:10ED8000004D011396E6034601D996E6033E0811AD
:10ED900097E7043D0ED997E70740151198E70C4314
:10EDA00012DA98E812460F1198E918490CDA98E936
:10EDB0001D44081198EA243D05D898EB293A03111F
:10EDC00098EB2C3707D898EC2D38093398ED2E3D69
:10EDD0000ADC98ED2E3E0A3398EE2D3F0BDB98EFC0
:10EDE0002C420C3398F02B430ED998F02B3D113761
:10EDF00098F12D3710D898F130340D7398F23433E0
:10EE00000FD698F237330F7798F339331CD597F331
:10EE10003C32167797F43E2F11D797F440280973A8
:10EE200097F4422109D797F4461F0AB396F44B2171
:10EE300008D796F45325083396F45C2505D796F445
:10EE40006723023395F4722503D695F3782B0231AC
:10EE500095F37B3102D695F27E31063395F1832FFF
:10EE600004D695F18A2F023395F0913201D596F0B0
:10EE70009638061196EF9A3F02D497EF9D450213FC
:10EE800097EE9F4704D497EEA247073398EEA64427
:10EE900008D398EEAA430B3399EEAD440CD499EE07
:10EEA000B1400D339AEE013F11D39AEE054512772A
:10EEB0009BEE064A15D59BEE064712779CEF05425E
:10EEC00012D79CEF063E0F779DEF084111D39DEFBF
:10EED000094619779EF00B4718D39EF00D431C7717
:10EEE0009FF10F4015D69FF1114113779FF2134602
:10EEF0000ED9A0F2174A0B33A0F31C4A08D4A0F491
:10EF000023420333A0F42A3305D3A0F53127071198
:10EF1000A0F5382300D29FF53D2702339FF6442900
:10EF200003D39FF64F2808119EF55E2807D19EF562
:10EF30006C2D04119EF4752F01D09EF47C2D0433AA
:10EF40009EF3822B04D09EF3872E05119EF28B3503
:10EF500007D09EF2903D01119FF1954203D09FF0A2
:10EF600094400333A0F09F3F0BD0A0F0A13D0F379A
:10EF7000A0EFA33C0DD1A1EFA43C0C33A1EFA43C26
:10EF80000AD0A1EEA53D0533A2EEA63C00D1A2EE2B
:10EF9000A8390211A3EEAA3C04D0A3EEAD3F05119F
:10EFA000A4EEB24008D0A4EE03410C11A5EE064138
:10EFB0000AD2A5EE08450711A6EF094A05D2A6EF29
:10EFC000094C0111A7EF0A4807D3A7F00B420B1118
:10EFD000A8F00B420DD4A8F00D461311A9F111466B
:10EFE00014D9A9F1173F1B11A9F21E381ADAA9F397
:10EFF00021381811A9F31F3A17DFA9F41839151190
:10F00000AAF4163A1DDCAAF5183C1A11AAF51C3A06
:10F010001AD9AAF61F391A11ABF6203615D9ABF753
:10F0200021341711ABF8203B19D9ABF81E3F17114B
:10F03000ACF91D4011D9ACF91E3F0E11ACFA1F40BE
:10F040000CD6ACFB22410D11ACFC23450FD6ADFC18
:10F0500023490B11ADFD214A0DD6ADFE2047091104
:10F06000ADFE21450CD6ADFF22430E11AE00224568
:10F070000CD8AE01214B0A11AE0220500DD7AF03C0
:10F080001D4F0B11AF031A5109D9AF04174A0D11C7
:10F09000B00418470BDBB0051A500A11B0061C5516
:10F0A0000ED7B1071C560B11B10719470ED9B1087D
:10F0B000173C0C11B208183D0CDCB2091C490E11AA
:0DF0C000B20A1E4E0AD9B30B1D500B11B33E
:10F0CD000C1A5109D9B30C174F0711B40D17490B71
:10F0DD00DBB40D17480D11B50E19490ADCB50F1922
:10F0ED004F0B11B50F185605DBB61017550711B696
:10F0FD0011174C0ADBB61116430B11B711173F0D43
:10F10D00DDB71219430C11B7131A480BDCB8131ADB
:10F11D00450F11B81419410DDCB81418400B11B975
:10F12D001518430DDBB91618470F11B91618490DEF
:10F13D00DBBA1718470A11BA1717450CDBBB1814A1
:10F14D00460F11BB18134C0EDBBC1912510A11BC22
:10F15D001A125007DBBC1A12470B11BD1A10400DC5
:10F16D00DCBD1B10400A11BE1B124509DCBE1C156F
:10F17D00490B11BE1D184A0ADBBF1D1B4A0811BFE2
:10F18D001E1B480CDBBF1F1A470E11BF1F1A490B60
:10F19D00DBC0201B4B0D11C0211C4910DBC0211DF4
:10F1AD00470F11C1221D4711DBC1231C4B0F11C18C
:10F1BD00231B4B0EDBC22419441111C224193D0F20
:10F1CD00DBC2251B3B1011C2261D3F0DDAC2261EC8
:10F1DD00411011C3271D3F12DAC3271C3D0F11C368
:10F1ED00281B3D10DBC4291C401111C4291C450FDF
:10F1FD00DCC42A1C460E11C42A1B4510DCC52B1974
:10F20D00431111C52C184511DDC62C164A1011C617
:10F21D002D174A11DEC62D18491211C72E19471088
:10F22D00DEC72F1A460E11C72F1C4410DFC7301F23
:10F23D00471111C731214B0CDBC832224D0E11C8BD
:10F24D0032224A10DAC83321471111C83420460F33
:10F25D00D9C83520461111C93521430CDBC93623D8
:10F26D003F0F11C937253D11DBC93725400E11C997
:10F27D0038254211DCC93925431311C939254312EB
:10F28D00DCC93A25431111CA3B24400DDCCA3C248C
:10F29D00411011CA3C23400EDCCA3D22401111CA57
:10F2AD003E20420FDECB3E20451011CB3F204714B0
:10F2BD00DECB4021441211CB40213F10DFCB412248
:10F2CD003C0D11CB42234011DFCC42233E1111CC1A
:10F2DD0043202F0EE0CC4319221211CC43122011E2
:10F2ED00E3CC4311250E11CD43132B10E3CD441266
:10F2FD002D1111CD440F2B0FE3CD44092B1211CE3F
:10F30D004404320FE2CE4401360E11CF44B3370D13
:10F31D00E0CF44B3330E11D04401370EE0D0440595
:10F32D003D0D11D0450A3B0CE3D14512330D11D1E2
:10F33D00451A2D0EE3D1461E2B0F11D1461D2E0F52
:10F34D00E4D1471D300F11D1471E320EE3D24821B3
:10F35D00330F11D248233510E2D24923350F11D284
:10F36D004A20360EE3D24A1D360E11D24B1B3410F5
:10F37D00E3D34B1B320F11D34B1B300EE4D34C1B7D
:10F38D00340D11D34C1B3A0DE5D44D1A3B0E11D44F
:10F39D004D1B360AE6D44E1D340E11D44E1E360DBD
:10F3AD00E5D44F1F360C11D5501F350EE5D5501F26
:10F3BD00340D11D5511E340EE5D5511E370C11D516
:10F3CD00521E390EE5D652203B0F11D653223C0F5B
:10F3DD00E4D65423391111D654243710E3D65524CD
:10F3ED00360F11D655253310E3D65626330D11D6CB
:10F3FD005627350BE2D657273A0C11D658273C0F16
:10F40D00E2D75827391011D75927370FE2D75A2786
:10F41D00381011D75A283B0FE2D75B293C1111D771
:10F42D005C2B3C12E2D75C2D391111D75D2C3910B4
:0DF43D00E3D75E2B3C0F11D75E293B0EE399
:10F44A00D75F27371011D75F26360EE3D760273CE0
:10F45A000E11D761284310E3D76229451111D762EB
:10F46A00293F0FE4D763283A1011D763293A11E4E8
:10F47A00D7642A3E1011D7652C4211E4D7662E4272
:10F48A001011D7662D3F11E4D7672F3A1011D768AC
:10F49A002D3B0CE4D7682E3D0711D7692E4204E4B0
:10F4AA00D76A2E470111D76B2E4702E4D76B2D403E
:10F4BA000513D76C2B3503E4D76C2A2B0711D76DAC
:10F4CA002B2909E5D76D2B300611D76E2A3A04E4A9
:10F4DA00D76F28400611D76F283E08E4D77027381F
:10F4EA000C11D87026320DE6D871252F0911D87162
:10F4FA0024310AE9D87221340811D8721B3A08EA71
:10F50A00D9730D420A11D973104909EADA730C4505
:10F51A000811DA730A3B06E8DB74093D0211DB7451
:10F52A000A4003E9DB740B3C0213DC75103406EA6B
:10F53A00DC7517350333DC761A3F06EADD771C469D
:10F54A000433DD771F4001E8DD7824360731DD78A2
:10F55A002C3206E7DC7933320413DC79373409E7D5
:10F56A00DC7A3A340C33DC7A3C3508E7DC7B3D370D
:10F57A000233DB7C3C3A05E7DB7C3C3D0333DB7D35
:10F58A003B3A04E7DB7D3B320331DA7D3E2D09EA63
:10F59A00DA7E43270D11DA7E4D230AE9DA7E5726F1
:10F5AA000B11D97D5E2C0BE9D97D61300C11D97D07
:10F5BA00632F08EAD87D662F0511D87C683005EAE2
:10F5CA00D87C6D330611D77B733608E9D77B7C3834
:10F5DA000511D77A853A04E8D8798B3B0711D8798F
:10F5EA008E3809E9D8788F371011D878903B0BE814
:10F5FA00D87791420D11D976954A08E7D976984974
:10F60A000411D9759D4008E8DA75A23A0B33DA7508
:10F61A00A53C0AE8DB75A8430031DB74AA4603E976
:10F62A00DC74AF460213DC74004A02EADD75054C4D
:10F63A000333DD75084D00EDDE75084B0533DF76C3
:10F64A00064902EDDF76044A0131E076044902EA0E
:10F65A00E076044C0513E176045006EAE176014DA2
:10F66A000D33E276B1450FEAE276AD3F1077E375E6
:10F67A00AB3F0DEAE375AC430A33E475AE4604EAE0
:10F68A00E475B0400131E575B23908EAE575013C27
:10F69A000611E675054607ECE6760A4B0311E7768E
:10F6AA000F4604EEE777163B0611E778203405EC9F
:10F6BA00E77827350611E7792D3409ECE7793234F2
:10F6CA000B11E77A3B260AECE67A45250B11E67A16
:10F6DA004D230BEAE67A56250711E67A5F270AEAEE
:10F6EA00E579672A0C11E579731F0AEBE578792E1B
:10F6FA000811E578843302EAE5778D3B0313E67651
:10F70A00954104EAE676993F0733E6759A3801EAA5
:10F71A00E67595310531E6748F3202EAE6748E3564
:10F72A000111E773923301EAE77398310413E77220
:0AF73A009D3304EBE872B4370911A7
:00000001FF
